:10B6E800414952434F54454300405053332E35305F
:10B6F800404E4C20004143435500532F4E214641B4
:10B70800494C555245005245454E54455221532FF8
:10B718004E00434F4E5441435420414952434F54E5
:10B7280045430047505300403244400040334440B2
:10B7380000554954214E4557404D454E55000A166F
:10B74800000180000300007E0000FE00001E0000D3
:10B75800360003E60001C4000000000FFFE0205A95
:10B768004F454B40534154532000204750534056B7
:10B77800414C49442000404B4559320050494354FC
:10B788005552450052414E4B494E47004D415020BD
:10B79800202020200043454E544552202000564189
:10B7A80052494F202020004241524F4752414D00FC
:10B7B800524F55544553202000444943485453544C
:10B7C80045005741595054532020004D41524B5386
:10B7D8002020200044454641554C5400202020217B
:10B7E80047454D21202020204146530020545241F6
:10B7F800434B214F4E20200020545241434B214FB0
:10B80800464620004D41524B0020545241434B2D97
:10B818005550212000204E4F5254482D555021207C
:10B82800002154455255470153454C40524F5554F9
:10B83800450153455420484F4F47544501564C55F0
:10B84800434854454E686901574159505453202084
:10B85800686901524F555445532020686901414990
:10B86800525350414345686901494E5354454C2051
:10B8780020686900414343454C45522E6869005A87
:10B88800455420484F4F475445004241524F404885
:10B898004F4F4754450047505320484F4F47544552
:10B8A80000514E4820202020402148504100464C5D
:10B8B800004C4F47424F454B204C45454720003EE2
:10B8C800215445525547002154455255470153507C
:10B8D800454C454E015A454E440157495353454E30
:10B8E800002154455255470120555342204F4E4C94
:10B8F800592001544E432031232035374B01544EF3
:10B908004320312320392E3601015057434031302E
:10B91800234035374B0150574340313023403139AC
:10B928004B01014D5850403130234035374B014DC4
:10B9380058502034232035374B014D58502031239F
:10B948002035374B014D5850403130234031394B69
:10B95800014D58502031232031394B002154455294
:10B968005547014E494555572057505420014544E5
:10B9780049542057415950540157495320205741A1
:10B988005950540101434F4D3A014F4E5456414EC0
:10B9980047205750015A454E4420574159505401A9
:10B9A8005A454E4440414C405750200101414653AE
:10B9B800542057502D57500157495340414C405738
:10B9C80050542000504549202141465354005341CA
:10B9D8005645200041435455454C4540504F532E41
:10B9E800004F50534C41414E202020002053544FCB
:10B9F80052452157505420002046554C4C200021D8
:10BA08004057495353454E0053455220004952442C
:10BA18004100555342200055534220004C4953548D
:10BA2800005A454E4400205452414E534D4954202B
:10BA38004552524F52200021544552554701534513
:10BA48004C40524F555445014E4945555720525484
:0DBA58005020014544495420524F5554459B
:10BA6500014F4D4B4552454E2052540157495320E5
:10BA7500205254502020015749532020524F5554ED
:10BA8500450143594C2052414449555301434F4DBB
:10BA95003A014F4E5456414E47205254015A454E95
:10BAA5004420524F55544501434845434B20525479
:10BAB5000053454C21524F555445004E4945555765
:10BAC50000204E574540504F5340210021404F4DD7
:10BAD5004B4552454E40004F4D4B45455200214088
:10BAE500574953405750545300214057495320520A
:10BAF5005445004E494554204C45454720002140BA
:10BB05005A454E444052544500202052414449551F
:10BB15005300215445525547014C4F41444043542D
:10BB2500522150430156494557404354520144451B
:10BB35004C40414C4C214354520101434F4D3A0175
:10BB45005245435620204354520153454E4420202C
:10BB55004354520056494557204354520020204D26
:10BB65004F56450020204D4F564520544F00534316
:10BB7500414C452020582F59202045584954004311
:10BB85004C522044495354004155544F43454E545B
:10BB9500004155544F204F46460020202053434135
:10BBA5004C450044495354204B4D004449535420BF
:10BBB5004E4D0021544552554701564152494F209B
:10BBC500202068690158432D534554202068690198
:10BBD5005254452D5345542068690147454E4552F9
:10BBE500414C206869015049435455524553686991
:10BBF500010101454153592D5345540146414354D3
:10BC05004F5259534554210144454D4F464C4947E0
:10BC15004854002154455255470153494E4B544F02
:10BC25004E450153494E4B212D0153494E4B404D35
:10BC35004F440153494E4B40494E560156415220FF
:10BC45005443402020402301564F4C554D45015645
:10BC55004152494F204E554C4C01504954434801DF
:10BC6500504552494F4401564152204156402030DB
:10BC75004023014E4554544F2D01534F554E4443D7
:10BC85004845434B0053494E4B21544F4E450053B5
:10BC9500494E4B54214F4646004745454E20445595
:10BCA500414C2000564152494F204E554C4C0020E6
:10BCB5005741434854403130404D494E20202020C3
:10BCC50000564F4F52204E554C4C494E47202000B0
:10BCD5002154455255470153504F4F5220202001C2
:10BCE5004155544F43454E54010147454D2F41465B
:10BCF500535401474C494A50414420014C2F4401BB
:10BD05000157494E4421542D55500143454E542168
:10BD1500542D555001574159505421425247002145
:10BD250054455255470153544152544054494D4589
:10BD35000146495253540144454C544120203A018F
:10BD45004D554C5449504C45014C415354014359B0
:10BD55004C53494740202040230153454C40524F06
:10BD65005554450101010143594C520143594C2099
:10BD7500542D555000215445525547010145454E16
:10BD85004801434C49434B40302C40202301434F4D
:10BD95004E5452415354014E4D45412131383301E2
:10BDA500494D50454C4C455201494D502D43414C50
:10BDB50001432D564152494F01544543202020400F
:10BDC500303040250141004E4F20414750532F460A
:0DBDD5004C00414C54492D47505320200094
:10BDE200464C47542D4C4556454C00414750532034
:10BDF2003C3E20464C002057414954004E4F2046BD
:10BE02004C49474854004045584954204C4F4740FC
:10BE12003F40004D4D2E59590020606869003C2D6D
:10BE220020202020202D3E2020202053454C003C65
:10BE32002D20202020202D3E20202045584954002E
:10BE42003C52454320205245433E20202053454C3E
:10BE520000522D4F464600202052454300414343A5
:10BE6200454C455241542E00472D554E49545300DE
:10BE7200215445525547015245434D4F44452020D8
:10BE820058015245432E2031352F23015245432E6E
:10BE92002036302F23015350454C452F5A454E44EE
:10BEA2000157495353454E40414C2001434F4D3AAF
:10BEB20000205C2020202053454E4400405750541F
:10BEC200204245535441415420414C40005741596E
:10BED200504F494E540020205445525547202100CE
:10BEE2004F4E5456414E47005652494A40003C2D4F
:10BEF200204C495354202D3E20204558495400538C
:10BF0200454C004E455854004E4558542054505408
:10BF120000505245562054505400434C5220404C3D
:10BF2200454700434C52204053554D00554954203B
:10BF32002020202020202000205549540047505323
:10BF420020464F555420004F50534C41414E005211
:10BF52004F55544500444943485354004C495354A7
:10BF6200200045544500414C544030004C45474563
:10BF72002052544520200020544F4F404D554348F5
:10BF82002000214053454C404C4953540020534516
:10BF92004C4057505440210021404F4E5456414E80
:10BFA2004740002020404F204B40202021004F4B93
:10BFB2000056415200464958004741544521580015
:10BFC20053544152544C4E20202000535443594C58
:10BFD2002000405549540054502000406A40494EC8
:10BFE20020004067404F5554002020464F555420B2
:10BFF2002021002045584954004544495400404AF4
:10C002004041004544495420204E455720534C415D
:10C01200204F50004E4558542053454C4543542020
:10C0220045584954005843542D464C4947485420DA
:10C03200005553454400454E54455220004D4D2E67
:10C042004D4D4D20004D4D2753532E53005747530E
:10C05200213834002040554054404D402000554086
:10C0620054404D002055544320004C4F43414C0056
:10C072005357495353474400414C54005355494088
:10C0820058004156474020304023003530300031BF
:10C0920036343000205D203130404B632F70005D1C
:10C0A2002020203140632F2300205D202035404B8B
:10C0B2005453005D203230304046504D00406340C2
:10C0C200204B63004654204B6300406340204E4D9A
:10C0D200004654204E4D004D2F53003230305E004A
:10C0E2003530305E00312200322200332200352208
:10C0F20000382200464C3700464C313600464C335D
:10C102003300464C36350046313030004631363049
:10C112000046323630005E252640534F47005E25EA
:10C12200264054415300414C540056415200225E75
:10C132002F24004B545300532F4E002224004B5403
:10C1420000225E004E4D00302C3500312C30003282
:0DC152002C3000302C3600312C3200322C05
:10C15F003500332C3800372C350040313500403353
:10C16F003000403630005441534B00464C2D444173
:10C17F00544500545000544F460053544100464913
:10C18F004E004C414E00534554204F4646534554A4
:10C19F000049534120484549474854004155544FA1
:10C1AF002D474F20005354415254002043484543DC
:10C1BF004B40414C4C0052414420444953540040A1
:10C1CF0053454C404845494748543A00475053401F
:10C1DF004241524F40414C4C0053494E4B40312D40
:06C1EF003221632F230042
:106F3B00304D2475A7049005C2E0F51CE0F51DE06B
:106F4B00F51EE0F51FE0F56DE0F56EE0F56FE0F591
:106F5B0054127AFD12753B2275C70375C6E475B9D9
:106F6B0001E5BCB48143127AFD1261158E628F6309
:106F7B007568F9756900127011203C2D203B2B129E
:106F8B00714612711A856D1C856E1D856F1E855499
:106F9B001F12707D203C12203243201D231271469C
:106FAB0012753BE532242850DC2212707D203CF90F
:106FBB00203DF6203205201DBD80EF301DB880EA44
:106FCB0012714612753B856D1C856E1D856F1E8576
:106FDB00541F12713012753B203DCE80991273698C
:106FEB00201D0D75531074001272CC203DBB808692
:106FFB00E553540FC553C4540F2035051271E1806E
:10700B00031272CC808BC23CD23B1270CDFD12703E
:10701B00CDFC1270CDC39573F565EC9574F564EDED
:10702B009575600504600A800EE56424E0501180BC
:10703B0006E564242040091270CD1270CD0270CD8C
:10704B001270CDFD1270CDFC1270CDC39576F56725
:10705B00EC9577F566ED9578600904600122E5669D
:10706B00F48002E5668562F0A474E025F04002C26C
:0D707B003B22C23C1270CDA2E7923DA2E67E
:10708800921DA2E592324026A2E492E592E692E7AA
:10709800FC1270CD2565F565EC3564F5641270CD8C
:1070A800FC1270CD2567F567EC3566F56622A2E41B
:1070B8009235540F79C6F71270CD09F7301D0512B5
:1070C80070CDF55322E5697023E5686030240440EB
:1070D8002CE56875F004A485F0C7F5C675B901E517
:1070E800BCB4811985BD68756902801E540370108F
:1070F80005C675B901E5BC056953690F22D23C2262
:10710800147004E5BD80F0147004E5BE80E9E5BFA5
:1071180080E575A7009006F6E56DF0A3E56EF0A38F
:10712800E56FF0A3E554F02275A7009006F6E0F5A8
:107138006DA3E0F56EA3E0F56FA3E0F55422E564D6
:10714800B2E7F56D85656EAB67E566FC30E707C3AA
:10715800E49BFBE49CFCAA62A963125E0FE566301F
:10716800E707C3E49DFDE49EFEEEB2E7F56F8D549C
:107178002275380C1273D212741DD553012275383A
:107188000C1273A3127413D55301227538001273AD
:0E719800BB1273E2D55301227538001273A3A7
:1071A6001273E2D55301227538031273D212744E4C
:1071B600D55301227538031273A3127444D55301B3
:1071C6002275380F1273BB127473D55301227538AA
:1071D6000F1273A3127473D55326229071E623738C
:1071E6008091807780688059804A803B802C801D02
:1071F600800E80DA80CB80BC80AD809E808F8080C0
:107206007538151273D2127495D553012275381537
:107216001273A312748AD55301227538091273BBEF
:1072260012745BD55301227538091273A312745B6D
:10723600D55301227538061273D2127405D553013F
:10724600227538061273A31273FAD55301227538C4
:10725600121273BB12742BD5530122753812127396
:10726600A312742BD5530122027179753815127346
:10727600D2127495D553012275380F1273A3127466
:1072860073D553012275380F1273BB127473D5531D
:1072960001227538031273A3127444D55301227563
:1072A60038031273D212744ED55301227538001268
:1072B60073A31273E2D55301227538001273BB1201
:1072C60073E2D55326229072D12373809E80A980C3
:1072D600B480BF80CA80D580E08010801B80268065
:1072E60031803C80478052805D806875380C12730F
:1072F600A3127413D553012275380C1273D212746B
:0E7306001DD55301227538121273A312742B79
:10731400D55301227538121273BB12742BD5530145
:10732400227538061273A31273FAD55301227538E5
:10733400061273D2127405D55301227538091273DB
:10734400A312745BD55301227538091273BB1274EE
:107354005BD55301227538151273A312748AD55361
:10736400012202727178C686040886037AED125DE2
:10737400CD78CAA60408A60378C686040886037ACC
:1073840062125DCD78CCA60408A60378C6860408EC
:1073940086037AB5125DCD78C8A60408A6032275C3
:1073A4001A6A751B0A78CA86180886191275E6784F
:1073B400CC86060886072278C88618088619E4F55C
:1073C4001AF51B1275E678C886060886072278C661
:1073D4008618088619751A00751B010275E6E51DE5
:1073E4002519F51DE51C3518F51CC3E51F9FF51F70
:1073F400E51E9EF51E22C3E51F9FF51FE51E9EF5A3
:107404001EC3E51D9519F51DE51C9518F51C22E50F
:107414001D2FF51DE51C3EF51CC3E51F9519F51F31
:10742400E51E9518F51E22C3E51D9FF51DE51C9E5E
:09743400F51CC3E51F9519F51FB5
:10743D00E51E9518F51E22E51F2FF51FE51E3EF5DD
:10744D001EE51D2519F51DE51C3518F51C22C3E596
:10745D001D9519F51DE51C9518F51CE51F2FF51F3C
:10746D00E51E3EF51E22E51D2FF51DE51C3EF51C06
:10747D00E51F2519F51FE51E3518F51E22C3E51D5F
:10748D009FF51DE51C9EF51CE51F2519F51FE51E35
:10749D003518F51E22E51A7009E51B70058C068D51
:1074AD000722ED851BF0A4A2F792D5ED851AF0A465
:1074BD00AEF0FFEC851BF0A4A2D53FEE35F0FF92A8
:1074CD00D5EC851AF0A42FFFE435F030D50104FE7C
:1074DD0022E4F51AF51BEF4E7003051B22EF65191B
:1074ED007006EE65187001227808C3EF33FFEE3396
:1074FD00FEEF9519F5F0EE95184003FEAFF0E51A85
:10750D0033F51AD8E5F4F51A751BFF7805C3EF337B
:10751D00FFEE33FEEF9519F5F0EE95184003FEAF33
:03752D00F0E51B6B
:1075300033F51BD8E5F4C403F51B22E51D9511E5D1
:107540001C9510500BE56E9511E56D9510500122BC
:10755000E51F9511E51E9510500BE5549511E56F4B
:107560009510500122E51D9513E51C9512400BE581
:107570006E9513E56D9512400122E51F9513E51EEA
:107580009512400BE5549513E56F95124001225377
:107590002CF8C3E51F9554FFE51E956FFE926050D1
:1075A00007C3E49FFFE49EFEC3E56E951DF519E554
:1075B0006D951CF5189261500BC3E49519F519E40B
:1075C0009518F518C3E5199FE5189E9262500AE5D3
:1075D00018CEF518E519CFF5191274DEE52C54070D
:1075E00075F003A4F538E5389075EC730276040263
:1075F000761802762602763E02765102766402768C
:107600007202768A851C16851D17C3E4951FF51531
:10761000E4951EF51402769D851C16851D17851EA2
:1076200014851F158077C3E4951DF517E4951CF5A7
:1076300016C3E4951FF515E4951EF514805FC3E4A9
:05764000951DF517E4A3
:10764500951CF516851E14851F15804CC3E4951FE2
:10765500F517E4951EF516851C14851D15803985CD
:107665001E16851F17851C14851D15802BC3E495D3
:107675001FF517E4951EF516C3E4951DF515E4955C
:107685001CF5148013851E16851F17C3E4951DF57B
:1076950015E4951CF5148000C3E5179513E51695BB
:1076A5001210D70122E5159513E514951210D7018F
:1076B50022E519F92517FFE518F83516FED3EF95DC
:1076C50011EE9510500122E5119517FDE51095165F
:1076D500FC402A4D60271274A2E5152FF515E51417
:1076E5003EF514E5159513E514951210D70122E51D
:1076F500199DF9E5189CF8851016851117E51729C8
:10770500FFE51638FEE5139FE5129E500BC3E51302
:107715009517F9E5129516F8E51A700AE51B700636
:10772500AA00AB018013E9851AF0A4E5F0FBE88512
:107735001AF0A42BFBE435F0FAE5152BFBE5143A1A
:06774500FAE5119BE510BE
:10774B009A10D70122EB9515FDEA9514FCC3E515AC
:10775B009511E514951010D717E5139BE5129A5068
:10776B0036E5139515FFE5129514FE127A1A80274C
:10777B00EB9511FFEA9510FEAA00C001127A1AD000
:10778B0003E5172BFBE5163AFAEB99F517EA98F593
:10779B0016851115851014C2D5E5466002D2D5AAFF
:1077AB0056E98AF0A4ABF0E88AF0A42B30D5047527
:1077BB00F00384F8700122E5172513FDE516351249
:1077CB00FCED8AF0A4ABF0EC8AF0A42B30D5047559
:1077DB00F00384FEE5152513FDE5143512FCED8A47
:1077EB00F0A4ABF0EC8AF0A42B30D50475F0038435
:1077FB00F9E5389078027302781A02782602782F0E
:10780B0002783802783E02784A027851027856C3E1
:10781B00743E9EFFC3743E99FE8032C3743E9EFF3E
:10782B00AE018029AF06C3743E99FE8020AF06AE31
:0D783B0001801AC3743E9EFEC3743E99FF87
:10784800800EC3743E99FF8007C3743E9EFEAF014D
:1078580008EF2437FFE51B7007E51A700CE8800E67
:10786800A2E7E51A50030460F488F0A4E5F060018B
:1078780004F923FA98FBC3E998C333F990788AE5A9
:1078880038730278A20278CF02790402793102793A
:107898005E02798B0279B80279E505A7800BEB3097
:1078A800E7032A8002291E1FFBEEC45403F583EE6A
:1078B8005408C42FF582EE5407243883F5F0E045C8
:1078C800F0F0D8DA05A72205A7800BEB30E7032AEA
:1078D8008002290E1FFBEEC45403F583EE5408C43E
:1078E8002FF582EE5407240B83F5F0E045F0F0D82D
:1078F800DA05A722804020100804020105A7800BA2
:10790800EB30E7032A8002291E0FFBEEC45403F56F
:1079180083EE5408C42FF582EE540724EC83F5F067
:10792800E045F0F0D8DA05A72205A7800BEB30E791
:05793800032A80022972
:10793D000E0FFBEEC45403F583EE5408C42FF582ED
:10794D00EE540724BF83F5F0E045F0F0D8DA05A733
:10795D002205A7800BEB30E7032A8002291F1EFBAF
:10796D00EEC45403F583EE5408C42FF582EE54078C
:10797D00249283F5F0E045F0F0D8DA05A72205A7AB
:10798D00800BEB30E7032A8002291F0EFBEEC45457
:10799D0003F583EE5408C42FF582EE540724658356
:1079AD00F5F0E045F0F0D8DA05A72205A7800BEB3E
:1079BD0030E7032A8002290F1EFBEEC45403F58322
:1079CD00EE5408C42FF582EE5407243883F5F0E009
:1079DD0045F0F0D8DA05A72205A7800BEB30E703B9
:1079ED002A8002290F0EFBEEC45403F583EE5408D2
:1079FD00C42FF582EE5407240B83F5F0E045F0F02B
:107A0D00D8DA05A7228040201008040201EC701F6F
:087A1D00ED20E740D2E023CF89
:107A250023CF30E7F980357B08801A7B1080167BE1
:107A35002080127B40800E20E4ED20E3EE20E2EF73
:107A450020E1F07B80EE8BF0A4CF8BF0A4E5F02F46
:107A5500FFEC8BF0A4CD8BF0A4E5F02D2499838F5A
:107A6500F0A433E5F033FBE98BF0A4E5F0C88BF027
:107A7500A428F9E435F0F822FFFEFCFAF8F6F4F252
:107A8500F0EFEDEBEAE8E6E5E3E1E0DEDDDBDAD9B0
:107A9500D7D6D4D3D2D0CFCECCCBCAC9C7C6C5C40E
:107AA500C3C1C0BFBEBDBCBBBAB9B8B7B6B5B4B328
:107AB500B2B1B0AFAEADACABAAA9A8A8A7A6A5A414
:107AC500A3A3A2A1A09F9F9E9D9C9C9B9A999998D8
:107AD5009797969594949392929190908F8F8E8D7F
:107AE5008D8C8C8B8A8A898988878786868585840B
:107AF500848383828281818075A700907B23E546FC
:107B0500FA24FA50027A05EA2323F978107F0493C0
:107B1500F60809E9DFF9907B3BEA93F556227FC227
:107B2500803E7F4680BA7E8C81747D1882E87A30EB
:107B350085D074608BA0808040201008127B47029E
:107B45007D9DD215D274D273C219C23A1261158EB7
:107B550047757D0075460575520212AA001201DCB3
:107B6500E53524EB500E12AA007F1990BB841281D3
:107B75003712F16EE55275F016A4F570127D537546
:107B85007E15127C1E7F237E0990BB6212814912ED
:107B9500F16E10000810010D10021280E2127CC671
:107BA50075330180DA127D0B75330180D2757E0045
:107BB500127C1E7E0090BB7312817C7F237E059014
:107BC500BB69128149127C6F12F16EE55210000FEC
:107BD50010010510028780D5045403F55280CE129A
:107BE5007C1E7F237E0B90BBA1128149E546600771
:107BF50014600414124D2212F16EE54610000810AF
:107C0500010B10021180D860D6154680D2B405024A
:107C150080CD054680C9027B6275320012F2E57F90
:107C2500017E1190BB5912817C7E0012E9A4E57E8C
:107C3500D26612E9FB75170812EE31124D617571A6
:107C450000C20612EB4B741BFFF5177E0F90BBA805
:107C5500305D0390BBB012817C12AA4312674612B5
:107C650052C7C206126F63022829E55260141460D8
:107C75001E1460297F647E2D791C127CB91E1FD9C4
:107C8500F9227F6A7E1F7928127CB91FD9FA227FD3
:107C9500487E2D791C127CB90F1ED9F9227F567E9C
:107CA5003379281F12F2000F0F12F2001F12F20093
:107CB5001ED9F0221E12F2000E0E12F2001E02F262
:107CC50000E552605514606814606D800075709E03
:107CD500127D408003757000E5732540F573E4352A
:107CE50074F574E43575F57522757016127CDD80B2
:107CF5000375702DE5762542F576E5773541F577FF
:107D0500E43578F57822E55260CB1460DC1460E147
:107D15008000757044127CF9800375705AE573957F
:097D250040F573E5749400F57457
:107D2E00E5759400F57522757071127D22800375CC
:107D3E007088E5769542F576E5779541F577E578A5
:107D4E009400F57822E546907D6993F540FEAD47A7
:107D5E00E4FFFC125EA28E418F4222020C183060AC
:107D6E00C07F4012189812283F12F16E128018EB45
:107D7E00700590B8C0800B127E2690BFA550039060
:107D8E00BFEB7F3F7E0412814912F16E12F1231276
:107D9E00F16475370990BB17122725907DAD7302DC
:107DAE00023D027F6D027B41028049027D9D027D74
:107DBE00C5027DDE027D6F7F2E1220CD80D17F36F3
:107DCE007E0490BF7912814912F16E12F12380BFA9
:107DDE007F3712189812283F12F16E127FFC125440
:107DEE0057D2AC1000A9306DFA127ED6203BCF4090
:107DFE00ED7568F9751600127F2340FB1280BF7F68
:107E0E00367E29E51612E78212F16E05161281EE04
:107E1E0078C6B6F7E2027FF67C0512545712EFC70A
:107E2E00744112EFD8745312EF88EB12EFB6128230
:107E3E00005003DCE5227515F975160010000EE5ED
:107E4E00156025127E784005127E9F5002D3227F48
:107E5E003F7E29E51612E78212F16E7F1412F13A77
:107E6E000516E51664F870D4C3221287BD75B901E4
:107E7E00E5BCB4811AE5BDF51570037516F778C625
:0B7E8E00A6161289061288FE1288FE5C
:107E9900C30288FED3227F0575F019D5E0FDD5F020
:107EA900FA12545712EFC7744112EFD8744212EF05
:107EB900887E0F78C6E60812EF88DEF912EFB9124C
:107EC9008200400122DF012275F00080CEC23B1200
:107ED9005457D2AC12F000204C3CB440F712F005D4
:107EE900B4400312F005B4412DF53812F005B4532E
:107EF9002512F005FA12F005E538701A12F005B4EA
:107F09000D1412F005B40A0EC3E5169A4003028156
:107F1900E5C2ACD23B22C2ACD322128244125457DE
:107F2900D2AC1000F112F000204CEBB440F412F086
:107F390005B4400312F005B441DCF53812F005B47C
:107F490042D47E1078C612F005F608DEF9E53870DD
:107F5900C512F005B40DBF12F005B40AB9C2ACC31D
:107F690022027D9D7F0A12189812283F12F16E1283
:107F79007FFC125473D2AC1000E712F005B440F53F
:107F8900F53812F005B46EED12F005E538600A1205
:107F99005473744F12EF9480DC125473744012EFCF
:107FA900D8E51612EF9412EFA47568F97516001248
:107FB9005473D2AC10003912F005B440F7F53812F9
:107FC900F005B44EC07E1078C612F005F608DEF949
:107FD900125473E5386007744F12EF9480D1128000
:107FE900BF0516745112EF9478C6B6F7C212805CB9
:0C7FF900027D9D7515007516031287B4FB
:1080050075B901E5BC30E70205160515E51524200F
:1080150050EB227B007515F91287BD75B901E5BCDA
:10802500B481010B0515E515240450EC75150112F5
:1080350087B475B901E5BCB481010B0515E51524B7
:108045002050EC227F1C12189812289C40067515AA
:10805500F912805C027D9DE51560372404401A24E1
:108065001E5019E5152407400280271287BD12808E
:10807500980515E515240450F27515011287B47598
:10808500B901E5BC30E7031280980515E5152420F4
:1080950050EA221280AD1255F705C61255F705C6EE
:1080A5001255F705C60255F774FF80057404800163
:1080B500E4F5BCF5BDF5BEF5BF22E568606AF515CA
:1080C5000515E5152404501D7515011287B475B9FC
:1080D50001E5BC30E70280190515E515242050EBB4
:1080E500751500800C241C60F750E0E5152406503A
:1080F50037E56875F004A485F0C7F5C675BC81E55C
:1081050015F5BDF56878C6B6F70375BD000812818B
:108115002212811C12811C86BC0886BD0886BE08F9
:0981250086BF081255F705C622B9
:10D3DA0012CCB612D4D9128CC112D45E128CC912D4
:10D3EA00D46B02CCBA12CCB612D4D9128CC17F5AE1
:10D3FA00C23C128BA3128D9F783F79437F607EEAED
:10D40A0012D4CD128CC97F65128BA3128D9F783DE1
:10D41A0079417F207E4E12D4CD303C2012D68F1215
:10D42A00D4EA783F794312D449783D794112D449F4
:10D43A0012D68F78D7E65480F675370002C3A7C391
:10D44A00E796FF1819E796FE0809C3E69FF7181929
:10D45A00E69EF7227F5B7E0690C07E12817C1F804B
:10D46A000A7F667E14745912E89D1F128A2C7E392F
:10D47A00E402E8BC7866E620E73418C3E69472084A
:10D48A00E694045029C318E6941F08E69404401E43
:10D49A007869E620E71818C3E6940E08E694015066
:10D4AA000DC318E6947508E694004002D322C322FD
:10D4BA00E67D0030E7011D08E62BFB18E63CFCE49C
:0ED4CA003DFD22C3EB9FF6F71819EC9EF6F716
:10D4D8002212D47E400CE47842F608F67840F6082A
:10D4E800F6227864C3E6946AF55708E6944CF55634
:10D4F8000808C3E69458F55B08E694AEF55A753902
:10D5080000AC56AD57EC12D04C784C12D0DAAC5A6D
:10D51800AD5BEC12D04C785012D0DA7F2B7E867D32
:10D52800777C1812D011785012D0CE12CF1D12D09D
:10D5380011785012D0CE12CF1D12D011785012D0BF
:10D54800CE12CF1D12D0117F367E847D257C6412C9
:10D55800D011785012D0CE12CF1D12D011784C12A3
:10D56800D0CE12CF1D12D0117F3F7EA27D607C8B62
:10D5780012D011785012D0CE12CF1D12CD0B12CD71
:10D588000B12D0E67F3F7E807D057CE6053912CF01
:10D598001D784812D0DA7F2C7E937D477C7F12D08D
:10D5A80011785012D0CE12CF1D12D011785012D04F
:10D5B800CE12CF1D12D011784C12D0CE12CF1D1220
:10D5C800D0117F357EB47DF87CDF12D011785012EF
:10D5D800D0CE12CF1D12D011785012D0CE12CF1D3E
:10D5E80012D0117F3F7EED7D227CCD12D011784C78
:10D5F80012D0CE12CF1D12CD0F12CD0B784412D0FF
:10D60800DA7F317E397D9D7CE712D011784C12D0BB
:10D61800CE12CF1D12D011784C12D0CE12CF1D12BF
:04D62800D011784461
:10D62C0012D0CE12CD0F12D0117F2C7E377D0C7CF8
:10D63C00A312D011784C12D0CE12CF1D12D011786B
:10D64C004C12D0CE12CF1D12D011784C12D0CE125B
:10D65C00CF1D12CD0F12D0E67F3F7E807D027C9FC6
:10D66C00053912CF1D784412D0DA784812D0CE1278
:10D67C00D0838E428F43784412D0CE12D0838E400A
:10D68C008F4122753900AC42AD43EC12D04C784836
:10D69C0012D0DAAC40AD41EC12D04C784412D0DA56
:10D6AC007F2B7E537D507C0912D011784812D0CE3E
:10D6BC0012CF1D12D011784812D0CE12CF1D12D01D
:10D6CC0011784412D0CE12CF1D12D0117F347EF2BD
:10D6DC007DCD7CA312D011784812D0CE12CF1D1262
:10D6EC00D011784812D0CE12CF1D12D0117F3F7EB0
:10D6FC000A7D2E7CAE12D011784412D0CE12CF1DE2
:10D70C0012CD0B12CD0B784C12D0DA7F2B7E4F7DC5
:10D71C00AF7CB212D011784812D0CE12CF1D12D0DD
:10D72C0011784812D0CE12CF1D12D011784812D0D9
:10D73C00CE12CF1D12D0117F357EB17D4B7C951250
:10D74C00D011784812D0CE12CF1D12D011784412BD
:10D75C00D0CE12CF1D12D0117F3F7E497DCD7C459E
:10D76C0012D011784812D0CE12CF1D12CD0F12CD7F
:10D77C000B785012D0DA784C12D0CE12D0838D5553
:10D78C008E568F57785012D0CE12D0838D598E5A18
:04D79C008F5B7864C3
:10D7A000E557246AF608E556344CF608E555340486
:10D7B000F608E55B2458F608E55A34AEF608E43579
:03D7C00059F622F5
:10C1F50012CCB612C88612CCBA7F6690C060128186
:10C205007A12C2637F5A78C412C23F12C24778C6F7
:10C2150012C23F12C22A7F6578C812C23F12C247B6
:10C2250078CA12C23F7E2DE51B12E8BC7E33E51AA3
:10C2350012E8BC7E39E51902E8BC860408860302CB
:10C245005D6C7E15E51C12E8BC7E1BE51B12E8BC87
:10C255007E21E51A12E8BC7E27E51902E8BC7F5A63
:10C265007E01E53A12E7D07E0B90CC7AE53B93024E
:10C27500E8CFE6FF08E6FE08E6FD339217E4500135
:10C28500F4FC12D0F775130A75390112D2F578D777
:10C29500E6C2E775F00A84F9303D02A9F012D0F73D
:10C2A5008913053912D2CE30170A053912D2E105A4
:10C2B5003912D2E1A80302D0DA12CCB612C886C26E
:10C2C5003C7F5A7E03128F5012C26312F16E10002A
:10C2D5000810011510022080EFE53A146004153AA4
:10C2E5008003753A3CD23C80DFE53AB43C05753AAB
:10C2F5000180F2053A80EE7E03128F4B7E0B128F82
:10C305005012C26312F16E100008100115100220C0
:10C3150080EFE53BB40205753B158002153BD23C29
:10C3250080DFE53BB41505753B0280F2053B80EEE9
:10C335007E0B128F4B7F5A78C412C23F12C247122E
:07C34500C3B0128DAF78C4F4
:10C34C0012C40878C612C23F12C22A12C3E2751C6C
:10C35C0000128DAF78C612C4087F6578C812C23F30
:10C36C0012C24712C3B0128DAF78C812C40878CA73
:10C37C0012C23F12C22A12C3E2751C00128DAF7892
:10C38C00CA12C408303C14E53B24F4500B78C9E6BF
:10C39C002410F618E63427F612C40E12CCBA128901
:10C3AC003102F16EC2247E15E51C128EA0F51CD252
:10C3BC00247E1BE51B128EA0F51B1023E77E21E5C6
:10C3CC001A128EA0F51A1023E67E27E519128EA0FC
:10C3DC00F5191023E822C2247E2DE51B128EA0F540
:10C3EC001BD2247E33E51A128EA0F51A1023E77E99
:10C3FC0039E519128EA0F5191023E622ECF608EB9C
:10C40C00F62212CC9278C8E6FE0886073395E0FD3A
:10C41C00FC12D0117FE87E037D007C0012D2F51255
:10C42C00D01178CAE6FE0886073395E0FDFC12D2DF
:10C43C00CE12D0117F807E697D677CFF12D2CEEC4C
:10C44C0012D04812D0117F3F7E807D0D7C1D12CF03
:10C45C001D12D0117F3D7E407D007C0012D01178E2
:10C46C00BC12D0CE12CF1D12D0117F3E7E807D002B
:10C47C007C0012CD0F12D01178BC12D0CE12CF1D71
:09C48C0012D0117F3F7E807D007B
:10C495007C0012CD0B12D01178B412D0CE12CF1D64
:10C4A50012CF95783C12D0DA7F407E807D007C00EB
:10C4B50012D011783C12D0CE12CF1D12D17412D0E9
:10C4C500117F3F7EA87D007C0012D01178B812D074
:10C4D500CE12CF1D12CF1D12D0117F407E007D00E0
:10C4E5007C0012D011783C12D0CE12CF1D12D1741F
:10C4F50012D0117F3F7EC07D007C0012CF1D12CD72
:10C505000F12D01178B812D0CE12CF1D12D01178DB
:10C515003C12D0CE12CD0F785412D0DA12D15E78FB
:10C525005812D0DA12D01112CF1D12D01178C012C4
:10C53500D0CE12CF1D784412D0DA785412D0CE1254
:10C54500D174783C12D0DA12D01112CF1D12D0114D
:10C5550078BC12D0CE12CF1D783C12D0DA7F3E7E49
:10C56500C07D007C0012D011783C12D0CE12CF1DB8
:10C5750012D0117F3F7E007D007C0012CD0F12D0BE
:10C5850011783C12D0CE12CF1D12D0117F3F7E8084
:10C595007D007C0012CD0F12D01178B412D0CE12CE
:10C5A500CF1D787012D0DA78C4E6FE088607339579
:10C5B500E0FDFC12D0117FE87E037D007C0012D2E5
:10C5C500F512D01178C6E6FE0886073395E0FDFC26
:10C5D50012D2CE12D0117FE07E5E7DF87CFF12D2A2
:10C5E500CEEC12D04812D0117F3F7E7F7DE57CC90D
:05C5F50012D011787066
:10C5FA0012D0CE12CF1D12CF95785012D0DA7F3FCB
:10C60A007EF07D007C0012D011783C12D0CE12CF81
:10C61A001D12D0117F3F7EC07D007C0012CD0F120B
:10C62A00D011783C12D0CE12CF1D12D0117F3F7E8E
:10C63A00807D007C0012CD0F783C12D0DA78BC12D3
:10C64A00D0CE12D0117F3F7E807D007C0012CD0BB0
:10C65A0012D011783C12D0CE12D01178B412D0CEAA
:10C66A0012CF1D12CF1D784012D0DA785412D0CED4
:10C67A0012D1AC783C12D0DA12D01112CF1D7874D4
:10C68A0012D0DA7F417E107D007C0012D01178C072
:10C69A0012D0CE12CF1D12D0117F407E807D007C39
:10C6AA000012D011784412D0CE12CF1D12D0117FB1
:10C6BA00417E207D007C0012CD0B12D011784412ED
:10C6CA00D0CE12CF1D12D0117F407E407D007C005B
:10C6DA0012D011787412D0CE12CF1D12D0117F4011
:10C6EA007EA07D007C0012CD0F12CD0F12CD0B1251
:10C6FA00D011785012D0CE12CF1D12D0117850120C
:10C70A00D0CE12CF1D12D0117F3D7E2A7DAA7CABDE
:10C71A0012CF1D12D0117F3F7E007D007C0012CD0A
:10C72A000B12D011783C12D0CE12D011787012D0E0
:10C73A00CE12CF1D12D011784012D0CE12CF951240
:10C74A00D011785012D0CE12CF1D12D011785012BB
:10C75A00D0CE12CF1D12CF1D12D011785412D0CEC6
:0CC76A0012CD0B12D0117F4A7E517DD2FF
:10C776007CCB12CF1D12D08378AC12D0DA7F407EEC
:10C78600007D007C0012D011787412D0CE12CF1D1D
:10C7960012D0117F3F7E807D007C0012CD0F12D01B
:10C7A60011784412D0CE12CD0F12D011785012D07B
:10C7B600CE12CF1D12D011785012D0CE12CF1D122C
:10C7C600D011785012D0CE12CF1D12D0117F3E7EDE
:10C7D6002A7DAA7CAB12CF1D12D011785012D0CE72
:10C7E60012CD0B12D011785812D0CE12CF9512D08E
:10C7F600117F4A7E517DD27CCB12CF1D12D083127F
:10C80600D011AF3AEF3395E0FEFDFC12D0117F4018
:10C816007E7E7D057C0012D2F512D0117F607E757A
:10C826007D587CFF12D2CE12D2CE78B012D0DA78F2
:10C83600AC751B6412C85D8F1C78B0751B6712C877
:10C846005DE51C75F00AA42FFF249C50027F00783A
:10C85600D7E654802FF62275390012D0CE12D011A9
:10C866007F0A7E007D007C0012D3A1A81BE513F68B
:10C8760008E512F608E511F6335004EFF404FF223A
:10C88600C23D78647BAC12C277D23D78677BB0122A
:10C89600C27712CC927F007EE47D577C0012D011C5
:10C8A60078AC12D0CE12D2CE12D0117F007E537D3C
:0EC8B600077C0012D3A112D03085133B7F8087
:10C8C4007ECB7DA47C0012D01178B012D0CE12D2CF
:10C8D400CE12D0117F407E7E7D057C0012D3A11242
:10C8E400D030E513F56F04F53A85126E85116D8528
:10C8F400106C7F407E7E7D057C0012D011786C1216
:10C90400D0CE12D2F512D0117F607E0C7DA27C00B5
:10C9140012D01178B012D0CE12D2CE12D2E1786CED
:10C9240012D0DA78AC12D0CEEC12D04812D0117FEB
:10C93400347E9C7D2B7C5F12CF1D785412D0DA128A
:10C94400D15E785012D0DA786C12D0CEEC12D04886
:10C9540012D0117F347E9C7D2B7C5F12CF1D12D0B0
:10C9640011785012D0CE12CF1D784012D0DA7F4009
:10C974007E007D007C0012D011785412D0CE12CFEC
:10C984001D12D17412D0117F3D7EC07D007C001237
:10C99400D01178BC12D0CE12CF1D12D0117F3E7EA2
:10C9A400C07D007C0012CD0F12D01178BC12D0CE05
:10C9B40012CF1D12CF1D12D0117F3D7E407D007C11
:10C9C4000012D01178BC12D0CE12CF1D12D0117F1C
:10C9D4003E7E807D007C0012CD0F12D01178BC12F7
:10C9E400D0CE12CF1D12D0117F3F7E807D007C00FF
:10C9F40012CD0B12D011785412D0CE12CF1D12CDFD
:10CA04000B12D0117F407E807D007C0012D0117803
:10CA14005412D0CE12CF1D12D17412D0117F3D7E8C
:10CA2400707D007C0012D01178BC12D0CE12CF1DC4
:10CA340012D01178BC12D0CE12CF1D12CF1D12CD40
:10CA44000F12D01178B412D0CE12CF1D785812D054
:10CA5400DA785412D0CE12D174783C12D0DA7854E9
:10CA640012D0CE12D1AC785412D0DA783C12D0CE97
:10CA740012D01112CF1D12D01178BC12D0CE12CF09
:10CA84001D783C12D0DA7F3E7EC07D007C0012D03F
:10CA940011783C12D0CE12CF1D12D0117F3F7E00F0
:10CAA4007D007C0012CD0F12D011783C12D0CE1232
:10CAB400CF1D12D0117F3F7E807D007C0012CD0FF0
:10CAC40012D01178B412D0CE12CF1D787012D0DAF1
:10CAD400785012D0CE12D01112CF1D12D01178C0BE
:10CAE40012D0CE12CF1D784412D0DA785412D0CEA0
:10CAF40012D01112CF1D787412D0DA784012D0CE31
:10CB040012D01112CF1D783C12D0DA7F407E807D86
:10CB1400007C0012D011784412D0CE12CF1D12D056
:10CB2400117F417E107D007C0012CD0F12D0117850
:10CB34004412D0CE12CF1D12D011787412D0CE125E
:10CB4400D0117F407EA07D007C0012CD0B12CD0F52
:10CB540012D011783C12D0CE12CF1D12D0117F3DCD
:10CB64007E2A7DAA7CAB12CF1D12D0117F3F7E009E
:10CB74007D007C0012CD0F12D011785412D0CE1249
:10CB8400D011787012D0CE12CF1D12D011783C1271
:10CB9400D0CE12CF1D12CF1D12D011785812D0CE84
:10CBA40012CD0F12D0117F3F7E7F7DE57CC912CF5D
:01CBB4001D63
:10CBB50012D0117F4B7E187D967C8012CD0F12D03E
:10CBC5008312D0117FE87E037D007C0012D3A11271
:10CBD500D03078C8A61208A61308A60608A60778B6
:10CBE5007412D0CE12D0117F3F7E807D007C001262
:10CBF500CD0B12D011784412D0CE12CD0F12D01118
:10CC05007F3E7E2A7DAA7CAB12CF1D12D0117840C3
:10CC150012D0CE12CF1D12D011783C12D0CE12CF29
:10CC25001D12D011784012D0CE12CD0F12D0117F27
:10CC35003F7E7F7DE57CC912D011787012D0CE126F
:10CC4500CF1D12CF1D12D0117F487EF47D247C00AC
:10CC550012CD0F12D08312D0117FE87E037D007CA8
:10CC65000012D3A112D03078C4A61208A61308A6C4
:10CC75000608A607223F3F4344454647484A4B4CD2
:10CC85004D4E5051525354555657583F3FE4F53980
:10CC9500F5A790CCA6791078B4E493F6A308D9F952
:10CCA5002232A5C24A4A19DC3A885CDB3BFFD6DC56
:01CCB5003B43
:10CCB600D2D58002C2D575A70490040078107F0BE8
:10CCC60012CCE278267F0512CCE2783C7F2212CC89
:10CCD600E2786A7F0F12CCE275A7002230D506E60D
:10CCE600F008DFFB22E0F608DFFB22DA0CD902802F
:10CCF6000BD906303701B3500502CE7E923702CEED
:10CD06006AD9F680F9D2368002C23612CEAF3036F4
:10CD160006C86002B237C89236DAD0D9E4B8000A3B
:10CD260012CEF6A236923702CE5360FBB513004000
:10CD36000F12CEF6A23692F7A2379236A2F79237A4
:10CD4600C398F40424E740DF2419AD29AC28AB27A7
:10CD56007A00C394084008CDCCCBCAE4CD80F42435
:10CD6600086010F9C3ED13FDEC13FCEB13FBEA139B
:10CD7600FAD9F1A236303701B340308A17E5102BC5
:10CD8600F518E5113CF519E5123DF51A501A13F59B
:10CD96001AE51913F519E51813F518E51713F5171C
:10CDA6000513E5137002051402CE09E4C39AF517BC
:0CCDB600E5109BF518E5119CF519E5123D
:10CDC2009DF51A500DB237C378177F04E496F60822
:10CDD200DFFA7A047019E513C39408F513500215AB
:10CDE20014E4C517C518C519F51ADAE802CEAA2047
:10CDF200E7BAE5137002151415137817C37F04E61A
:10CE020033F608DFFA80E8E51A20E7137817C37FC4
:10CE120004E633F608DFFAE513700215141513E57C
:10CE2200173378187F03E63400F6500E08DFF775E3
:10CE32001A800513E51370020514E51420E75470F7
:10CE420027E513604E046020851A12851911851892
:10CE5200105326F0AC10AD11A237E51313FFE51203
:10CE620092E7FEA81302D030E4F512F511F510F5A1
:10CE7200147513FF5326F043260580D8E5FFF512FB
:10CE8200F511F510751400F513D2375326F0432629
:10CE92000980C15326F0432603E4F512F511F5107B
:10CEA200F514F513C23780AC5326F080EC79017A81
:10CEB200018512F0E513A2F7339237751400F513CA
:10CEC2006002D2F785F012A813B8FF0809E512C272
:10CED200E76001098C278D288EF0A2F7EF330470EA
:01CEE2000A45
:10CEE3000AC2F705F00AD5F0011A146002D2F785D9
:10CEF300F02922C88813C512C529C512C511C52832
:10CF0300C511C510C527C51022DA03B8000302CE28
:10CF13007ED9028002D9F702CE6A12CEAF30370132
:10CF2300B392377004D9E78005DADEB8000302CE86
:10CF3300AAD9E2C3947E500215142513F5135002A7
:10CF430005147815760008B81BFA78277915E608D2
:10CF5300FAE8FC78108AF0E608A427F709E5F03729
:10CF6300F7500989F00907E760FBA9F0B813E61940
:10CF730019ECF8B82AD802CE0902CE95B8FFFA0206
:10CF8300CE7ED9FB02CE6ADAF6B800F002CEAA1240
:10CF9300D0E612CEAF303701B392377007D9E3B87A
:10CFA30000E280DBDAE1B8000280E1D9D5C8C3989A
:10CFB30050021514247F50020514F513781A7600D5
:10CFC3007A1A7B80C3E5109527E5119528E512951C
:10CFD300294016C3E5109527F510E5119528F5119D
:10CFE300E5129529F512E64BF6DA0302CE09EB03B7
:0ACFF300FB30E703187600C3E510D9
:10CFFD0033F510E51133F511E51233F51240CA3052
:10D00D00E7DD80B6E53905396010D0F0D0E0C0100D
:10D01D00C011C012C013C0E0C0F08F138E128D115D
:10D02D008C1022E539146010D0F0D0E0D013D0125E
:10D03D00D011D010C0E0C0F01539227920800C79C4
:10D04D0010800479087D007E007F003392D5500357
:10D05D0012D0C0EC33400FEF33FFEE33FEED33FD56
:10D06D00EC33FCD9EE22EECCF5F0747E29A2D5136B
:10D07D00FF92F7AEF022EF8EF0A2F7D2F73392D5F2
:10D08D00C3947F5006E4FFFEFDFC229420400474FF
:10D09D00FF80F304CCFEE4FFFAE5F0CC6012C3CCC4
:10D0AD0013CCCD13CDCE13CECF13CF0450EEDAEC7F
:10D0BD0030D5D7C3E49FFFE49EFEE49DFDE49CFCC8
:0CD0CD0022E6FC08E6FD08E6FE08E6FF8F
:10D0D90022ECF608EDF608EEF608EFF622CFC513B6
:10D0E900CFCEC512CECDC511CDCCC510CC22E4F51D
:10D0F90013F512F511F51022E493FCA3E493FDA3B3
:10D10900E493FEA3E493FFA322C0E012D01112CF4F
:10D119001D12D14512D101D0E0C0E012D01112D1B7
:10D129003C12CF1D12D01112D10112CD0FD0E0D572
:10D13900E0E722AC48AD49AE4AAF4B228C488D4955
:10D149008E4A8F4B2274FF7809FFFEFDFCE52654B9
:10D15900F048F5262212D20504A2E1927F1420E0BC
:10D169001590D286740412D112802912D20530E1A9
:10D1790002B27F20E0EB8C4C8D4D8E4E8F4F90D2BA
:10D189009A740412D11212D011AC4CAD4DAE4EAFFF
:10D199004F12CF1D307F04EF6480FFEE33EF337001
:10D1A90001FF2212D205C0E08C4C8D4D8E4E8F4F5F
:10D1B90090D2BE740312D11212D011AC4CAD4DAE47
:10D1C9004EAF4F12CF1DECC54CFCEDC54DFDEEC564
:05D1D9004EFEEFC54F02
:10D1DE00FF90D2AE740312D112D08212D011AC4C89
:10D1EE00AD4DAE4EAF4FE58230E00712CF95B27F18
:10D1FE00809D12CF928098EE33EF3324605007D08B
:10D20E00E0D0E002D14EEFA2E7547F927FFF12D022
:10D21E00117C837DF97E227F3E12CF1DEE33EF33DC
:10D22E002481501012D01112D08312D048EFB2E7E1
:10D23E00FF12CD0FEE33EF33602A2403F8C313FF32
:10D24E00EE92E7FEE82481E4501A12D01112D08338
:10D25E00EF04C2E0FCF58212D050EFB2E7FF12CD20
:10D26E000FE58203FAEE33EF33600B148FF0A2F763
:10D27E0013FFEE92E7FEEA2283FA703AE4E9AABCC3
:10D28E00F8E0813EE6E99DBF0000803F1A3C283958
:10D29E00666999BBE335A33DE75D25BFDB0FC93F4B
:10D2AE00CCDB8D41EE3649C43F91C9453DF8B0C542
:10D2BE000000803F34F517C373FA2F45DDFD0AC613
:10D2CE00EF2513FFEE3512FEED3511FDEC3510FC9A
:10D2DE0002D030C3EF9513FFEE9512FEED9511FDC2
:10D2EE00EC9510FC02D030EFF88513F0A4FFE51397
:10D2FE00C5F0CEF9A42EFEE435F0CDFA88F0E51295
:09D30E00A42EFEED35F0FDE43320
:10D31700CC8513F0A42CFCE5128AF0A42CFCE511B3
:10D3270089F0A42CFCE51088F0A42CFC89F0E51208
:10D33700A42DFDEC35F0FCE51188F0A42DFDEC35AE
:10D34700F0FC8AF0E513A42DFDEC35F0FC02D0309B
:10D35700E4CCF8E4CDF9E4CEFAE4CFFB75F020C3D2
:10D36700E51333F513E51233F512E51133F511E53E
:10D377001033F510EF33FFEE33FEED33FDEC33FCE6
:10D38700EF9BEE9AED99EC98400CFCEF9BFFEE9A21
:10D39700FEED99FD0513D5F0C622C2D5EC30E705A1
:10D3A700B2D512D0C0E51030E70DB2D512D3C412F2
:10D3B700D35712D0C0800312D35730D515C3E49585
:10D3C70013F513E49512F512E49511F511E4951090
:03D3D700F510222C
:108F9E00E57124885002D2191261158E4712E5E050
:108FAE0012AA431264D1305E0F12646F12A12F12F7
:108FBE0063A0129D6F124E5C124578125403103648
:108FCE0026301219E4129121129136129231129218
:108FDE00533051030292DD1295AE205109C251E475
:108FEE00F552F545F5442275A700758307E559C47A
:108FFE0054F0F582E0F538A3E0F518A3A3A3E0F54D
:10900E001E74FF1291211261158E1C8F1B7510DFBD
:10901E00751100E51164B470061290EC7511101202
:10902E0090B94028AE1CAF1B12619D20321EAC03BE
:10903E00AB027A0C125DA4ED701275A70075830455
:10904E00851182ECF00583E510F00511D510C412E0
:10905E0090EC75C70375C6E075A7049005007F04F4
:10906E001290A7DFFB75A70012385712646FE4F554
:10907E00A7F8F559758307E8C4F582E065387011D5
:10908E00A3E06518700BA3A3A3E0651E70038859B7
:10909E002208C3E5589850DC22E0F5BCE0F5BDE0AF
:1090AE00F5BEE0F5BF1255F705C622E51075F004C2
:1090BE00A4F5C685F0C775B901E5BC33401F05C6DA
:0B90CE0005C675B90185BE6485BF654D
:1090D90005C675B90185BC6685BD6785BE6885BF4E
:1090E90069C322E51124FE502E75A7007F10AE1129
:1090F9001E7583048E82E0FD1582E0CDB505005012
:1091090012F00582CDF00583E0FD1582E0CDF00572
:1091190082CDF0DEDCDFD7227FB475A7549004003E
:1091290005A7900500F0F0DFFC75A7002212993918
:10913900C2517B077AFFE47F00F5A79004001292E1
:109149001DED244C4035EC603075A7008D8205A7D4
:109159001291E37583058D82E02410401CF005A768
:10916900E02CF0500505A7E004F0BA000CBB00099B
:10917900D251EF24DC50027F23DFC3EA600512914C
:10918900968006EB60031291CE75A7002230E004A9
:109199007553082230E1047553182230E2047553DF
:1091A900282230E3047553382230E40475534822E9
:1091B90030E5047553582230E6047553682230E7C8
:1091C900037553782230E0047553882230E1047521
:1091D90053982230E2037553AA22ED54F0C4232395
:1091E9009091ED735302FE225302FD225302FB229A
:0791F9005302F7225302EFBD
:10920000225302DF225302BF2253027F225303FE66
:10921000225303FD225303FB225303FB22129833F4
:1092200012B191E4F5F7E4ADF7F5F7E4ACF7D2B29B
:109230002290050078B4E06015FD54F0C4CD7C00A8
:10924000540FFE1583E0FF125EA2EFF00583058246
:10925000D8E42275830478FF088882E060FAF5D3A9
:109260008812E512244C50012285D3D288D488126A
:1092700079FF0512E51260F00908E875F0B484A8DA
:10928000F08882E060ECF5D3B9000280D5B9230004
:1092900050D0C395D292D15002F40409FEE4FFFCF1
:1092A000AD01125EAF7401FA25D475F0B484A8F054
:1092B000AC06AB07125D96EB30E7010CE5D22C3023
:1092C000D1029C9C8882F00AEAB501DCE512244CAC
:1092D00050012285D3D28512D4A812809390040025
:1092E00012939C8C068B0512939CE4FFF512F511EA
:1092F0008C148B13C3ED9BF9EE9CFA4012E5119987
:0B930000E5129A500A8C148B138A129D
:10930B0089118F528F82E0F9C3ED99FDEE9400FE27
:10931B00E582245A5002244C75F0B48485F082E027
:10932B00FA2DFDEE3400FEEB9AFBEC9400FCE92BDE
:10933B00FBEC3400FC0FBFB4B0E55224D340022445
:10934B00B4F552C3E51333FBE51433FCE511FE2BE7
:10935B00FBE512FF3CFC125F04E9F89093AE93F52A
:10936B0011FDEBF513FFECF514FE7C00125EA28FE2
:10937B0044E89094AE93FAAB13AC14125DCDAF03EB
:10938B00AE04AD117C00125EA2EF7002F552F545F2
:10939B00227C007B007F5AE02BFBEC3400FC058227
:1093AB00DFF522B4B4B4B4B4B4B4B4B4B4B4B4B498
:1093BB00B4B4B4B4B4B3B3B3B3B3B3B3B3B3B3B36D
:1093CB00B3B3B2B2B2B2B2B2B2B2B2B1B1B1B1B175
:1093DB00B1B1B0B0B0B0B0B0B0AFAFAFAFAFAEAE89
:1093EB00AEAEAEAEADADADADADACACACACACABABA7
:1093FB00ABABAAAAAAAAA9A9A9A9A9A8A8A8A8A7D0
:10940B00A7A7A7A6A6A6A5A5A5A5A4A4A4A4A3A300
:10941B00A3A2A2A2A2A1A1A1A0A0A0A09F9F9F9E38
:10942B009E9E9D9D9D9D9C9C9C9B9B9B9A9A9A9975
:10943B0099999998989897979796969695959594B4
:10944B009494939393929292919191919090908FF7
:10945B008F8F8E8E8E8D8D8D8C8C8C8B8B8B8A8A39
:10946B008A8989898888888787878686868585857E
:10947B008484848383838282828181818080807FC4
:10948B007F7F7E7E7E7E7D7D7D7C7C7C7B7B7B7A05
:10949B007A7A797979787878777777767676757549
:1094AB00757474000203050608090B0C0E101113DA
:1094BB00141617191A1C1D1F2122242527282A2BA5
:1094CB002D2E303133343637393A3C3D3F40424311
:1094DB00454648494B4C4E4F505253555658595A86
:1094EB005C5D5F606163646667686A6B6C6E6F700E
:1094FB007273747677787A7B7C7E7F8081838485A8
:10950B008688898A8B8D8E8F909192949596979859
:10951B00999B9C9D9E9FA0A1A2A4A5A6A7A8A9AA22
:10952B00ABACADAEAFB0B1B2B3B4B5B6B7B8B9BA08
:10953B00BBBCBDBEBFC0C0C1C2C3C4C5C6C7C7C804
:10954B00C9CACBCCCCCDCECFD0D0D1D2D3D4D4D51D
:10955B00D6D7D7D8D9DADADBDCDCDDDEDEDFE0E04C
:10956B00E1E2E2E3E4E4E5E5E6E7E7E8E8E9EAEA95
:10957B00EBEBECECEDEEEEEFEFF0F0F1F1F2F2F3F2
:10958B00F3F4F4F4F5F5F6F6F7F7F8F8F8F9F9FA69
:10959B00FAFAFBFBFBFCFCFDFDFDFEFEFEFEFFFFF6
:1095AB00FFFFFFC251E4F544F814FB900400A9003F
:1095BB007C0FC2D11296C9E82405F8B8B4F08B130E
:1095CB00E5122403FA244C5001FABBFF012275115A
:1095DB002C8A191297008F16203D12AA1975112388
:1095EB001297008F15751600303DE280117511230F
:1095FB001296A8751500303D05E82F13F51575115A
:01960B00124C
:10960C001296A8751400303D05E82F13F514EA24C2
:10961C0004F552244C5002F552E4F51AF51BF51CD6
:10962C00E516600AFB7A00AF137EFF12966EE51505
:10963C00600AFB7A4FAF137EFF12966EE516600D33
:10964C00FB7A00E5146006FF7ECF12966EAE1CAF5F
:10965C001B7C00AD1A125EA28F45EF2513F544D288
:10966C005122EFF5F0A4FCADF0EBF5F0A49CFCE579
:10967C00F09DFDEB8AF0A4FAABF0EF8EF0A49AF813
:10968C00E5F09BF9E833F8E933F97B00125F480504
:10969C001AE51B2BF51BE4351CF51C22EA2511F9E8
:1096AC00244C5001F9C2D11296C7303D428F00C3F1
:1096BC00EA9511F9500324B4F9D2D17C09E4FDFEEA
:1096CC00FF8982E060062FFFE43EFE0D09B9B4026B
:1096DC007900DCEDED20D118F51E24FE923D500FE3
:1096EC00125EAFEFB503005006851E1FFB881222D9
:1096FC00F51D80E61296A8203D43740212979F1226
:02970C0096A81D
:10970E00203D3874041297A71296A8203D2D74069A
:10971E0012979F1296A8203D2274081297A71296B0
:10972E00A8203D17740A12979F1296A8203D0C741C
:10973E000C1297A71296A8203D0122C3E89F6050F5
:10974E0088148F158A1640081ABAFF0A7AB3800653
:10975E000ABAB4027A001296A8303D34C3E89FF9D3
:10976E00602EC3E5149515FB6930E7D4E930E703A5
:10977E00F404F9EB30E702F404C3995002AA16E59B
:10978E00142515C82F28FFE4FC33FE7D04125EA2BB
:10979E00222AFA244C5001FA22C3CA9AFA50032400
:1097AE00B4FA2212188E85BF6C85BE6B756A0002E4
:1097BE00B174129CEB852E72E55F030354C0F8E57D
:1097CE005E543F28F57C3055062212B0ED80031210
:1097DE00B0DD7410256A54F0F56AE4356BF56BE470
:1097EE00356CF56C24815003756C0022756A00E4AB
:1097FE00D380E8E54B75F010A4256A54F0F56AE5C0
:10980E00F080D8E56A24F054F0F56AE56B34FFF584
:0E981E006BE56C34FFF56C24815003756C7E95
:10982C0022E56A24FF80E4E56D24F054F0F56DE543
:10983C006E34FFF56EE56F34FFF56F2481500375C0
:10984C006F7E221298AB129908C22DC254C255E5F4
:10985C007F7002D255147002D254E54A30E00122D6
:10986C00B4062120540C129811129BBD129C6C0250
:10987C009D02129DE37E0412F130754A0112F12A09
:10988C00756A202220550C1297E0129C3D129CEB1D
:10989C00029B96129DE37E0412F130754A0522124A
:1098AC00B17C7870E4F5F7E4A6F708B880F6D2B28C
:1098BC0022129939756D1012B191E4F5F7E4E5F7C0
:1098CC00D2B264C0702D756D1E12B191E4F5F7E43F
:1098DC00E5F7C4F9E4F5F7E4E5F7D2B2C4F8E954D6
:1098EC000FFD5301F0E8540F49FCE854F0FB7F03E3
:1098FC00129B28056EE56E540370B922E575F85479
:10990C001F30E40244E0F57585722EA2779226E5AD
:10991C007C543F30E50244C0F55EE57C54C0232303
:10992C00F55FE57FC2E779BCF709A77E22856C6FEE
:10993C00856B6E856A6D22856F6C856E6B856D6A25
:10994C0022FA7420303B0274608510F0A4256EF569
:01995C004DBD
:10995D00E5F0356FF54EEA2323303B0475F003A493
:10996D00254DF54DE5F0354EF54E754C00227580C3
:10997D0000C2B212F138D2B222758000C2B2F5F730
:10998D00A4D2B222758000C2B2F5F7A48DF7A48CD3
:10999D00F7A48BF722EB241054F0FBE43CFCE43DE0
:1099AD00FD22EB24F054F0FBEC34FFFCED34FFFD15
:1099BD0022758000C2B2F5F7A4856FF7A4856EF706
:1099CD00A4856DF722E56D241054F0F56DE4356E28
:1099DD00F56EE4356FF56F22756D00E56E24045458
:1099ED00FC80EDE56D24F054F0F56DE56E34FFF57A
:1099FD006EE56F34FFF56F22756D00E56E24FC5436
:109A0D00FC80EC758000C2B2F5F7A4854EF7A485F5
:109A1D004DF7A4854CF722740F254CF54CE4354DCC
:109A2D00F54DE4354EF54E2274F1254CF54CE54DD2
:109A3D0034FFF54DE54E34FFF54E22754C00E54DE6
:109A4D0024FC54FC80EC7403129A1075A70090044A
:109A5D000075F700A4E5F7F0A3E58324F850F2753F
:039A6D00F700A45B
:109A7000E5F7D2B2C23C30E602D23C754C00E54D6F
:109A8000240454FC80A77403129A1075A700900454
:109A9000007F22129ABB8010E54C2411FBAC4D0CC8
:109AA0000CAD4E740312999175A7009004117F00BC
:109AB000129ABB7FEF129ABBD2B22275F700A4E5CF
:109AC000F7F0A3DFF622D23CE4F56FF56EF56D7486
:109AD000031299BEE4F5F7A4E5F7D2B204600BC215
:109AE0003C1299D2E56F24FE50E5923D227F107919
:109AF000B8740612998674021299BE87F709DFFBC3
:109B0000D2B280337F1079B874031299BEE4F5F7AE
:109B1000A4A7F709DFF7D2B278B9793A12DB770256
:109B20009C8AAD6FAC6EAB6D74061299867402128E
:109B300099918FF7A4D2B2758000C2B275F705A4CF
:109B400075F705A4E5F7D2B220E0EC227403129970
:109B500091E4F5F7A4E5F7D2B222E4FEFF740775AD
:109B6000A704F5838E8274FFF0DFFD75A7002274D1
:109B7000067E007FB0129B5FE4F55AF55B2275A765
:109B800004758306E55A600A75F00A84E5F07002F0
:0B9B9000740AC4F58222307720E55AE9
:109B9B0024024002055A129B7EE55AF0E573F0E56C
:109BAB0074F0E575F0E576F0E577F0E578F075A7FC
:109BBB0000223077F9129B7E7F1074FFF0DFFDE5FA
:109BCB005A24F55003129BE8155AE55AB4FF0205C7
:109BDB005AC3E55A955B50D6755B0080D112993903
:109BEB007F0A056D056D12B191E4F5F7E4E5F7D247
:109BFB00B230E704DF02800512983380E5056D1261
:109C0B00B191129B7EE55A24F6F07F06E4F5F7E45A
:109C1B00E5F7F0DFF7D2B275A700227F42129C2E38
:109C2B00DFFB22302B0C0542E542247C40012275E0
:109C3B004280053FE53FB43C17753F00053EE53ECE
:109C4B00B43C0D753E00053DE53DB41803753D0074
:109C5B00802D302B0C1542E5422483500122754296
:109C6B0080153FE53FB4FF17753F3B153EE53EB40E
:109C7B00FF0D753E3B153DE53DB4FF03753D177874
:109C8B00ABA63A08A63B08A63C121875E5BF253DC6
:109C9B00240C75F0188478AEA6F018600564026089
:109CAB00182216E670121816E67004760C18167841
:099CBB00ACE6909CDE9308F62251
:109CC4000618E608909CDE930466700D760118066B
:109CD400E6640D70047601180622001F1D1F1E1F66
:109CE4001E1F1F1E1F1E1F0542E542B43C0F754276
:109CF400000541E541B43C0575410005402215428B
:109D0400E542B4FF0F75423B1541E541B4FF0575CB
:109D1400413B154022AC40AB41A842EC75F03CA459
:109D24002BFBE435F0FC7A3C125D96EB28FBE43C1B
:109D3400FC22AC3DAB3EA83F80E178AE8604AB3E4E
:109D4400E53FC313F8800C7800121857E5BE75F090
:109D540005A4FBE5BF75F03CA42BFBE435F0FC7ACD
:109D64001E125D96EB28FBE43CFC22129D4BAE04D4
:109D7400AD03129D3E8C148B13121861E5BFFF24B2
:109D8400F650027F01E5BE75F096A4AAF0F9C3ED82
:109D94009513FBEE9514FC924E4B701120110E306E
:109DA400480B75364B3003037536FFD22E304E0206
:109DB400DF1F7A02125D9675A7009004EEECF0A303
:109DC400EBF0C3E5BF9F04BF0102D2E79005CBF0DF
:049DD40022ED29FD56
:059DD800EE3AFE80B52B
:10F11D0012F12612F12612F1267E0480067E02805F
:10F12D00027E017F0080087F6480027F017E00EFF8
:10F13D004E6012E4FD0D1D0DEDC394AD40F7EF1FB4
:10F14D0070ED1E80EA2212F2E590BFF57F0012816C
:10F15D003712F16E12F126753500C200C201C202DE
:01F16D00227F
:10F2D100F5D8D2DCE5F520E7FBE5DA540FFEAFD92E
:04F2E10075D80022BA
:10EED9007F767E0690B6FD128149740412F2D17CC8
:10EEE900007D52125EA2EFF875F00A84C0F07F76B9
:10EEF9007E2312E8BC7E29742E12E8CF7E2ED0E044
:10EF090012E8BC7E35745612E8CF7F6B7E1190EF04
:10EF19004212E8FBE824E04001220423F824E750E8
:10EF290002781812EF32D8FB227F6CE82411FE799F
:10EF39000512F2000E0FD9F922071DFFFFFFE0802D
:10EF4900000020C0000038E0000008F0000038F898
:07EF5900000020FFFFFFE0B4
:10EFDD0012F00530E6022409540F75F00AA4F51558
:10EFED0012F00530E6022409540F25152212F00502
:10EFFD00540F2275F000800875F044800375F007FA
:10F00D00E4206D09D5E0FAD5F0F7D24C229247C233
:10F01D00ACE54F623885504FA26E926D859950C206
:10F02D006FD2ACC24CA2472212F03FC4FA12F03F8D
:10F03D002A2212F00520E603540F22540724092238
:10EF6000E612EF6718E608FAC412EF6DEA540F4490
:10EF700030F924C6E950112407800D75F00A84C0C9
:10EF8000F012EF86D0E0443030530975F00085E090
:10EF9000E0D5F0FA3099FD75F019D5F0FDC299F57C
:10EFA00099623822E53880EC742A12EF946238E5D1
:10EFB0003812EF67800812EF88E53812EF88740D79
:10EFC00012EF88740A80C1744012EF88744080B8D0
:0DEFD000742C80B4742E80B075380080ABB6
:10F2F70085A0835383FE438380858384F0758400D0
:01F3070022E3
:10ED860074A212F2F774A112F2F774A612F2F774D3
:10ED9600A412F2F774C012F2F7742512F2F712EE0B
:10EDA6001775C70375C6FC75B90112AA63740812F4
:10EDB600F2D1EE75F020A4FEEF54F80303032E24DF
:10EDC60092C313FE24EA50027E16EE90EE009325BF
:10EDD600BCFE24E6502024E8401C748112F2F7EEB3
:10EDE60012F2F712EE24744012F2F7742F12F2F7B1
:10EDF60074AF12F2F7227E2680E0F7F7F8F8F9FAF8
:10EE0600FBFCFDFEFF0000000001010202020303FD
:10EE160003A8BCA9BDAABEABBFACC7ADC62288BC01
:0BEE260089BD8ABE8BBF8CC78DC62241
:10F16E00C006C007C5F075A7019000007EB7E58CFC
:10F17E00240340FA12F1901EBEAFF3C5F0D007D0B3
:10F18E00062275A700EE12F2F7741012F2F774044D
:10F19E0012F2F785A08343838185838475A7517FFF
:10F1AE0020E0F0E0F0E0F0E0F0DFF6E4F5A7F58423
:01F1BE00222E
:10F2E50075A711900000E4C583F0C58330E2F8F5F9
:02F2F500A7224E
:10F20000EF20E723EE20E71F20E61C05A7C45403E8
:10F21000F583EE5408C42FF582EE5407240983F5D4
:10F22000F0E045F0F005A72280402010080402011C
:10F23000EF20E723EE20E71F20E61C05A7C45403B8
:10F24000F583EE5408C42FF582EE5407240983F5A4
:10F25000F0E055F0F005A7227FBFDFEFF7FBFDFEE2
:10E87A00FDA42582F582E5F03583F583ED227E003D
:10E88A00906AE57A0475F00512E87A7D05805E7A69
:10E89A000580027A04547FC0E0C083C082C39420FA
:10E8AA005001E4906A9512E88F802E906BF37A05F6
:10E8BA008005906CB07A0675F00712E87A7D0780B9
:10E8CA002C7A0580027A06C0E0C083C082C39420F5
:10E8DA005001E4906C4012E8C1D082D083D0E0228B
:10E8EA00906A0975F00A12E87A7D0A7A07C2D1801D
:10E8FA0002D2D1C0A7C082C083C007C006C0E03020
:10E90A00D10975A704E493FDE493FAEEFB75A70415
:10E91A00EBFEEAFC7901D9067908E493F5D4E5D44B
:10E92A0023F5D420E01612F2300EDCEA0FDDE1D036
:10E93A00E0D006D007D083D082D0A72212F200807E
:10E94A00E890694975F00E12E87A7D0E7A0812E8A5
:10E95A00F79069F175F00212E87AE493FDE4A39363
:10E96A00FACE2408CE7C0812E9787C06AD02ED23A3
:10E97A00FD20E00712F2300FDCF42212F20080F7D9
:10E76500F5D2C2D58036F5D2D2D58030F5D224F691
:10E7750050090E0E24A650030E0E0EE5D2F5D275E5
:10E78500F0648485F0D3C2D57009D2D5742012E81F
:10E79500CF800312E8BCCE2406CEE5D375F00A84FB
:10E7A50085F0D3700A30D507742012E8CF800312A4
:10E7B500E8BCCE2406CEE5D312E8BCE5D222F5D2DC
:10E7C50075F0648485F0D3C2D58022F5D2C2D58098
:10E7D50025F5D2D2D5801FF5D275F0648485F0D3A6
:10E7E500C2D57009D2D5742012E8CF800312E8B5DE
:10E7F500CE2405CEE5D375F00A8485F0D3700A30B2
:10E80500D507742012E8CF800312E8B5CE2405CED3
:10E81500E5D312E8B5E5D222F5D2C2D58035F5D2D9
:10E82500D2D5802F30E70DF404C0E0742D12E89D99
:10E835000E0ED0E0F5D275F0648485F0D3C2D570A4
:10E8450009D2D5742012E89D800312E88ACE2404EB
:10E85500CEE5D375F00A8485F0D3700A30D50774F8
:10E865002012E89D800312E88ACE2404CEE5D31257
:05E87500E88AE5D22253
:10812E0090B9E912813702F16E7E00800E7405FE61
:10813E00F51EE4FFF51DF51F203C3375A700E493F3
:10814E00700122A3B40204051D8003B4010A051FA9
:10815E00EF2409FFAE1E80E612E8CF7D06B4400282
:10816E007D03B421027D02EE2DFE80D27E0075A726
:10817E0000E493700122A3B40204051D8003B40130
:10818E000F051FEF2407FFAE1E80E612E899800848
:10819E00B45B0050F612E89D0EB4210280D30EB4EB
:1081AE00400280CDB42C0280C80E0EB45F0280C196
:1081BE00B45B0040BC0E80B9E60812E8CFEE240690
:1081CE00FED513F42290B72B30740990B72F30736D
:1081DE000390B73402814975F019D5E0FDD5F0FA58
:1081EE0012545712EFC7744F12EFD8744B12EFB6EA
:1081FE00C322C250128244125457D2AC12F0003035
:10820E004C1212F000304C0C12F000304C06D250D2
:10821E00C2ACD322B440E512F005B4400312F0050F
:10822E00B44FED12F005B44BE712F00512F0051243
:10823E00F005C2ACC32230530975F008D5E0FDD568
:10824E00F0FA227F0575F019D5E0FDD5F0FA12543B
:10825E005712EFC7745712EFD8745012EF8874810B
:0A826E0012EF88E56312EF88E56265
:1082780012EF8878D0E612EF8808B8D7F8E6F879D0
:108288005F30E702792FE912EF8812EF8812EF8842
:1082980012EF88745812EF88744312EF88E412EFD3
:1082A80088E8C2E775F00A84C425F012EF8878647C
:1082B800E612EF8808B869F8E612EFB612820040B5
:1082C8000122DF02800A20508B75F0008080D25096
:1082D800C2ACD322128244C250125457D2AC2002EC
:1082E800EF12F000204CE7B440F412F005B440035C
:1082F80012F005B457DAF53812F005B450D212F07E
:108308000512F005F56312F005F56278D012F00554
:10831800F924A0500353015FE924E04002795FA6E5
:108328000108B8D8E8780612F005D8FB12F005FC69
:1083380053040FC4540F75F00AA42CFC249C50025B
:108348007C0078D78601E4B92F02D2E72CF678644E
:1083580012F005F608B86AF812F005E5386003026D
:1083680082D812F00512F005C2ACC32290BEBE80BE
:108378000390BA2E7F2012817A12F16E02F12E75C7
:108388003400C26B12844312F12E1287FAE516608C
:108398000312839F020211128A4F12287312F16E80
:1083A80010002010010280F8128865501312287EF0
:1083B80012837410000D10010280F812281980D75A
:0483C8001285E62212
:1083CC00C26BD22775480A12384B753400128925B6
:1083DC00C26A123FDD106A0512020280ED1202021F
:1083EC0012878C1288E412893178D0E664266044B6
:1083FC00128A4F12287312F16E100038100102808D
:10840C00F8128865501BE96515601812287E1283D6
:10841C007412F12610001D10010280F81228198028
:10842C00BCD26B1289107516078559171238C47592
:10843C00350080960202111287FA12846512893176
:10844C007F1912847F90BEEA7E1212817C7E23E516
:10845C001602E83990C03380EF7862E412847678A3
:10846C00D0745F12847618E4F6227F08F608DFFCDD
:10847C00227F7B7E007810742012E89DCE2404FEAF
:10848C00D8F5221220C37F197E0812817C7E289099
:10849C00BA1A30530390BA1502817CC26B128465F0
:1084AC001284B2020211C25112893190BEE21284BE
:1084BC008F12283F1287FA7F2012844E12F16EE53C
:1084CC0016700512F123803675A6FF305103128108
:1084DC00EE125457D2AC200025306DFA1282DF40D8
:1084EC000C12886540111285E6D25180BB105003E6
:1084FC00128379C25180D1D25112837480CAC2AC1A
:10850C0022D22775480A12384B753400C26B128977
:10851C0025C26A123FDD106A0512020280EB1202BC
:0F852C000212878C1288E412893112853E50DAD0
:10853B0002021190BA2912848F12285812F16EC3BD
:10854B0010001310010510020E80F412825140012D
:10855B002212837980DDD3C2AC22D227C26B75483D
:10856B000A12384B753400128925C26A123FDD108E
:10857B006A0512020280EDD26B12878C1288E4120C
:10858B0087B475B901E5BCB2E7F5BC1255F77516A2
:10859B00078559171238C480CB1287FAE516601F6E
:1085AB0078D0E53D1285D7E53E1285D7E53F12859C
:1085BB00D7765A08765F12DB6D1289100287CB7F54
:1085CB003E7E1190BA0012814902F16E75F00A8459
:1085DB004430F608E5F04430F60822D26B128910CD
:1085EB001287CBE51775F01084240AF54824E85060
:1085FB000375480A12385785585922D22075320014
:10860B00129B5A75A7049007007515001287B47555
:10861B00B901E5BC20E705E515F0801004600D6499
:10862B0082600975BCFF75B90575B9020515E515AD
:10863B00242050D8E58224FE40030286E1A882184C
:10864B007F0075A7007583078882E0FE75F004A490
:10865B0012875FA9BCAABDABBEACBF1582E0FD758E
:10866B00F004A412875FC3E995BC404C7052EA95A5
:0D867B00BD4045704BEB95BE403E7044EC99
:1086880095BF4037703DEE75F004A40412875FA9CA
:10869800BCAABDABBEACBFED75F004A40412875FE5
:1086A800C3E995BC4015701BEA95BD400E7014EBEC
:1086B80095BE4007700DEC95BF5008EEF00582EDB1
:1086C800F01582E5826009C3EF9582500302865552
:1086D8000FC3E89F400302864D75A70490070075F5
:1086E800C70375C6A8E0F5BCE0F5BDE0F5BEE0F54A
:1086F800BF75B90575B90205C6E58224204006E5AF
:10870800C6242050E00875C70375C68075B901E511
:10871800BC128749F5BCE5BD128749F5BDE5BE1217
:108728008749F5BEE5BF128749F5BF75B90205C689
:10873800E5C6245850D6E5320470FB75A700C22060
:1087480022B4FF0122F975A704900700E58268604A
:1087580005E06970F7E922F5C685F0C775B901E546
:10876800BC645F700375BC27E5BD645F700375BDAD
:1087780027E5BE645F700375BE27E5BF645F7003BD
:1087880075BF272275C703E54875F004A42480F552
:10879800C6E55975F00484A8F00825C6F5C675B96C
:0787A80001A9BCAABDABBE94
:1087AF00ACBF861522E515242050037515DFE5159E
:1087BF0075F004A454FCF5C685F0C722E5172420F4
:1087CF004028E51775F00484A8F00824A8F5C675AD
:1087DF00C70375B901A9BCAABDABBEACBFA61589AD
:1087EF00BC8ABD8BBE8CBF1255F722E4F516F5156A
:1087FF0079FF1287B475B901E5BCB4FF040516A95A
:10880F00150515E515242050E9891579FF75C7035E
:10881F0075C6A875B90109E5BC04601B09E5BD045F
:10882F00601509E5BE04600F09E5BF04600905C6C0
:10883F00E5C6242050DD098917227516007515012C
:10884F001287B475B901E5BC20E70205160515E5D9
:10885F0015242050EB227900E975F004A454FCF59F
:10886F00C685F0C775B901E5BC20E73078D06670D2
:10887F002B08E5BD66702508E5BE66701F08E5BFCD
:10888F0066701905C675B90108E5BC66700E08E576
:10889F00BD66700808E5BE667002D32209E9242080
:1088AF0050B6C3221288D31288BBA8017F08E0F606
:0C88BF0008DFFB221288D31288CBA8012E
:1088CB007F08E6F008DFFB2278D0796275A7047584
:1088DB008307EBC454F0F582221287B478D0128848
:1088EB00FEE5BCF9C23C20E702D23C1288FE78625E
:1088FB001288FE75B901A6BC08A6BD08A6BE08A6BF
:10890B00BF0805C622D2201287B478D012811C1260
:10891B00811C786212811C02811C12646F12F2E5B9
:10892B00129F2502F16E12F2E57F007E0990BECFF9
:10893B001281497F0A7E12E5150412E7717F14122A
:10894B00DD5E1228197F277E0875130778D01281F8
:10895B00C6E6793E30E702792F7E34E912E8CF7F05
:10896B003D7E0190C04F12817C20311B30300312B1
:10897B00C1F5C23B128BE1128997D23B128BE112EC
:10898B0089A9128C28807C12D3DA80E6C23B7F4403
:10899B007453201702744E7E0012E8CF8017D23B1F
:1089AB007F4F745720170274457E0012E8CF7E0666
:1089BB00E51E12E8BC7E0CE51D12E8BC7E12E51C20
:1089CB0012E8BC7E17748112E8CF7E1CE51B12E8FF
:1089DB00BC7E22E51A12E8BC7E28742E3026027467
:1089EB002712E8CF7E2DE51912E8BC7E33E518126D
:1089FB00E8BC7E39302607742C12E8CB7E3BE5377A
:108A0B0002E8BC742D201702742B7F707E1512E8C0
:068A1B00CF128A2C7E3A06
:108A210012E71A7E0190C07A0281497E1BE51C1271
:108A3100E8BC7E21E51B12E8BC7E27E51A12E8BCE2
:108A41007E2DE51912E8BC7E33E51802E8BC128AD6
:108A5100CD128AF8128DCF128931128E2720171E5E
:108A610010021B12B23B12DB6D128AB51228247F51
:108A7100347E2F1281D312896A12F16E80E212289C
:108A810019203026203128C23B128BE1128B0D7840
:108A910066128CE1D23B128BE1128B227869128C27
:108AA100E1128C28128B9C028D8412C2BE80F212BC
:108AB100D3EF80EDE57D75F01084AAF075F00AA47E
:108AC1002A547FFA78D7E654802AF6227F277E0837
:108AD10079D08700C001D224B9D002C224128EAE4F
:108AE100D001A70010230909EE2406FEB9D7E3221D
:108AF10019EE24FAFE80DB7E3479D7E7A2E79217DC
:108B0100128E5B79D7E7A21792E7F722C224C23B04
:108B1100751E007F447E00128E6B801E1023ED8037
:108B21002AD23BC2247F4F7E00128E73D2247E064E
:108B3100E51E128EA0F51E1023E7D2247E0CE51D42
:108B4100128EA0F51D303BD41023E1D2247E12E514
:108B51001C128EA0F51C1023E17E1CE51B128EA0B9
:108B6100F51B1023E67E22E51A128EA0F51A1023BA
:038B7100E87E2D6E
:108B7400E519128EA0F5191023E87E33E518128E3C
:108B8400A0F5181023E87E393026027E3BE5371223
:108B94008EA0F5371023E3227F707E15128E63C2F8
:108BA400247E1BE51C128EA0F51CD2247E21E51B1D
:108BB400128EA0F51B1023E77E27E51A128EA0F56E
:108BC4001A1023E67E2DE519128EA0F5191023E85C
:108BD4007E33E518128EA0F5181023E82278D7E624
:108BE400C2E775F00A847866F537303B0578698505
:108BF400F037128C5130262BE53775F003A40404AA
:108C040075F00584FBE51975F00AA4251875F006BE
:108C1400A42BFBE435F0FC125FBEF537125FBEF502
:108C2400188B1922E563FC339217AB625003126070
:108C34002F305C0A7AD2125DA47840125F46AE04EB
:108C4400AF037C277D10125EAF8F1C8037E6FD33A7
:108C5400921718860418860350031260377A09792C
:108C64002778C0125F438B1EADD3ACD2AB0679EA32
:108C74007860125F418B1DAF06AED27C177D7012F7
:108C84005EAF8F1CAF05AE047C037DE8125EAF8F30
:108C94001BAF05AE047C007D64125EAF8F1AED75C8
:0A8CA400F00A84F51985F01822EC9F
:108CAE00339217500312602F751D30301786751DC5
:108CBE002D808178427B607CEA800678407B207C28
:108CCE004E12D4BA79277810125F418B1CAF06AEC4
:108CDE00D280AB30262AE51975F00AA4251875F056
:108CEE000AA42537FBE435F0FC7A05125D968C0656
:108CFE008B077C007D03125EA28E048F03128C1BE9
:108D0E00E51E75F00AA4251D75F00AA4251C75F044
:108D1E0006A4251BFBE435F0FC7A0A125D96EB25C2
:108D2E001AFBE43CFC7A0A125DA4EB2519FBE43C29
:108D3E00FCE43DFD7A0A125DB6EB2518FBE43CFC23
:108D4E00E43DFD301703126037A60518A60418A6D9
:108D5E000378D7E6A2E7923DC2E775F00A84FCAB32
:108D6E00F0303B0EAB37EC75F00AA42BA23D92E728
:108D7E00F622AC3780F0128D9F305C0A7A40125D7D
:108D8E00A478D2125F4630170312602F8C638B6269
:108D9E0022128DAF7A0A125D96EB2518FBE43CFC8D
:108DAE0022E51C75F00AA4251B75F00AA4251AFBF2
:068DBE00E435F0FC7A0A26
:108DC400125D96EB2519FBE43CFC22128E0112F194
:108DD4002AC202C223128E011000081001051002DB
:108DE4001B80F51031ED10300D102604D22680E3DF
:108DF400D230C23180DDD231C23080D7227F35906B
:108E0400C03812817A90C05620300F90C072203141
:108E14000990C04720260390C03F1F7E1712814946
:108E240002F16E7F357E0190B9DC12817C7F347E45
:108E34003A128F50744E12E8CF12F16E12F12AC218
:108E4400027F347E3AD21775115975124E802675F9
:108E5400112E751227801E75113E75122F801675FE
:108E6400112B75122D800E75114E751253800675D7
:108E74001145751257128F50E511301702E5121281
:108E8400E8CF12F16E10000810010510020B80F5F6
:108E9400D23C1017E3D21780DF028F4B4430F81214
:108EA4008EAAE8540F22C2218002D221A224922247
:108EB4009223128F50E830E709D23C7430302102FB
:108EC400745FF812E8CF12F16E100034100105102F
:108ED400025D80F5D23C102266102367B439097410
:108EE4005F2021DF743080DBB45F04742D80D4B440
:108EF4002D04744180CDB45A04743080C60480C3F8
:108F0400D23C302406102237102338B44104742D87
:108F140080B1B42D04745F80AAB45F04743980A353
:058F2400B43009745A8D
:108F290020219B74398097148094B48908D223E84E
:108F390012E8CF800DF8C223800874898001E80205
:108F49008EC7908F9A8003908F96C007EF2408FFF1
:108F590012E8FBD00702F16E128F50E830E704D215
:108F69003C7441F812E8CF12F16E1000081001119B
:108F79001002CF80F5D23CB44104745A80E51480C4
:108F8900E2D23CB45A04744180D90480D60205F86F
:058F9900F802050000D4
:10F0BD0075A70090F0EF75F02D84C2D5C2D1601701
:10F0CD00D2D1146007D2D514600DC2D1E5F093FCF6
:10F0DD00742D95F093FB22E5F093FB742D95F09331
:10F0ED00FC220009121B242C353E474F58606870D6
:10F0FD007880888F969DA4ABB2B8BEC4CACFD4D940
:10F10D00DEE2E6EAEDF0F3F6F8FAFCFDFEFFFFFFB6
:10F1BF00D23D8002C23DED8BF0A430E70205F0C3D3
:10F1CF00E895F020D50425F025F0FEED8CF0A43065
:10F1DF00E70205F0C3E995F030D10425F025F0FFE3
:10F1EF00203D0B2487500122EF24CC40012202F254
:01F1FF00000F
:10EB4B00203A7A7E1C7F5312F2007F5912F2001E7C
:10EB5B007F5712F2007F5512F2007E2312F2007FD4
:10EB6B005712F2001E7F5912F2007F5312F2001F50
:10EB7B007E2012F2007F5A12F2007E1E12F2007FEC
:10EB8B005212F200121861E5BD20E0143006117F1D
:10EB9B00357E1C90EC09E571700390EC1302E8FBD9
:10EBAB00E5716018E57012F0BD781F79567D09127A
:10EBBB00F1C3303A0312EBDC0DBD16F3227E1C7F42
:10EBCB005390EBF212E8FB200CD67E1F12DDC580B2
:10EBDB00BEC0060E30D5021E1E12F200D0061F302C
:10EBEB00D1020F0F02F200070700386C446C38009B
:10EBFB0005052070D8702005057088A88870080757
:10EC0B0010387CFE383838000807102844C62828EE
:02EC1B003800BF
:10DB990090C0847F717E2312817C121861E5BC7E5E
:10DBA9003112E88A30121AC23C121861E5BCFB75C1
:10DBB900F00AA4F904FAC23D12993912DE3C303D4B
:10DBC9000122DAF712DD3E7C00EBF4042E4019AD98
:10DBD90003125EA2EFA2D1203C077E237F6502E4F7
:10DBE900E7AE16AF1702DCDFAD01125EA2EF12E558
:10DBF900D5203C077E237F6502E50BAE16AF1702E1
:10DC0900DD037F567E0512DD6A7F3D12DD7D7F6F64
:10DC190012DD7D12DDC57E0A7F4112DDF87E227F8D
:10DC29005912DDF820120122129939857A1D855E73
:10DC39001C857B1B855F1A7AC0C23D12DE38203DE8
:10DC49005212DD3E7C007D14125EA274562F20D143
:10DC5900029F9FFF24CB40028037EF248850028027
:10DC690030EA1475F00384FE12F200C3E51B957BBC
:10DC7900FEE51A955F92D55004EEF404FEEEC31347
:10DC8900FE24E0400C741F2E30D5029E9EFE12F237
:10DC990000DAA8227F5212DCAF7F5A12DCAF751767
:10DCA90053751600802B7E0012F2300EBE12F92237
:10DCB9007F157E28742012E8CF7F1C7E2812F2304F
:04DCC9000EBE40F952
:10DCCD00223012E712DCB975171575162DD23C02EC
:10DCDD00DBB2C23D6002D23D92D175F080305C0462
:10DCED00F5F08001A4A2E792D5E5F075F03284F845
:10DCFD00E5F075F00584C0E0E5F0A2D533C0E0E8AD
:10DD0D00601E12E8BCEE2406FED0E0F8D0E012E86A
:10DD1D00BCEE2406FE742C12E8CF0E0EE802E8BC11
:10DD2D007420303D07742B20D102742D12E8CF8062
:10DD3D00D4C3ED957AFFEC955EFE92D1500312603F
:10DD4D001F227F1512DD567F327E3E12F200DEFB62
:10DD5D00227E0912F2000EBE36F9227E0112F20069
:10DD6D000E0EBE3FF8227E3312F2000EBE40F92297
:10DD7D007E047D1112F2000E0E0EDDF81F1F7E3592
:10DD8D0090C08D305C057E3190C09102817C740510
:10DD9D00305C097E32740112E88A74067E3612E810
:10DDAD008A7E3A740012E88A7E3D02E88A7F151257
:10DDBD00F2000F0FBF2DF8227F417E1F7D0F12F253
:10DDCD00000F0F0FDDF8227F687D0380047F677DD4
:10DDDD000512F2000FDDFA227F667D0780F37E1FAC
:07DDED007F5012F2001F1F1E
:10DDF400BF3EF8227D0A12F2000E0E0F0FDDF7224D
:10DE0400203D071248B47003D23D22056D12B19132
:10DE1400E4F5F7E4ABF7F5F7E4E5F7FA30E411EBF2
:10DE2400251DF51DE4351CF51C0519EA30E3010E2A
:10DE3400D2B28015780380027801203D071248B4DD
:10DE44007003D23D22D8F3056DE56D2409F56D12FA
:10DE5400B191E4F5F7E4ADF7F5F7E485F71BF5F7D1
:10DE6400E4E5F7FCD2B2543F30E50244C0CC54C0E0
:0BDE74002323F51AE56D24F6F56D225E
:10EA72007E017F0990EAF012E8FB2051097E037FB4
:10EA820000743F02E8CFE4FEFFC3E54512E310FD48
:10EA9200940AED403D9464ED4002746312E76B7E8C
:10EAA200017F09E552240575F02D84AAF075F00561
:10EAB200A4CA75F00B842A90EADB9312F0BDBCB8AD
:10EAC200027BB87D04EE2DF8EF2DF90D12F1BFDDBA
:10EAD200FB227E0312E8BC80C6000C1622222D39CE
:10EAE200444F4F5A66707C7C87939EA9A9000909FE
:10EAF2000800410000000000888000000000410082
:10EB02000800121875E5BCB4F8339004C3E0602C19
:10EB1200FA24F340277F137E0012F2000F0F12F245
:10EB2200000E12F2301F1F12F2300EDAEC7F147E4A
:10EB32000012F2000E12F2300EBE12F5229005CC37
:09EB4200E0C3941240F60480C700
:10E31000305D0A75F08AA42480E5F0340022207470
:10E32000157F017E1190E39812E8FB7F0A7E0AE5D3
:10E330002E540702E7827F087E1190E3A812E8FBC3
:10E3400020730C7F0A7E1712F2300E0E12F2307F0D
:10E35000007E0BE57112E31012E7717F0C7E11E570
:10E3600071602F0EE57064B4602864B475F0328477
:10E37000C0F012E8B5CE2405CED0E075F00584C01B
:10E38000F012E8B5CE2405CED0E023302D010402F2
:10E39000E8B590A121028149070FFFFFC473BDAF0B
:10E3A000A463B5FBCDE7FFFF030F0100FFFE038071
:10E3B000306701227F3F7E00748812E8CFE551600C
:10E3C000F212187A85BCF01207A512E31075F064FA
:10E3D00084F87E06E5F012E7D0E860D77E0002E818
:10E3E000BC12187AE5BE70012214600814603BE587
:10E3F0003F1340367F367E00747712E8CF207301DA
:10E400002279BC8704098703125D3E7E05781DE6EC
:10E4100060097E0012E8B5EE2405FE18E6600712DA
:10E42000E8B5EE2405FE18E6801990B8B67F377E71
:10E430000012817CAB60AC61125D411F7E09781DCA
:10E44000E6600712E8B5EE2405FE18E612E8B5EE20
:03E450002405FEA2
:10E4530018E602E8B5202C012290E46202E8FB05ED
:10E463000EFFF0E01CF004F81CFFF0301201227FD5
:10E47300637E0090B74612E8FB7F1512DD567F1FBF
:10E4830012DD567F2912DD567F177E06E53F30E009
:10E493000B90C0A1305C0390C0B5800990C096304A
:10E4A3005D0390C0AB1281497F2190B7722074063F
:10E4B30090B766028137E53770F9E53F20E0F43025
:10E4C30073F190B77E1281377E1BAC4EAB4D12E6D3
:04E4D3009602E71AAC
:10E63D00125D3E7F207E05751900781DC2D5E6302E
:10E64D00D51712E8B5EE2405FE18B818F17E1F7423
:10E65D0063305C02748202E8CF7005B8191880E24D
:10E66D00D2D5CE24FACE7484301702742D12E8CF91
:10E67D00EE2406FE80C8742012E8CB80C8781C807A
:10E68D000D7F007E23AC5EAB7A125D3E781DC2D548
:10E69D00E630D50C12E8BCEE2406FE18B818F122AF
:10E6AD007005B8191680EDD2D53017E4CE24FACE08
:10E6BD00742D12E8CFEE2406FE80D5742012E8CF1B
:10E6CD0080D5125D3E781DC2D5E630D51612E88A8A
:10E6DD00EE2404FE18B818F10E745E305C02742737
:10E6ED0002E8997005B8191680E3D2D53017DACE45
:10E6FD0024FCCE742D12E89DEE2404FE80CB7420F4
:10E70D0012E89D80CBC23D12E7250F0F0E0E7463EC
:10E71D00305C02748202E8CF125D3E781DC2D5E6F0
:10E72D0030D50C12E8EAEE2408FE18B818F1227064
:10E73D0005B8191680EDD2D5301716740BCE24F806
:10E74D00CE12E8EAEE2408FE80D5740C12E8EA80B9
:08E75D00D5303DCB740A80E5C4
:10EC1D007F797E24E55F30E70122AC5F1CAB7B1270
:10EC2D005D6CE51B700E742012E8CFEE2405FE120C
:10EC3D00EC6B800C12EC6BE51B12E8B5EE2405FEB7
:10EC4D00E51A12E8B5EE2405FE742C12E8CF0E0E6F
:10EC5D00E51912E8B5EE2405FE745E02E8CF742DB9
:10EC6D00201702742B12E8CFEE2406FE22E55F304A
:10EC7D00E70122AC5F1CAB7B125D6CE51B700E7463
:10EC8D002012E89DEE2404FE12ECC4800C12ECC49C
:10EC9D00E51B12E88AEE2404FEE51A12E88AEE243A
:10ECAD0004FE742C12E89D0E0EE51912E88AEE246E
:10ECBD0004FE742A02E89D742D201702742B12E8AD
:06ECCD009DEE2404FE226E
:10E4D7007F097E2530040512E5D18028A275E579EC
:10E4E700C23D6002D23D92D175F080305C04F5F0F8
:10E4F7008001A4A2E792D5E5F075F03284F8E5F043
:10E5070075F00584C0E0E5F0A2D533C0E0E8602AE5
:10E5170012E8EAEE2408FED0E0F8D0E012E8EAEECE
:10E527002408FE0F0FE52B5403701F746012E8CF09
:10E537001F1FEE2404FEE802E8EA740C303D06745F
:10E547000A20D1010412E8EA80C9205904742E80F8
:10E55700DC205804747F80D5748080D13004051284
:10E56700E5D18028A275E579C23D6002D23D92D1FE
:10E5770075F080305C04F5F08001A4A2E792D5E540
:10E58700F075F03284F8E5F075F00584C0E0E5F049
:10E59700A2D533C0E07F3E7E1CE8602012E94BD055
:10E5A700E0F8D0E07F3E7E2812E94B7F447E32744C
:10E5B7002E12E8CF7F3E7E37E802E94B303DE0740C
:10E5C7000A20D1010412E94B80D59005CAE075F005
:10E5D7000A84F8E4C5F0C2D522301105E54AB40231
:10E5E70050C39006E9E0957AFB9006E8E0955EFC5B
:06E5F700500312602FEC3E
:10E5FD00C31360047B63800FEB13FB249C40F52455
:10E60D004F4004C20480079005CAEBF0D204900677
:10E61D00E6E09006E8F09006E7E09006E9F0E55EAA
:10E62D009006E6F0E57A9006E7F02212E61B80DE12
:10DE7F00E54424F64001227800E552206607C39559
:10DE8F0070500224B40475F00384F9E928FE24C409
:10DE9F005001FE12DEC112DECD1E12F200C3E99850
:10DEAF00FE5003243CFE12DEC11E12F20008B81F02
:10DEBF00DA22EE2420FE24C250032402FE22E8249C
:10DECF00F1E8C2D55006D2D5E8F4241F23FF90DF26
:10DEDF004F93CF0493FAE545F5F0A4ACF0FB125D38
:10DEEF00CDE544F5F0A49BFBE5F09CFCEB2420FB77
:10DEFF00EC3400FC12DF30FAE5458FF0A430E70276
:10DF0F0005F0E5F020D502F4042A75F00520190379
:10DF1F0075F00384FF24DF50027F20C374329FFF0C
:10DF2F0022EC24F0500BEB2460EC340090DF9F9335
:10DF3F0022EB33FBEC33FCEB33EC3390DF6F9322AC
:10DF4F00FF00FF03FA0BF318EA2ADE40CF58BE7327
:10DF5F00AB8D96A880C068D64FE835F51BFD00FF46
:10DF6F0000080B0E101214151718191B1C1D1E1F5D
:10DF7F0020212223242526262728292A2A2B2C2D27
:10DF8F002D2E2F2F3031313233333434353636375F
:10DF9F00373839393A3A3B3B3C3C3D3D3E3E3F3FBB
:10DFAF004042444648494B4D4E505253555658598E
:10DFBF005B5C5D5F60616364656668696A6B6D6E0B
:10DFCF006F7071727374767778797A7B7C7D7E7FD0
:10DFDF00808182838485868788898A8B8B8C8D8EBE
:10DFEF008F9091929394949596979899999A9B9CC8
:10DFFF009D9E9E9FA0A1A2A2A3A4A5A6A6A7A8A9E5
:10E00F00A9AAABACACADAEAFAFB0B1B1B2B3B4B413
:10E01F00B5B6B6B7B8B9B9BABBBBBCBDBDBEBFBF4D
:10E02F00C0C1C1C2C3C3C4C5C5C6C7C7C8C8C9CA92
:10E03F00CACBCCCCCDCECECFCFD0D1D1D2D2D3D4E0
:10E04F00D4D5D5D6D7D7D8D8D9DADADBDBDCDDDD36
:10E05F00DEDEDFDFE0E1E1E2E2E3E3E4E5E5E6E691
:10E06F00E7E7E8E8E9EAEAEBEBECECEDEDEEEEEFF3
:10E07F00EFF0F1F1F2F2F3F3F4F4F5F5F6F6F7F75A
:10E08F00F8F8F9F9FAFAFBFBFCFCFDFDFEFEFFFFC9
:10E09F00E54524FD400122E552206607C3957050E7
:10E0AF000224B40475F00384241FFE24C2500324F9
:01E0BF00025E
:10E0C000FE12DDBAEEFD241EFE24C250032402FE21
:10E0D00012DDBAE544240275F00520190375F0033A
:10E0E00084F4042432FF24EE500F12E0EFAE051E3C
:0AE0F0001E7C0512F2000EDCFA227D
:10E98A007E00206615E5700475F0B484E5F075F034
:10E99A000384FE6004C3743C9EFE745312E9B5748A
:10E9AA005712E9B5744E12E9B574457F2F12E89DE6
:10E9BA00BE00077E3C12E89D7E00EE240875F03CFE
:10E9CA0084AEF00F0F0F12F2000E12F2000F12F2C5
:10E9DA00001E12F200EE240775F03C84AEF02230DD
:10E9EA00745C301259E54AB4040122B4060122E5E6
:10E9FA007112DF198F057C037E1E30662AE57004CA
:10EA0A0075F00384241EFE24C6501C24FB500424E3
:10EA1A00038013C00612EA31D0E024C67C016006E6
:10EA2A000C1460020C14FE12EA3D0EEE24C14002E0
:10EA3A00DCF5228D0712F2000FEF24CE50F722E503
:10EA4A0053206607C39570500224B40475F00384FA
:10EA5A00241FFE24C250032402FE12EA680E7F23FA
:08EA6A0012F2000FBF2DF9228A
:10F260007E0E78ADE612E7D0EE2405FE742C12E88F
:10F27000CF0E0E0E18E612E7D0EE2405FE742C1207
:0AF28000E8CF0E0E0E18E602E7D0EC
:10E0FA007F017E00745212E8CF7E06E51512E7D63C
:10E10A007F0A7E0178B8E67D0130E5027D03ED12D3
:10E11A00E8BC7E07E67D58A2E4922B50027D46EDCC
:10E12A0012E8CF7F017E1812F2627F0A7E1378AE60
:10E13A00E612E765EE2406FE743A12E8CFEE2405ED
:10E14A00FEE53E12E765EE2406FE743A12E8CFEECB
:10E15A002405FEE53F02E7657F797E00E54012E788
:10E16A00D07E0A743B12E8CB7E0CE54102E7D07FF1
:10E17A00797E16743B12E8CB7E18E53F12E7D07F12
:10E18A00797E0078AEE612E7D07E0A743B12E8CBBD
:10E19A007E0CE53E02E7D0305EE52043E27F6D7EED
:10E1AA000078AEE612E7D07E0A743B12E8CB7E0C0A
:10E1BA00E53E12E7D07F757E00E53E75F00A84E5FC
:10E1CA00F012E8EA0F0F7E08743A12E8CB1F1F7E9E
:10E1DA000DE53F75F00A84C0F012E8EAEE2408FE65
:10E1EA00D0E002E8EA851C1E851B1FAB1BAC1C3065
:10E1FA005D0A7A1B125DA47832125F46C3EB33FBC9
:10E20A00EC33FC923D125D75303D087409F51DF53D
:10E21A001CF51B7F75E51D60157E2412E8EA7E2C2D
:02E22A00E51CF1
:10E22C0012E8EA7E34E51B12E8EA803D7E22E51C0A
:10E23C00601912E8EA7E2AE51B12E8EA7F787E3143
:10E24C00742E12E8CB7F75E51A8019E51B12E8EAEB
:10E25C007F787E29742E12E8CB7F757E2DE51A12FD
:10E26C00E8EAE5197E3512E8EA7F777E3C1267050D
:10E27C00851E1C851F1B227F397E1F12F2000FBFCB
:10E28C0040F9781F79567A007D1A12F0BD12F1C34D
:10E29C00EA2406FABAAEF3781BC3E5119570500266
:10E2AC0024B4FA604214603E14603A2450603A146C
:10E2BC006036EA24A540278A1E751D007D1912E2DE
:10E2CC00D50D30740312E2D50D781F7956AA1DEACC
:10E2DC0012F0BD12F1C30AD3EA951E40F2228A1D38
:10E2EC00751EB380D7080808087F367E1C90EC0991
:10E2FC00E571700390EC1312E8FB7F3CAE00908F3D
:04E30C009602E8FB92
:10EE3100787512EE817453201702744E207406E522
:10EE41002E54074430AF1712EEAB7E3BE57DC45420
:10EE51000F12E8BC2074077E07742012E8CF78787F
:10EE610012EE81E5172409FF74572017027445201B
:10EE71007402742012EEAB7E3BE57D540F02E8BCB8
:10EE8100E6FD3392171886041886033017031260C3
:10EE91003779177870125F418B13AF06AED27C00C1
:10EEA1007D64125EAF8F148D15227E0012E8CF7E35
:10EEB10007E51312E7827E19748112E8CF7E20E5FF
:10EEC1001412E7657E2B742E2073030E742C12E846
:08EED100CF7E2FE51502E76575
:10F04D00E54A602E7A2420E00E7A26141460087AA0
:10F05D0028141460027A297F667E01EA12E8CF2017
:10F06D005505205406800B745B8002745C7E001283
:10F07D00E8CF20110778A9B60007802130261EC2DF
:10F08D002690B80C7F661281377F64A85AE54AB482
:10F09D00060108E875F06484E5F012E1DD20080F43
:10F0AD00E537640260097F367E2E744112E89D2299
:10ECD30020144F740512F2D1EF33EE33F9EF03032F
:10ECE300541FF5F090ED26E993A4C5F013C5F01376
:10ECF300C5F013C5F013C5F0135403FCE5F013FB83
:10ED0300E9242093C9244093C39BC4540FFBE99C7B
:10ED1300C4FC540FF9EC54F02B2446F57BE934F68C
:10ED2300F55F22FFFFFFFFFFE6C5AD9C8F857D7773
:10ED3300726E6C6A696A6A6C6F747A828D9DB4D9DB
:10ED4300FFFFFFFAE9DCD3CEC9C6C3C0BEBBB9B768
:10ED5300B5B4B2B0AFADABAAA8A6A4A2A09E9C992D
:10ED630096918C00381CE735D137246F00C5B3C1A9
:10ED7300E61F66B60E68C21867AADBF4EDB94675DE
:03ED830010A200DB
:10F2B100D2A27408D2A1D2A300C2A3C2A1D2A30038
:10F2C100C2A3D5E0EF7405D2A300C2A3D5E0F82212
:10F28A00C2A3D2A2D2A1D2A300C2A375F00833921C
:10F29A00A1D2A300C2A3D5F0F5C2A175F003D2A3EF
:07F2AA0000C2A3D5F0F82219
:10D7C30012F28AD2A300C2A3C2A175F008E4D2A3C5
:10D7D30000C2A3A2A233D5F0F5FE75F008E4D2A3EC
:10D7E30000C2A3A2A233D5F0F5FFD2A300C2A322A5
:10D7F300E478806608B88BFB70012274D512D7C316
:10D803007881C3EE13FEEF13F692D118EE2460F67F
:10D8130074D612D7C37888EF33CE33CE33CE33CE1C
:10D8230033A2D192E25407FCEEFB7A08125D96EC28
:10D83300244FF608EBF674D912D7C3EF543F78821E
:10D84300F67886EF33CE33CE33CE33CE335403F66E
:10D8530008EEF618161608E6C4FF54F0F618E6C4E8
:10D86300CF540F2FF674DA12D7C3EF232354FC7867
:10D8730083F67884EEF608EF54C0F67880E4660801
:10D88300B88AFBF62212D7CB7889C3EF96FF18EE3E
:08D8930096FEA2E79216501068
:10D89B0012601F740FF8F9125DE3EF2CFFEE3DFEE3
:10D8AB00788BEEF608EFF622E6182016072CF7E633
:10D8BB003D19F722C39CF7E69D80F66A405E8056C1
:10D8CB00E050F04B0044803DC0384031D02BA025B8
:10D8DB00601F2018D014000F000AA001440158014A
:10D8EB00680178018801A001B401D001EC0210029B
:10D8FB0038026802A002DA030C034D78BE80208543
:10D90B008E8A9D8F4D95BA9A97A0BEA631AC53B215
:10D91B002AB801BD6AC1EDC4D1C78812D7CB788DA7
:10D92B00EEF608EFF67887798C125DE378837990C1
:10D93B0012D8B37885798C125DE37881799212D8FD
:10D94B00B3788DE624E4FE08E63392D13392D554B6
:10D95B00FCFFEEA2D133A2D533FE780F7992125D84
:10D96B00E378947990C3EC97F61819ED97F67994C0
:10D97B0090D8C67F1F7D11EF93C3971F19EF939715
:10D98B001F091DED600240EF0F90D8E6798DEF93E4
:10D99B00F7090FEF93F7788E7994125DE390D90620
:10D9AB00EF93C39BFB1FEF939C2420FC7897E62BF4
:10D9BB00F618E63CF618E436F6740612F2D1EEFCD5
:07D9CB00EFFD740712F2D119
:10D9D200C3ED9FFFEC9EFE78B7E6FD337C0050015D
:10D9E2001CEF2DFFEE3CFE789CEF26F618EE36F685
:10D9F2002220140F789DE6B4050912DA9312DAC8D0
:10DA020012DB0C222014577897799A12DB3D125FB1
:10DA1200A7C3EE9420FE9245500312601F7C007D46
:10DA220005125EAF30450312601F8E618F60E531D3
:10DA3200B40C2B12EE17E56120E71124F8500DFA11
:10DA4200C3E5609AF560E5619400F561121884E51A
:10DA5200BC2560F57AE5BD3561F55E12EE24789756
:10DA6200799AC3E697FB1819E697FC7A02125D963B
:10DA720012DA9312DAC820140312DB0C7895799823
:10DA8200E6F776000809E6F776000809E6F7760079
:10DA920022799CE77700FB19E77700FC789DE6B4D2
:10DAA2000506EB33FBEC33FCECA2E792D5500312F4
:10DAB200602F7A32125DA4ECFBEDFC30D5031260CC
:0ADAC2002FECFEEBFF22EE2408FE1D
:10DACC007406307511789DE6B40504740C8007F467
:10DADC002406C323540FFD7C00125D82789FE6FC64
:10DAEC0008E6FBC374109DFA125DA4EFF8EEF91270
:10DAFC005FA7E878A02FF6FF18EE39F62480FE22F7
:10DB0C009275400312601F78BBE6F5F02438400391
:10DB1C0075F0E1EF33EE3378A8F6A485F07930E7B1
:10DB2C00020579C276307508E57924F15002D27677
:10DB3C0022E627FB1819E637FC1819E637FD227583
:10DB4C006A0079C6876C09876B22756A2080F3128C
:10DB5C00DB4B1298AB7F087871793A12DB79029C17
:10DB6C008A855E63857A62787379647F06E6F70846
:10DB7C0009DFFA227864797380F1787379AF80EBDE
:0DDB8C0078AF797380E5E6F008A3DFFA2298
:105D1C00E4FEFFFC7D0A791DE7540F2FFFE43EFEE5
:105D2C00B91902800619125D8280ED3017031260DA
:105D3C001F22305C2BEC339217500312602FEC2493
:105D4C00D950047C277B007AD2125DA4EB33CC3380
:105D5C00CD33CC33ED33FBEC33FC30170312602F17
:105D6C00EC339217500312602F7919125FBEF709AA
:105D7C00B91DF8A70322EFF88DF0A4FFEDC5F0CE06
:105D8C00A42EFEEC88F0A42EFE22EB8AF0A4FBE5F8
:105D9C00F0CC8AF0A42CFC22EB8AF0A4FBE5F0CC2E
:105DAC008AF0A42CFCE435F0FD22EB8AF0A4FBE590
:105DBC00F0CC8AF0A42CFCE435F0CD8AF0A42DFDB7
:105DCC0022EB8AF0A430E70205F0E5F0CC8AF0A4CF
:105DDC002CFBE435F0FC2286F0E7FDA4FAABF019BD
:065DEC00E786F0A42BFB8A
:105DF200E435F0FC18E68DF0A42BFBEC35F0FCE466
:105E020033FDE687F0A42CFCED35F0FD22EB89F0A2
:105E1200A4CBAEF08AF0A42EFEE5F03400FDEC89AE
:105E2200F0A42EFEE5F03DFDE433CC8AF0A42DFD76
:105E3200E5F03CCEFC22EB89F0A4CBAFF08AF0A4D3
:105E42002FFFE5F03400FEEC89F0A42FFFE5F03ED1
:105E5200FEE433CC8AF0A42EFEE5F03CFCED89F0A2
:105E6200A42EFEE5F03CFCE433CD8AF0A42CFCE544
:105E7200F03D8E058C068F04FF22C2D5EC30E7057B
:105E8200B2D5126027EE30E70DB2D512601F125E56
:105E9200AF1260278003125EAF30D50312601F225B
:105EA200C3EC13C0E0ED132FFFD0E03EFEBC000BAD
:105EB200BE0029EF8DF084FFADF022E4CCF975F03D
:045EC20008EF2FFFB7
:105EC600EE33FEEC33FCEE9DEC994005FCEE9DFEB8
:105ED6000FD5F0E9E4CEFD22EDF9F5F0EE8420D2FF
:105EE6001CFEADF075F008EF2FFFED33FD4007996E
:105EF6005006D5F0F222C399FD0FD5F0EA22EC3315
:105F0600EE3400FEEF3400FF7D007A007900780958
:105F1600C3ED9AFDEE9BFEEF9CFFB392D54009EDD3
:105F26002AFDEE3BFEEF3CFFA2D5E933F9ED33FD4A
:105F3600EE33FEEF33FFD8D92279007A00C38015FD
:105F460079007A00C3EA13FFE913FEE8132BFBEE90
:105F56003CFCEF3DFDE4F5D2F5D333FE7F19C3EEED
:105F660098FEE5D299F5D2E5D39AF5D3B392D5400A
:105F76000DEE28FEE5D239F5D2E5D33AF5D3A2D512
:025F8600EB33FB
:105F8800FBEC33FCED33FDDF0122EE33FEE5D233CB
:105F9800F5D2E5D333F5D380C3AD6FAC6EAB6DED01
:105FA800C454F0FEECC4FF540F2EFEEF54F0FFEB88
:105FB800C4540F2FFF22EC75F00A84FCEB54F02533
:105FC800F0C475F00A84C4CBC454F025F0C475F04D
:105FD8000A842BFBE5F022AC10AB11125FBEA904BA
:105FE800AD03FA7C197B99125D96AE04AF03EA758E
:105FF800F006A4F8AC12AB13125FBE2875F00A8441
:1060080085F014F8EF2BFFEE3CFEEF28FFE43EFE90
:10601800E43DFDE439FC22C3E49FFFE49EFE22E454
:10602800C39DFDE49CFC22C3E49BFBE49CFC22C3CF
:10603800E49BFBE49CFCE49DFD2275D4107B807AF4
:0C6048000079807800EAF5F0A4FCADF0CF
:10605400EBF5F0A4FEAFF0EB8AF0A4C333C5F03344
:10606400C5F092D52DFDC5F03EFEE430D501043FC8
:10607400FFB5150DEEB51409EDB51305ECB5120118
:10608400224006EA98FAEB99FBD5D40ABB00012218
:106094000ABA00010B22C3E913F9E813F8EA28FA53
:1060A400EB39FB80A478087B807D807C00EDF5F0E3
:1060B400A4FAE5F08EF0B5F007EA8FF0B5F001220E
:1060C4004003ED9BFDD827BDFF0122EDF5F0A4F9B7
:1060D400A8F0ED04F5F0A4C399FAE5F09813CA13F7
:1060E40029F9E83AF8C3E99FE89E50010D22C3EB71
:1060F40013FBED2BFD80B6C374689511FB740195F9
:1061040010FC8004AC10AB117A0B79B8125E0F80CE
:10611400177473F8F9E627FB0809E637FC0809E663
:0261240037FD45
:1061260030E703126037EB33FBEC33FCED3323FD32
:10613600242083F8ED241C83FFED241883FAED2434
:106146001483F9EF99F9E89AFA125E0FEF9DFFE8CA
:106156009EFE22FFFFFFB6FED7FD63FB5DF8C4F58A
:106166009BF1E3ED9EE8CFE379DD9ED743D06BC983
:1061760019C153B91CB079A7709E06943F8A237F34
:10618600B674FF6A045ECB535B47BB3BF130042316
:10619600FB17DE0BB2FF80C21DC232532CF8C3E5DB
:1061A600679576FBE5689577FCE5699578FD30E7B8
:1061B60005D26112603724F05003126271AA06A953
:1061C60007125E38EC2480E43DFBF9F51AE43EFC48
:1061D600FAF519E43F6002D232125E0F8B128C136D
:1061E6008D148E15C3E5649573FBE5659574FCE522
:1061F600669575FD30E705D262126037EBF9F51F3B
:10620600ECFAF51DED6002D23230320122125E0F39
:10621600EB2512F512EC3513F513ED3514F514EEE6
:106226003515F51540E102604212619D20323BEBC7
:10623600242E40D3EA2401CB3400FC7A07793D12A0
:106246005E0FC010C0118E108D118C128B13E4FCE2
:0E625600FD7E077FD012D357851203851302F9
:10626400D011D010BB0005BA0002D21D22B261C306
:1062740074809BFB74F59CFC74209DFD22204D6969
:10628400204866303F637F697E0112DD6A7E1F12FB
:10629400DDE575A7009004EDE0A2E792171392E7FD
:1062A400FC1582E013FB30170312602FBC003AEB9D
:1062B400603720E73420E63110E513201707C37454
:1062C4001F9BFE80027E1F12DDDA0EDBFA22FB200A
:1062D40017097E00C374209BFB8008EB241FFE7407
:1062E400209BFB12DDD40EDBFA2275A70075830711
:1062F400E559C4440FF582E0A2E792522212DB86EC
:106304001262EEC2E775F00A84FEAFF075A704537B
:1063140082F17864126377AE07786712637775A7A2
:1063240000E57DC4540FFEE57D540FFF78731263BE
:106334006BAE07787612636B74AF12611712622F1B
:106344008B148A131207D2ACCCAB017A0A125D9675
:10635400E5139B9004ECF0FBA3E5149CF0FCA2E78E
:10636400923DD23F02DB8C8603088604088605181A
:09637400188006E0FBE0FCE0FDEE
:10637D007A0A125DB620E70CEB2EF608E43CF6081F
:10638D00E43DF622C3EB9EF608EC9400F608ED947E
:10639D0000F622204D09204806C23F302A0522C2B0
:1063AD003380F6E54824F640F5E5580460F075A70E
:1063BD0000758307E559C42408F582E0FEA3E0FFCC
:1063CD001207D27437126463500B30381BC2387801
:1063DD00C5864680137432126463400C203809D28E
:1063ED003878C5A646754600740D126463404A128E
:1063FD006301303D38201122204D1F20481C2040C4
:10640D0019BCFF16EB24325011D24012185CE5BFB7
:10641D0075F019A4F536D22ED22F205238E55965D4
:10642D00586032204D2F20482CD23380282011095E
:10643D00204D06204803753600303319204D1220AB
:10644D00480F12AA000559C3E558955950038558B0
:10645D0059C233C2402229FBE435CCFCC3EB9FEC7F
:10646D009E22E558B4FF012285581175A704758346
:10647D0007E54824F65002805C201259202905209A
:10648D002A02805112DB86E4F516F51775100012FD
:0C649D0064FBE510700312DB8012651434
:1064A900302910E51B2517F517F51BE51C3516F5E1
:1064B90016F51C12652112DB800510C3E511951034
:1064C90050D175A70002DB8CE55AF51124F650036B
:1064D90075110A75A7047583067510001264FB12FD
:1064E90065141265210510C3E511951050EE75A7C5
:1064F9000022E510C4F582E0E0F564E0F565E0F519
:1065090066E0F567E0F568E0F5692275A7011269AB
:106519000D124AE775A70422E9F0E51CF0E51BF026
:1065290022E510C454F0F582E0F512E5822406F55F
:1065390082E0F511E0F51CE0F51B22E512B4261501
:106549007F757E34740D12E8EA2044257511001216
:10655900E2830266727F6D7E3BE012E8CFE5137E2F
:106569003512E8CFE5127E2F12E8CF20440312E25C
:106579008312E1EF026672202852E558B4FF012226
:1065890075A704758307E559F51030330965586017
:1065990005204802051012652AE0F513305E072030
:1065A9004304E5376095E07F797E3D12E89DE51368
:1065B9007E3912E89DE5127E3512E89D30480B7F41
:1065C9007F7E3512F2000EBE40F980392012012279
:1065D90075A704758306855B1012652A305E0A204B
:0265E900430766
:1065EB00E5377003026794E512700B7E3A7F79747E
:1065FB005D12E8CF800D75F06484E5F07E397F7A0B
:10660B0012E81DE537B4020512A8988045B40302C1
:10661B008040E51C7006E51B24FB5036E511F96440
:10662B00B4602F20062CE537600D200C0AC3E995CA
:10663B0070F9500324B4F9E912F0BD781D79547D3B
:10664B001D90EBFBE53F20E00390EC0212F1C3122F
:10665B00E8FB75177975161930280375161DE512A9
:10666B00642660031266B575A7009006E3E511F08A
:10667B00A3121875E5BC75F01970040475F014A419
:10668B00951BFBE5F0951CFC9224500312602FEC3C
:10669B00F0A3EBF0C24FC263EC700EEB24E64002AA
:1066AB00D24FEB24C84002D26322E51C24ED402BD1
:1066BB00AE1CAF1B1268D77C007D32125EAFC005DB
:1066CB00EFAF17AE1612E7D6CE2405CE742C12E818
:1066DB00CF0E0ED0E02312E7D0801B1268CE1267CC
:1066EB000FCE2405CE742C12E8CFCE2402CEE87543
:1066FB00F0058412E8B5CE2404CE7422305D02740A
:0D670B008302E8CBEE243D50047EC37F4B9B
:106718007C017DF4125EAFC004C005EF6007AF17BF
:10672800AE1612E7D6D007D0067C007D32125EAFD7
:10673800A805EFAF17AE16CE240ACE02E8B5126848
:10674800CEEE2450305D03EE24A150047EC37F4B6F
:106758007C017DF4125EAFC004C005EF6007AF177F
:106768007E2F12E823D007D0067C007D32125EAF60
:10677800C005EFAF177E3712E88A7E3B742C12E80B
:106788009D7E3DD0E075F0058402E88A7F6D7E2FFE
:10679800746312E8CFE51275F06484E5F07E351273
:1067A800E76512E28302E1EF30480320740122E436
:1067B800FCF5A79006E3E0F9A3E0FE24FE40EFA372
:1067C800E0FF7D78E5376008304FE3200C2A800B26
:1067D800121861E5BD20E010304F0DD206E5712496
:1067E800FE50151268C480107D3CE546600A7D1491
:1067F8001460057D0A1470B68911125D827D6F12CE
:106808005EA2BE00A9EF24E240A4AD07E51112F094
:10681800BD202404B2D5B2D1781F795612F1C3A88D
:1068280006A907E511242D75F0B484E5F012F0BD32
:106838007407304F02740EFDFA12F1C3B2D5B2D10B
:0768480012F1C3B2D5B2D179
:10684F00DDF0AD0212F1C3850616850717B2D5B27A
:10685F00D112F1C385061E85071F7A03304F027AC6
:10686F0006E511241675F0B484E5F012F0BDA816F4
:10687F00A917AD0212F1C3DDFBE51124EA40022492
:10688F00B412F0BDA81EA91FAD0212F1C3DDFBE5C6
:10689F00377021304F1E90C159305D0390C1557F25
:1068AF003C7E3312817C121861E5BD20E00612DDBB
:1068BF00EB12EB9A22C3E99570500224B4F922E54A
:1068CF001B2402FFE4351CFE305D1ABEC305BF4D0D
:1068DF00028012AC06AB077A1B125DA47832125FEE
:1068EF0046AE04AF03227873796412611912622FD6
:1068FF00751CC3751B4B2032048B1C8A1B2212681C
:10690F00F530320122AC19AE1AA91DAF1FB900051F
:10691F00BC00028010C3E913F9EF13FFC3EC13FCA3
:10692F00EE13FE80E8BF29005006BE290050012259
:10693F00C3EF13FFC3EE13FE80EB3E7FE3E3E3E30E
:10694F00E3E3E3E3E3E37F3E0C1C3C7C7C1C1C1C79
:10695F001C1C1C1C7F7F3E7FE3E3E3070E1C38707B
:10696F00E0E3FFFF3E7FE3E3030F0E0F03E3E3E3F9
:10697F007F3E070F1F3F77E7E7FFFF070707070771
:10698F00FFFFE0E0E0FEFF030303E3E37F3E1E3F74
:10699F0073E0E0E0FEFFE3E3E3E37F3EFFFFE3E3CB
:1069AF000303070E1C38383838383E7FE3E3E37FA4
:1069BF003E7FE3E3E3E37F3E3E7FE3E3E3E37F3FBB
:1069CF00030303E77E3C000000181818FFFF181898
:1069DF0018000000000000000000FFFF0000000092
:1069EF0000003FF00000381C38F00180C1F020F0AB
:1069FF00FC0038F03FE0000000007CC6C6C6C6C6EB
:106A0F00C6C6C67C1838781818181818187E7CC691
:106A1F00C60C183060C0C6FE7CC6C6061C0606C66D
:106A2F00C67C0C1C3C6CCCFE0C0C0C0CFEC0C0C00D
:106A3F00FC0606C6C67C3C66C0C0C0FCC6C6C67C8B
:106A4F00FEC6C6060C18303030307CC6C6C67CC6B3
:106A5F00C6C6C67C7CC6C6C67E060606CC780000B7
:106A6F0018187E7E18180000000000007E7E0000BF
:106A7F00000000000000000000000000C6E2E2D2AB
:106A8F00D2CACAC6C6C20000000000000000000043
:106A9F008080A0C0A000304020C08080C0A0A00097
:106AAF000060A0600000A040A05098D090882050B7
:106ABF00A850888850A8502060806000000040E0F7
:106ACF00400000000000800000E000000000000017
:106ADF0040002040800040A0A0A04040C04040E0C7
:106AEF00C02020C0E0E0204020E02060A0E020E0B7
:106AFF00C02020C06080E0A0E0E020404040E0A047
:106B0F00E0A0E0E0A0E020C00040004000008000D6
:106B1F0080002060E0602000E000E00080C0E0C066
:106B2F0080E0E0E0E0E0000000000040A0E0A0A076
:106B3F00C0A0C0A0C040A080A040C0A0A0A0C0E046
:106B4F0080C080E0E080C080806080A0A060A0A0B6
:106B5F00E0A0A0E0404040E0202020A040A0A0C046
:106B6F00A0A080808080E0A0E0A0A0A0A0E0E0E056
:106B7F00A040A0A0A040C0A0C0808040A0A0C06046
:106B8F00C0A0C0A0A060804020C0E040404040A016
:106B9F00A0A0A060A0A0A0A040A0A0A0E0A0A0A046
:106BAF0040A0A0A0A0404040E0204080E02020A8CE
:0D6BBF0070202070A8202008F030D01000B9
:106BCC0000F0A8A8000000E00000009020487088A9
:106BDC0098984000E0E0E000A0E0E0E04060301079
:106BEC0030604040E0404060909090909060206019
:106BFC002020202070609010204080F060901020A9
:106C0C0010906010305090F01010F080E010109048
:106C1C0060609080E0909060F010202040404060D8
:106C2C0090906090906060909070109060C0E0F0D8
:106C3C00F8F0E0C0000000000000000000000000C0
:106C4C00000050605000707050000078807008F0A8
:106C5C0000F8888888F800C0C8102040981800C038
:106C6C00B098B0C000602040000000000090D8FC3C
:106C7C00D8900000246CFC6C24000020A870A82084
:106C8C0000002020F8202000000000000000800000
:106C9C000000F00000000000000000606000081020
:106CAC002040800070888888888870206020202090
:106CBC002070708808102040F8F810201008887098
:106CCC0010305090F81010F880F0080888703040A0
:106CDC0080F0888870F808102040404070888870D8
:106CEC008888707088887808106000606000606028
:106CFC000000008000008000002040F840200000D0
:106D0C0000F800F80000002010F81020007088082F
:106D1C00102000200000000000000070888888F817
:106D2C008888F08888F08888F070888080808870E7
:106D3C00E09088888890E0F88080F08080F8F88077
:106D4C0080F0808080708880B8888878888888F8FF
:106D5C008888887020202020207038101010109007
:106D6C00608890A0C0A09088808080808080F88807
:106D7C00D8A8A88888888888C8A89888887088889F
:106D8C0088888870F08888F080808070888888A8CF
:106D9C009068F08888F0A09088708880700888705F
:106DAC00F82020202020208888888888887088886F
:106DBC008888885020888888A8A8A850888850205F
:106DCC0050888888888850202020F808102040801F
:106DDC00F800CCAC9CACCC0000CCD4E4D4CC0004FB
:106DEC00781828C800FC40A040182020180000008B
:106DFC00000000F800000000A040A0500078888837
:106E0C009868708840308870200000F0A8A8A8A866
:106E1C007848484848788870888080887020A8888E
:106E2C0098A8C88888805048FC485080304C5C60DA
:106E3C0060603C00E0F0080808F88044485C484476
:106E4C0080F880808080808078484848484888B89E
:106E5C00A8A8E8A8A8B88888888888F8085000707E
:106E6C00888888708080F088888888F888888888E6
:106E7C008888F09090909090F0A8A8A8A8A8A8F85E
:106E8C00888888F808080850008888888878A8A816
:106E9C00A8A8A8F8080000000000000000000000EE
:106EAC0000000088888888E8A8E8A8A8A870A8A886
:106EBC00A80000000000000000000000000000001E
:106ECC0000000000000000000000000000000000B6
:106EDC006000606000600060006060205020000076
:106EEC0000005090B890D090886050500070705056
:106EFC00008820208870000080C0A090F8003048E6
:106F0C00B4B44830003048B4B44830FC0098D020B9
:106F1C0058C800F8E8D880D8E8F8404050F85040FD
:0F6F2C0040A0C0A000203828A0C0A01038101826
:0B00000002005E000000000000000095
:03000B0002AA70D6
:10000E00206E06859950D26E32D26F32854F82E5C0
:05001E00143200000097
:1000230010990DC298206909206DE085994FD26D12
:01003300329A
:1000340085D01285835085824FF51485158275838A
:1000440004E515242140020515E599F0D26D8512C9
:07005400D085508380C0003D
:03005B000237F376
:10AA63008530F0C5F065308530F060F722C0D0C086
:10AA7300E0C0F0C0A775A700C083C08275D0087579
:10AA83008A00300503758A7A758CEA0532E53270DF
:10AA93000215320530E530640A6026201520E531C1
:10AAA300B40C0BE530B4010612AF6912ECD3E531F7
:10AAB300B4180BE530B4060612AF6912ECD302AC3E
:10AAC3008DC2AFD2C075C07AD2AFF5300531E53152
:10AAD30064197043F53120152CC225C22C7D0A74EC
:10AAE3000412F2D1EF33EE339005CCF0EE24F540AF
:10AAF300142402400E24014008202005DDE1023722
:10AB0300F3D225D22CE5A6600215A678B5E660013E
:10AB13001678B6E6600116302E0BE5367007C22FA5
:10AB2300C22E12AE4EE5367004C24B800215367843
:10AB3300A9E660011678D8E66001160535E535709B
:10AB4300021535E590307B0B30E008D278C27BC22A
:10AB530000801A307C0B30E108D279C27CC20180BC
:10AB63000C307D0930E206D27AC27DC202E5904400
:10AB7300F8F47003753500304A09E53324FA5003BD
:10AB8300753305E5336005153302AC32E590F454B3
:0EAB930007700302AC32A2E09200A2E1920130
:10ABA100A2E2920230100320143D75330820001BED
:10ABB10020100C2011098013E59030E10E8006E58C
:10ABC1003724FC40F3E543541FF53320100375A6E9
:10ABD100FF202E5D301004E536705620100C201138
:10ABE10009E53524F55003753304D21BD2A5D2A64D
:10ABF10012AE4E75B44075B24078D8E67002053495
:10AC010020272E20682B202928202A25A210721106
:10AC1100501FE52054076019E53424375004C24A17
:10AC2100800F2401400B200026200119D27D7534AC
:10AC3100C8201558E531702412F2B174E812F28A75
:10AC4100802A02AD91E53724FC40E6D27C80DF30DA
:10AC510011DFE53724FC40D9D27B80D275F0038423
:10AC6100E5F070DE12D88874E812F28AE531B40694
:10AC71000512D9F38016B40C0512DA06800EB4124F
:10AC81000512D9F38006B4180312DA0620141B80CA
:10AC91001990ACB5E532C4540F93FAE532540F6004
:10ACA100096A70061216ED12171CE59030E1153095
:10ACB100E2128016010204040404050506070708D0
:10ACC10009090A0020100820110520103C807D2070
:10ACD10027F82068F52029F2202AEFE534243040B6
:10ACE100E9240750E5600B205E088590F020F20210
:10ACF100740190AD0393D2A5201002C2A512AE3902
:10AD0100806FC8A08269554646202F12E536603C07
:09AD110024AA500AE53675F01978
:10AD1A0084E5F06040D2A6201002C2A6D2A5202F58
:10AD2A000C7418304B02746412AE39803BE53675E8
:10AD3A00F00C30480375F00684A2E0744640E974CA
:10AD4A003780E5E52B5403600C20100E301106E520
:10AD5A004A6402600512AE54800312ADA9101B08A2
:10AD6A00A25892A5A25992A675A700D082D083D0E4
:10AD7A00A7D0F0D0E0D0D020200C201009C5A670B2
:10AD8A00030237F3C5A632C218B40202D21812D986
:10AD9A002630180874E412F28A02AC6D02AC6878A4
:10ADAA00A7E5B4600924E04005760002AE54E53414
:10ADBA00702920412220751F300D1CE57924CE40D0
:10ADCA00167AFFE5B110E7010A2325B3F5B3EA3590
:10ADDA00B4F5B4C313F5B2E660021622C241207577
:10ADEA00028077C246E579FF605820120424FD509C
:10ADFA0051206502C21CD265EF24B050027F4FEF8A
:10AE0A0090AF199375C70375C6FC75B90185BFF074
:10AE1A00A4E5F0F624F44002760C301C2DE5BEC3FE
:10AE2A009FF5F0A4E5F024E0400375F020E5F0C2B8
:10AE3A001C79AA770375B300F5B4C31375B100F58D
:0CAE4A00B222C26578A77680D24179AAB6
:10AE56007703D21CE4F5B3F5B4F5B1F5B222C265B9
:10AE660079A1E57924CE500DE720E7E27628301C5B
:10AE7600DD743C80BE7680E720E7D3E57997404DC8
:10AE8600C24679AAE7FAE5792323B4C500400274DD
:10AE9600C42437300E31F42437300D15F7BA0302C7
:10AEA600FA0AC39AF5B175B300EAF5B4C313F5B25D
:10AEB60022101C07D21C76C802AE3B763274FF20E5
:10AEC6000E02749B02AE3BC313247E80CC75C7036F
:10AED60075C6FB75B901E5BD6026C395795004C2F8
:10AEE60046801D78A720461B301C11E57975F008B1
:10AEF600A42432F6E5792324AA02AE397605D24691
:10AF060002AE54301C077614747802AE397696C2B7
:10AF16004680EDFFF3E8DDD3C9C0B8B0A9A29A9484
:10AF26008F8A85817D7975716E6B6865625F5C5904
:10AF36005653504E4C4A48464442403E3C3A3836B8
:10AF460034333231302F2E2D2C2B2A292827262533
:10AF560025242423232222212120201F1F1E1E1DDB
:10AF66001D1C1CD2B5C28EAE8DAA8DAF8BAB8BE4E9
:10AF7600F58DF58BD28E3014012278B6BE0007EF20
:10AF860024E24002800806E624EC5002761420678C
:10AF960005E624F64005E4FEFAFFFB7C007D0A1276
:10AFA6005D827C007D5E125EA28F51EE600375515C
:0FAFB600FFEAFC7A33125D96EBF5F0A4E5F0CBE1
:10AFC5008CF0A425E0C5F035E0CB92D525F05006F0
:10AFD5000BBB0002D2D530E7060BBB0002D2D5EC85
:10AFE500F5F0A42BFBE5F03400FC30D5010C78A678
:10AFF500E6C39BFF18E608F6EB18F618E69CFE1864
:10B00500E608F6EC18F6301401227A0050040A120C
:10B01500601F7C007D6E125EA28FF078A2E6A4FB15
:10B02500ACF0125FBEEBBA0002F404FAE4F8FFEAF2
:10B0350030E70118E57960062075031FF4042AF549
:10B0450079EF38D27520E70860037579FF02DB2FA9
:10B05500C2750470F5E579F40460EFF57980EE12B8
:10B06500185778BBA6BC121875E5BE78A2F624F66B
:10B075005007E4F5BEF61255F7120BF6E5BEF54896
:10B0850024F65008E4F5BEF5481255F7E5BFF5433B
:10B0950024F3503924F3403512186B78A1A6BCE58A
:10B0A500BF789DF61424FB50087403F6F5BF1255BE
:10B0B500F778B7A6BE121861E5BDA2E39266A2E4D1
:03B0C5009267038C
:10B0C8005403C253B40102D25322740DF5BFF543A1
:10B0D8001255F780C0E56A700CE56B5403700612D0
:10B0E80098BD12B14775F08412B17F787086F70861
:10B0F800B880FAD2B275F08812B16D782575F00073
:10B10800758002C2B275F7D7E4F5F70000E5F7D20B
:10B11800B220E705D5F0E9D8E72275F08412B17FAF
:10B128008DF7A4D2B280CE75F08412B17F75F0008D
:10B1380075F7FFD5F0FAD2B222756BEC756A007517
:10B148008002C2B275F78475F70075F70075F700CD
:10B15800780075F7FF75F7FF75F7FF75F7FFD8F2F9
:10B16800D2B275F08112B17FD2B2808F75F05312CE
:10B17800B16D808775F003758002C2B285F0F785DE
:10B188006CF7856BF7856AF72275F003758002C244
:10B19800B285F0F7856FF7856EF7856DF722125443
:10B1A8004775382490B1FE12320B12EFA802F12E27
:10B1B8001254477D0E90B21512B1C87D1890B22373
:10B1C80074A012EF9474A212EF94E4FEFF12EF94AD
:10B1D800ED12EF94E493A312EF942FFFE43EFEDD0B
:10B1E800F3EE12EF94EF12EF9474B012EF9474B37D
:10B1F80012EF9402F13424505352463130302C303F
:10B208002C35373630302C382C312C300088000063
:10B21800040000000000000000000081020101009D
:10B22800010101000101010001000100000001000D
:10B2380000E10075160375170312B27B204C01223A
:10B24800D517F6D2A47F8CDFFEC2A412F12612B164
:0FB25800A612B1B812F126D516DC12F2E57F323C
:10B267007E0690BF3F12814912283F12F16E3000CF
:10B27700FD0237F3E4F5A79004DFF0D582FCF01266
:10B287005447D269D2ACE4F515F87903106DF7D8B5
:10B29700FBD9F9E4F515F8F97A05E515700FD8FA31
:10B2A700D9F8DAF6C2ACC269D24CD23D227800791D
:10B2B70007106DF9D8FBD9F99005FF7453F0753273
:10B2C70010C2ACC269C24CC23D7A0312B613103B1E
:10B2D700D388017A0312B629103BC9E89940C57A89
:10B2E7000112B6AE70BE7A0212B6AE70B77A03120A
:10B2F700B6AE70B07A0112B6137A4712B601303B78
:10B3070004D23D800B7A0512B63C12B68AB43024BB
:10B31700E49005DDF09005E5F09005D779BCF0F5F0
:10B327005DF7A309F0F55CF79005F27427F0A374B5
:10B337000FF08059D25712B64E9005DDF09005E513
:10B34700F012B64E75F00AA4FA20D1010812B67AA7
:10B357002A75F00AA4C5F09005F2F0A3E5F0F0E431
:10B36700FCFBFEC21712B68AB42D05D21712B68D92
:10B37700B42E02800512B5F2DEF330170312602FE8
:10B387009005D8EBF0F55C1582ECF0F55D7A0212CA
:02B39700B613EB
:10B399007A5312B601303B04D23D80647A0212B668
:10B3A9003C12B67A147006FA532EE080139005DE2B
:10B3B9007402F0D274C2737A05146004D2737A07E6
:10B3C9009005CEEAF09005DDE05407C52E54F82526
:10B3D9002EF52E7E0C7DE612B63AC2D512B65175FF
:10B3E90083058D82F00D30D504DEEF8002DEE8AEF4
:10B3F9005DAF5C207303E4FEFF79BCA70609A707CC
:10B409007A0312B6137A4D12B601303B05D23D02CA
:10B41900B52B12B64EF53D12B651F53E12B651C5D1
:10B429003F0475F03C84E5F0653F60069005FF74C4
:10B4390044F012B68AB4562D7A0612B63CC22DE4EF
:10B44900F571F5707E049005D9F0A3DEFC20571341
:10B45900F57D7E067973F709DEFC7E089005CFF04D
:10B46900A3DEFC8074B441A512B63AC23C7FCF1268
:10B47900B564C4F57D12B68AB43102D23C7FD312C9
:10B48900B564257DF57D12B63A12B5DE7AB9125D3D
:10B49900A4C0007864125F46D0009005D9ECF0A3EF
:10B4A900EBF0125FBE8B71EC60037571FF12B63A57
:10B4B90012B5DE9005DBECFEF0A3EBFFF07C007D1E
:04B4C90014125EAF4C
:10B4CD00C22DED24F150010F240A5002D22DBFB42C
:10B4DD00027F008F70C23C12B64EF53C24E0500244
:10B4ED00D23C12B651F53B24F35002D23C12B65168
:10B4FD00F53AE53D24E85002D23CE53E24C4500225
:10B50D00D23CE53F24C45002D23C303C02800F7542
:10B51D00A7049005DF793A7E06E7F009DEFB203DB2
:10B52D000320740C532EE0E49005CEF09005DEF070
:10B53D0075A7049005F4E561F0E560F0E55EF0E5D2
:10B54D007AF0E579F0E52EF0E55FF0E57BF0E55179
:10B55D00F075A700029C8A12B651303C0224647526
:10B56D00F03CA4ACF0FB12B6512BFBE43CFC7A642E
:10B57D00125DA40812B6512BFBE43CFCE43DFD1218
:10B58D00B67AF912B68AC21724AF5005D2171260D7
:10B59D0037BFCF358D758C748B73301703126037B1
:10B5AD007A0A125DB6EB29FBE43CFCE43DFD7E001E
:10B5BD003017041260371E7583058F82EEF0A3EDF0
:10B5CD00F0A3ECF0A3EBF0E9228D788C778B7680ED
:02B5DD00C9E4BF
:10B5DF00FCFBFE12B68DB42E02800512B5F2DEF31F
:10B5EF0012B68DCD7A0A125D96CD540F2BFBE43C2B
:10B5FF00FC22C23B080808758304888208E06A6051
:10B60F0002D23B22C23B7583047800888208B8E0DF
:10B61F000280EEE0B424F4DAF2227800888208B8CF
:10B62F00E00280DDE0B42AF4DAF2227A01758304B5
:10B63F00888208B8E60280C9E0B42CF1DAEF221252
:10B64F00B63A758304888208E0B42C04D2D5E4227C
:10B65F00540FFA08A3E0B42E04EAD2D122540FCA31
:10B66F0075F00AA42AC2D12212B63A7583048882D1
:10B67F0008E0B42E0308A3E0540F2212B63A7583E4
:10B68F0004888208E02212B69FC4FA12B69F2A22BB
:10B69F00888208E020E603540F225407240922125F
:10B6AF00B6137AE6753800888208E0B42A0612B617
:10B6BF00956538226238DAEF74462212547375A7F3
:10B6CF00009004007EE07D03E0A312EF94B40A041F
:09B6DF00DD028002DEF202F13806
:10005E00D2B47581C075AF017590F878FFE4F6D80B
:10006E00FDF4F5A6D220D2C075C07A75F83075D7DA
:10007E005075AE1375AF017581D87590F875EFBCDC
:10008E0075FDFFC2B7D2A412F12AC2A47450123861
:10009E0016758951D28C75A882D2BC12997B12F238
:1000AE00B112D7FE12B064C22012ED861236C57F91
:1000BE00407E0190B6F112814912549112F12A122A
:1000CE00EED912F16E12F1647C1412F13430000389
:1000DE000237E3DCF512B1A612B1B812F12A75A6F9
:1000EE00FF12B23B12B0641236C512F16E12F12637
:1000FE0012F16478B5761E12ED8612D7F3C215C2D0
:10010E00141236C590B7397F78128137205E0A7F78
:10011E00767E1290B74612E8FB7F4012F2607F495E
:10012E007E0912E138E53F20E00805A6E5A670023B
:10013E0015A67F5312DD5E7F577E0B12E69212E7F5
:10014E001A7F602073102074097E2BE52E5407123F
:10015E00E8BC7E17800E7E0BAC5DAB5C12E6961291
:10016E00E71A7E311281D37F697E1212EC2130257F
:10017E00087E1290EF4212E8FBE5A60303543FFD02
:10018E00FE0D7F7312F2000F12F2001EDDF478B531
:10019E00E57124F64002761E307419E6602B7F72EC
:1001AE007E16744012E89D7E17E612E8237E1F74B9
:0701BE005312E89D12F16EDF
:1001C50010000C10010C10020C12B23B02010502CA
:1001D50037E3023A3E8061E53524C85046E5902074
:1001E500E241D0E0D0E0120229027D9DE53524D21E
:1001F5005031E59020E22CD0E0D0E08038E5352480
:10020500D25020E59020E21BD0E0D0E012F2E5309C
:100215006B0B7F0912812E12562F128606120229A8
:100225000205702212F2E590BFF57F0012813712A8
:10023500F16E02F12312F153C215C214C227C2682E
:1002450012F16475370190B829122725900255736C
:100255000200EF0221F0020A08022AD2020570020A
:1002650005AD027D9D02027002052212F16475370B
:100275000790BBB81227259002807302023D020841
:100285001D02085702088B0202A102041102027026
:100295000202700202BF0202A60256FF12B23B80A2
:1002A5002A7F517E00747212E8CB12289C40BC1242
:1002B500554312ED8612B06480B17F49A25E120BE0
:1002C500E1925E120C0080A31255F712F1647537A6
:1002D5000290BD7A1227259002E07302027002187F
:1002E500A202190702195B0219B00219F4021A03D6
:1002F500020341020377021DC70203017F5B121847
:100305009812187AA8BE12032512F16E1000081073
:10031500010710020780EF18180880EA88BE80A838
:100325005300037F5A7E0590BDCCE875F00BA425DC
:0E03350082F582E5F03583F5830281497F4031
:1003430012189812187AE5BCF8E87F3F7E3212E75C
:10035300DC12F16E10000810010D10021280EA1871
:10036300B84AE6787D80E208B87EDE784B80DA888A
:10037300BC0202CD12F2E57F0F90C1E81281371261
:10038300283F12F16EC214C21512F12375106510C5
:1003930000DFE53170F9E5106465700D855E148545
:1003A3007A15E4F512F513800C78A8E51326F513F6
:1003B300E43512F5127F1E7E19E51012E782C3E5BC
:1003C3007A9515F517E55E9514F5167F287E0BAC27
:1003D30016AB1712E69612E71A12F16E12F134D524
:1003E30010ADAB17E516FC30E70312602F7A0A79DC
:1003F30000125E0FA912A813125F48EBF510243800
:1004030040037510C81218578510BC0202CD12F2B2
:10041300E590B7847F017E0912814990B78C7F0AEA
:100423007E091281497F1312DD5675170012186673
:10043300E5BC1204F1E5BD1204F1E5BE1204F1E5D9
:10044300BF1204F190B7DC7F5F7E06128149122848
:10045300DE12F16E7517001204D110000810011599
:1004630010024880F20517E51724F75003751700AB
:1004730075100080E2E5176408701512186675BCE4
:100483000175BD2375BE4575BF671255F70204118B
:10049300E51012050312F16E1204B1051053100793
:0604A300E51724FE4003F2
:1004A90053100380AC020270A9BCAABDABBEACBF9D
:1004B900E5171304F8E640085407C42510C480045E
:1004C90054702510F60287EE7800E875F009A42427
:1004D90017FF7E3B7D20E8651770027D89ED12E8E4
:1004E900CF08B809E502F16EF8C41204F7E812055D
:1004F900037E030517E51702E8BC540775F009A444
:1005090090B7942582F58250020583E51775F009A5
:10051900A42417FF7E0C02814912F16475370890F3
:10052900BE72122725900532730200EC02054E02B5
:10053900142F0212E2020D0F02568D0205477F3772
:100549001220CD80D47F0A121898120BF61220724D
:1005590012F16E10000810010510020680EFB25A60
:1005690080EB120C0080B2C26812F16475370590F5
:10057900B9641227259005827302023D028387021E
:1005890083CC0285650205700205A60284A702854F
:100599000D0221B902057002219F020B127F2E1252
:1005A90020CD80C312F16475370690BA3F12272512
:1005B9009005BD7302023D0221F60222580222D1A2
:1005C90002239E0223D00224470206020205FB02EF
:1005D90024900225350205E17F64121861E5BDA268
:1005E900E7120BE1121861E5BD92E7F5BD1255F767
:1005F90080B27F491220CD80AB1207BE12383D125E
:05060900F2E5122819C2
:10060E00E55804607790BB0E1206AB129FD512F11F
:10061E006E10000810011310021C80F50559C3E579
:10062E0058955950D575590080D01559E55930E770
:10063E00C985585980C4E559B40F02802FB51F02E1
:10064E00802A75F007A42408F51775162774B825A7
:10065E0059F9870012069912F16E10002810012820
:10066E0010020280F574B82559F9A700E53524FA71
:10067E00508878C7A6481207B512F2E512F16E122D
:10068E00F1260205AD1880CC0880C9E875F005A4E6
:10069E0085F01CF51BC0001266B5D0002212A066B4
:1006AE00B4FF0122751000751FFF12A07DE51064C6
:1006BE000F60171206E2401274B82510F8E675F0B6
:1006CE0005A485F01CF51B1267460510C3E5589569
:1006DE001050D722121BABF8602E6404602AE81467
:1006EE00B51025F51F121875E5BC70060475F014CB
:1006FE00800375F019A485F01CF51B1267467E2247
:10070E0090C18912817CD322C322E558B4FF012205
:10071E00751000E510640F602EE51075F007A42427
:10072E0009FF74B82510F8E612079F75F00A84C009
:10073E00F07E2012E8237E28742C12E89DD0E07EF5
:01074E002A80
:10074F0012E88A12075F0510C3E558951050C322AF
:10075F00121BABF8603964046035E8146510702F14
:10076F00121875E5BC12079FF8C313923D7E1C1239
:10077F00E8397E28742C12E89DE4303D067405B8E4
:10078F000001147E2A12E88A7E18742312E89D2233
:10079F00305D1275F036A42432FBE435F0FC125FA5
:1007AF00BE125FBEEB221207C712811CDFFB2212A3
:1007BF0007C71288FEDFFB2275C70375C6F078B82E
:1007CF007F042275C70375C6F375B901E5BFB54838
:1007DF0031E55924F1402BE55975F00484A9F02433
:1007EF00F0F5C675B901C5F0A9BC600CA9BD1460C0
:1007FF0007A9BE146002A9BFE975F005A4F985F039
:10080F00CC22121875A9BD75CC00221255F712F122
:10081F006475370390BC1812272590082D730202B8
:10082F0070020B2B021D1C020B40020B4B022117F7
:10083F00021DE0020C0C021E14021E5A0221660257
:10084F001D96021E9F1255F712F16475370490BC66
:10085F00D512272590086773020270020B5A020BFC
:10086F0065020857020B7B020B86021A1D020857FE
:10087F00020B95020B70020BAF1255F712F1647554
:10088F00370B90BD2412272590089B73020270022C
:0B089F001ACB021ACB02092102095FEC
:1008AA000208C20208E50221FC021B70021C3B027C
:1008BA001BE4021CCC020BC9121861E5BF1470C1FB
:1008CA007F2E1218981F121861E5BDA2E6120BE1DD
:1008DA00121861E5BD92E6F5BD80A37F371218981C
:1008EA0012185CA8BFE812091912F16E100008105C
:1008FA00010D10021280EE18B802EA780A80E608A2
:10090A00B80BE2780380DE12185C88BF0208887F81
:10091A00367E2CE802E76B7F1C121898121861A821
:10092A00BE12095312F16E10000810010D100214C4
:10093A0080EF18B800EB780B80E708E824F450E160
:10094A00780180DD88BE0208887F1B7E35E875F055
:10095A0005A402E7657F25121898121861A8BF122C
:10096A00099112F16E10000810010D10021480EFA7
:10097A0018B800EB780980E708E824F650E1780116
:10098A0080DD88BF0208887F247E3BE802E8BC122B
:10099A001857E5BF75F03CA4ACF0FDE5BE75F0054F
:1009AA00A42DFDE5F03CFC121861E5BF1460367514
:1009BA00F005A485BEF0A42DFFE5F03CFE7C007D89
:1009CA003C125EAFC005EF75F01884E5F07F2D7E0E
:1009DA002412E7657E30743A12E8CF7E35D0E012F1
:0709EA00E76502F16E7F2DAD
:1009F1007E0590C1AB128149121861E5BDA2E67F67
:100A01002D12206402F16E12F2E5122819120A1455
:100A110002023D7F177E0290B8871281497F4C7E8A
:100A21000290B89E128149AC5DAB5C7F577E041287
:100A3100E71212188485BC6285BD63E56124F84024
:100A41004490B8A97F37128137AE61AF607C017DD8
:100A51005E125EAFC3741F9FFAAC63AB62EC33925C
:100A610017500312602F125D96AB047C0030170300
:100A710012602F74F52BFB74033CFC125D6C7F3705
:100A81007E1512E68A90B8B67F697E0F128149E51C
:100A910060240FFBE43561FCA25C923BD25C7E1EBC
:100AA10012E696A23B925C7E30742012E8CF7E362D
:100AB100742012E8CFE5602562FBE5613563FC7FB8
:100AC100227E0412E712E56245637016742E7E3AA7
:100AD10012E8CF12F16E10000D100115100226025E
:100AE1000A3C742080E81562E562B4FF0C1563804E
:100AF100080562E56270020563E53524F55003756A
:100B01003301020A3C1218848562BC8563BD02551B
:100B1100F77F637E00747212E8CB12289C40087F35
:100B21006312812E1255FE02057012186BE5BCA2EC
:100B3100E77F0A120BE4E5BC92E7F5BC02081A7FD5
:030B41001CA20DE6
:100B4400120BE1920D80097F25A20E120BE1920E89
:100B5400120C0002081D7F0AA20F120BE1920F80F3
:100B64002A7F13A208120BE19208801F7F52A20C65
:100B7400120BE1920C80147F25A20B120BE1920B55
:100B840080097F2DA209120BE19209120C000208C0
:100B9400577F49121861E5BDA2E3120BE1121861F7
:100BA400E5BD92E39266F5BD0208547F5B121861BD
:100BB400E5BDA2E5120BE1121861E5BD92E5924391
:100BC400F5BD0208547F6D121861E5BDA2E0120B59
:100BD400E1121861E5BD92E0F5BD020888120BF63A
:100BE4008F1F9217121898AF1F1F7E39128E4BA2B7
:100BF400172212187085BC2B85BD2122121870850E
:100C04002BBC8521BD0255F712186B85BE12120C40
:100C14002112186B8512BE1255F702081D75A6FF26
:100C240012F2E512AA63740712F2D18FF07406125D
:100C3400F2D1EF2512C395F0A2E7923D4010FD24B6
:100C4400CD50027D32AC05C3743F9DFD800FF4048A
:100C5400FD24C850027D37AC0574402DFD7F401241
:100C6400DD567E1212F2000EBE1EF91F303D020F39
:100C74000FEF6D70EDE536700A753606EC2513F549
:0C0C8400148C13120C9F12F16E1000076C
:100C90001001083002072215128002051280827F9F
:100CA000377E28742E12E8CF7F347E21740A303DBF
:100CB000010412E8EAE514FC249C50027C637F34B2
:100CC0007E2DEC12E1DD7F437E1E12E6927E00E572
:100CD0001212E8297F057E0290BCA91281497F6D1E
:100CE0007E0190BCB412817C7F747E0490BCC612DD
:100CF000817C02281990B8C07F1B7E101281491296
:100D0000F16E12F123C214C21512F153020522D260
:100D100014D215E4F56EF56D756F02751501751435
:100D200001754280D233120D8EE51565146005857C
:100D3000151480F0C24D12F2E512847D90BE42126D
:100D4000817A129B0478B8E60460AA751000D24E2E
:100D50001211E9304D07C24D12F12AC202C23310FE
:100D6000000810012910024880F3E5151460C7D26D
:100D7000D5129A05E56F24FE400430339222129B6F
:100D80000478B8E630E6EA30D5221515801E1299AF
:100D9000E5E56F24F25005129A058010129B047845
:100DA000B8E630E6E9C2D50460C7051530338722BE
:100DB000E53514601324BE5003020D052419509D1F
:100DC00012284D12F16E8095E4F511F512122819D2
:100DD000E511451070087F7B90BA2912817A12E0E4
:070DE000FA1211C385111284
:100DE70012F16EE51110001310013410020280F3A6
:100DF700E53524E65056D24D020D366004151180B4
:100E070015E5107003020EDD151012F2E51211E759
:100E17007407F511F5127F42129C5DDFFB80A72452
:100E2700F940157479951775F00D8414D395114011
:100E3700B20511129C26808E203CA8303DA50510D6
:100E470012F2E51211E7129C26020DC8783A797161
:100E570012DB77854E63854D62120FBD756C7F750A
:100E67006BE8756AA512F2E51228F012E0FA121182
:100E7700361215EA12168A1216CA12F16E100008F7
:100E870010011810023780F5120F99E56B241840EE
:100E970005120FAC801C129C5D8017120FACE56B1E
:100EA7002414500BE56A24135005120F998003127E
:100EB7009C2EE53524F550AD75330180A8787179FE
:100EC7003A12DB7785634E85624D754C0012F2E569
:100ED7001211E7020DCD12290C12F16E1000051048
:100EE700010580F8020DCDC25312547312284D74B8
:100EF7004012EFD8747812EF88746312EF88746722
:100F070012EF88742312EF7B1231A6E51512EF67F3
:100F170078B8E6C4540344400412EF8812EFAFE4F4
:100F2700F51412994D129A53747012EFD8E51412F2
:100F3700EF6775A700900401E012EF7BA3E012EFC3
:080F47007BA3E012EF7BA3E0A5
:100F4F0012EF7BA3E012EF7BA3E012EF7B12EFAF68
:100F5F007F7B7E1DE51412E83912F16E10022875A1
:100F6F00A70090042275134275120F753800E01216
:100F7F00EF67A3D512F812EFAFD513EC0514303C81
:100F8F009C12303F12F134020DCD74F1256AF56ACF
:100F9F00E56B34FFF56BE56C34FFF56C22740F25B0
:100FAF006AF56AE4356BF56BE4356CF56C22756C9C
:100FBF007F756BE812B144E5104511C2306002D263
:100FCF0030303B028060303011E51112994D129A8A
:100FDF0048129A9890055B121123E51112994D1240
:100FEF009A86900411756AA512111C056B7FEF127A
:100FFF001125129A98900411056B756A9412111CA1
:10100F00056B7F6C12112512B1417F8312112512CE
:10101F009A7B129A86900400E020E60990041175DD
:10102F006A8312112322303011E51112994D129A51
:10103F0048129A981210D5121120E51112994D12DB
:10104F009A861210D5756AA5121120129A9812104D
:10105F00D5056B756A4A121120129A7B129A8690E7
:10106F000400E020E65D1210D5756AEF1211201210
:10107F009A981210D5056B756A94121120129A7BEB
:10108F00129A86900400E020E6391210D5056B7590
:10109F006A39121120129A981210D5756ADE7F22C2
:1010AF0090061012112512B1417F83121125129A49
:0B10BF007B129A86900400E020E608F7
:1010CA001210D5756A83804E02B14175A701900648
:1010DA001005A7900411AE838E16AF828F17E0F524
:1010EA00451212D5F5441212D5F5537C007D2D1206
:1010FA005EAFED6414600685168385178212176F3A
:10110A001260A905A7EDF0A305A7A3E58324FA5069
:10111A00C5227F0080059006107FA575F08412B164
:10112A007FE0F5F7A3DFFAD2B202B0FDC06FC06E5E
:10113A00C06D756F7F756EE8756D0012B191751788
:10114A00237E00D2D57B0579FF7A007C1520D50154
:10115A001CE4F5F7E4ADF71212B620320CB5010023
:10116A005001F9B502004001FADCE6C3EA9904FA33
:10117A00E904F5F0EA141445F07003E4F9FAAF0152
:10118A00EA600612F2000FDAFADB0B10D506D2D5A6
:10119A007B0580027B030EBE40ADD2B27E087F245F
:1011AA0012F2007F2812F2007E3712F2007F241218
:1011BA00F200D06DD06ED06F22E51275F00DA4FF4B
:1011CA0074739FFF7E00742012E89DE51175F00D7F
:1011DA00A4FF74739FFF7E00743F02E89DC24EE431
:0F11EA0012994D12E0FA751779121206203C0C7B
:1011F900203D09304EF4E53524FA50EE22751201EE
:10120900129A53C23D75A700900400E0F5F0A2E5DB
:10121900923BB4FF03D23C22E5176479600320F6C0
:10122900F490042275160475130FE5165401441041
:10123900F514E0FD303B2AF545C083C0821212D572
:10124900F5441212D5F55312176FAC06AB0712DF2E
:1012590030FDD082D083D5130875130F741E121276
:10126900D7AE161212B620320312F200A3303B2277
:10127900E58324F8501C0512E51224FC401F129A3C
:1012890053900400E030E604D23C801190042275AA
:10129900130FD5149D0516E51624C0508D12F16E55
:1012A900E51724F3F51724EE4002D23D22C232EDB0
:1012B90004601624FC501224A350027D5FEDC42360
:1012C900541FFFC3E5179FFF22D23222740F2582D4
:1012D900F582E43583F583E022D22B12141FD21450
:1012E90012ED8612F2E51228F912E12D12151112EA
:1012F90013F5751604751500E530651360FA853028
:1013090013533203E53270F01216ED12173C05152E
:10131900E51524C45006751500129C3D301A0312B8
:10132900179DE539600912139112136312F16E7555
:0B133900A6FF10000810011810020AA7
:1013440080BB301AB81214E38009201AB012B23BE1
:101354001214B6808E1214E3C237C22B020522E5A2
:101364001570030215377F0A147001221470077E6A
:1013740024E53E02E7651470097E1378AEE602E7C1
:101384006522146001227E35E53F02E765ED24E124
:10139400400574769D801A24E2400EED941E337548
:1013A400F00384FC74589C800804C313FCC3744485
:1013B4009CFCAE167F7612F200EFB5040B1FEF24EF
:1013C400ED500812F23080F51F80EBE516FE20E0A8
:1013D400147F2612F2007F3512F2007F4412F200CD
:1013E4007F5812F2000516E51624C0500375160442
:1013F400227F24740812E8887F33740612E8887FF9
:1014040042740412E8887F56740212E8887F657477
:101414000112E8887F74740002E888D215C21AC2E7
:101424001F12B23B1214BDE4029121C22BC214124A
:10143400141F75A6FF758AFC758CFFE4F532F53927
:10144400D205D23712ED8612F2E5129C3D12E12D3F
:101454001215111215841228F979197B1E123B17E3
:1014640079557B1E123B1779917B1E123B1779CD60
:0E1474007B13123B1710002210012F100221D3
:10148200301A11E53924F14008E532240340058081
:10149200EF12179DE532240250FA80981214E3806D
:1014A200DF201ADC12B23B1214B680D41214E3C24B
:1014B20037020522201A57D21AD21F12185C85BC95
:1014C2004C85BD4D85BE4EE54C700FE54D54037005
:1014D20009753910E4F5520291217401129A26809D
:1014E200E6301A2AC21AC21F12185C854CBC854DFE
:1014F200BD854EBE1255F7E4129121D214E54C700F
:1015020008E54D540370028003121801C214227FB1
:101512000A7E007401205A02740312E8B57E057433
:1015220058201A02742D12E8CF7E0B7446202B022B
:10153200742012E8CFC3E4954DFB740E954EFC4B1C
:10154200F5177A46205A027A17125DA48C038D048D
:10155200302B0CC3EC13CB13CBC313FCEB13FB12DA
:101562005FBEC0E07F017E00EB12E7D67E0AD0E0CC
:1015720012E8B5E517700A7F2F7E1090BA0012812B
:1015820049227F197E0590BE5F1281491215EA75C4
:10159200A7008552827583057E3F7C00E0B504007A
:1015A2004001FC1582E582B4FF037582B3DEEDECE7
:0E15B200230475F0038423FD249C50027D6306
:1015C000ED75F00A84C0F07F237E2512E8EA0F0F44
:1015D0007E2D742E12E8CF1F1F7E32D0E012E8EA73
:1015E0007F267E0590BE6A02817C7D057F3A12DDF2
:1015F00068EF240FFFDDF778087F387E01E812E8F6
:101600008AEF240FFF1818B8FEF17F3D02DDC77581
:10161000A700F5827583057E3FE92B203D012B95C0
:10162000324031E0FAC374769AFF1582E582B4FF46
:10163000037582B3E0FAC374769AFD1216551582CB
:10164000E582B4FF037582B3E0FAC374769AFD12A3
:101650001655DEC522BE3F0122203D1712F200C3FF
:10166000ED9F70012240060F12F20080E81F12F277
:101670000080E212F230C3ED9F70012240060F128B
:10168000F23080EF1F12F23080E912B17C1216A402
:10169000FD7E001216A4FFFC1216B38C050EBE4090
:1016A000F2D2B222E4F5F7E4E5F704C313FAC37407
:1016B000769A2212F200C3ED9F70012240060F12AB
:0D16C000F20080EF1F12F20080E9C3E56B1D
:1016CD0094E8FCAB6A7A08125D967D0078A5125FEE
:1016DD003FAE037F259016E802E8FB03052070F866
:1016ED0030B226758001C2B275F72475F700E4E5B6
:1016FD00F7F545F5F775F700E4E5F7F544F5F775FA
:10170D00F700E4E5F7F553D2B212176F0260A97531
:10171D00A700758305855282EDC313F00552E5527E
:10172D00244C5003755200E532B401037539007530
:10173D00A7007583048539820539E53924F05004F5
:10174D0075391022EDF0E5822410F582E545F0E5BE
:10175D00822410F582E544F0E5822410F582E553EC
:10176D00F022E54530E702F404F5F0A4AEF0FFE514
:10177D004430E702F404F5F0A42FFFEE35F0FEE55A
:10178D005330E702F404F5F0A42FFFEE35F0FE22FE
:10179D00E53924F0407904600122E54E24F2406FD2
:1017AD00240C506BE54C704CE54D54037046740899
:1017BD0030100104302B024410205A024420301FF7
:1017CD0004C21F444075A7009005CEF0A3783A7F60
:1017DD000612DB927F07301010786A7F0312DB92BE
:0F17ED0078707F1012DB927F1A9005CE1218428F
:1017FC007422129A2675A700900400205A0F758245
:10180C0010121820758220121820758230121820A0
:10181C0075390022E54C240E40047D0F800F04FD29
:10182C0074109DFCAF04121842EC129A26AF0512EC
:10183C001842ED029A2674061299867402129A10B6
:10184C00E0F5F7A3DFFAD2B2029B3775C6F4803508
:10185C0075C6F5803075C6F6802B75C6F780267573
:10186C00C6F8802175C6F9801C75C6FA801775C636
:10187C00FB801275C6FC800D75C6FE800875C6FF10
:10188C00800375C6FD75C70375B9012274721F12EA
:10189C00E8CB0F02F16E7F0A1218987E2A12B23B27
:1018AC00121875A8BF1218D61000121001051002DC
:1018BC001580F508E824E750EC781880E818E83033
:1018CC00E7E3780080DF88BF805F7F097E0590C0EA
:1018DC006CB80C0390C0661281497E27E53D282424
:1018EC000C75F01884E5F012E7657E33743B12E852
:1018FC00CF7E35E53E12E76502F16E7F1312189824
:10190C00120BF6121938100008100105100217807E
:10191C00F2105C07205D0BD25C80E8105DE5D25DB7
:10192C0080E1D25C80DD852BBC0202CD205C1020D6
:10193C005D1890C0BF7F127E2312814902F16E9018
:10194C00C0D3205DF090C0C680EB90C0CC80E67F09
:01195C001C6E
:10195D00121898121870A8BF1219921000081001D1
:10196D001110021A80F2E824F250031880EA780D63
:10197D0080E6E824E740030880DE781980DAE8F590
:10198D00BFF54380A37F1B7E26E412E8BCE823232A
:10199D00B464087E26740112E8BCE47E2E12E7655D
:1019AD0002F16E7F2512189812187FA8BCE8121943
:1019BD00EB12F16E10000810010D10021F80EEE801
:1019CD0024E050E9188006E824CF40E10812187F82
:1019DD0088BC1255F7D21512ED8680D180157F2463
:1019ED007E3724E202E7D67F2EA20A120BE1920A7D
:1019FD00120C000202D07F37121861E5BDA2E4126D
:101A0D000BE1121861E5BD92E49267F5BD0202CDBE
:101A1D007F367E00747212E8CB0F7E16743F12E88B
:101A2D009D12186BA8BD121A9612F16E10000810B7
:101A3D00010510021080EFE824875004240A80026B
:101A4D0024E8F880E17F377E16742012E89D7E2C05
:101A5D00743F12E89D121A9612F16E1000081001D3
:101A6D001410022080EF18B80904787880E7B87850
:101A7D00E478E780E008B87904780A80D8B8E8D52A
:101A8D00787980D188BD020854E82487923DE850CA
:071A9D000224917F367E3028
:101AA400C313923B12E7D67E3CE4303B027405122A
:101AB400E8B57E1A90BFB3303D0390BFB712814999
:101AC4007F3C7E3A02F2007F127E00747212E8CBF1
:101AD4000F7E20743F12E89D12185785BE1085BFF3
:101AE40011121B5210000810011110021B80F21574
:101AF40011E511B4FFEB75111780E60511E511240A
:101B0400E850DE75110080D9121B527F137E2074B9
:101B14002012E89D7E31743F12E89D12F16E100090
:101B24000810011110021B80DF1510E510B4FFD856
:101B340075100B80D30510E51024F450CB751000FC
:101B440080C61218578511BF8510BE0208887F12FF
:101B54007E24E51112E7657E30743A12E8CF7E35B3
:101B6400E51075F005A412E76502F16E7F491218BD
:101B740098121BABF853BF1F121BB11000081001C1
:101B84000D10021280F218B8FF02780480EA08B837
:101B94000502780080E212185788BD1255F7B80084
:101BA4000302088B021C3B121857E5BD227F487EB6
:101BB4000590BFCD128149E8601CB4040A7E0590EB
:101BC400BFC2128149800C90BFD91281497E38E886
:101BD40012E8BC02F16E90BFD47E2912814980F3D1
:101BE400121BAB601D640460197F5B121898120B02
:101BF400F6121C1612187010000B10010810020CBB
:0C1C040080EF02088B105FE9D25F80E5E2
:101C1000852BBC020888121BAB601F6404601B7F0D
:101C20005A7E0590BFCD1281497E2390BFDD305F83
:101C30000390BFE412814912F16E22121BAB7003B4
:101C400002088B7F527E11121898121875A8BC12C8
:101C50001C7B12187510000810010810020880EF94
:101C60001880EC0880E912187588BC1255F7121814
:101C70007FE875F005A4F5BD020888121BAB604B28
:101C8000E875F03270040475F028A4ADF0FC305D06
:101C900011ACF0FB7A8A125DA4EB30E7050CBC00B6
:101CA000010DAE05AF047C007D64125EAFC005EF90
:101CB0007F517E1A12E7827E2C742C12E8CFD0E07E
:101CC0007E2F12E765124DBF12F16E227F6412184B
:101CD00098121875A8BD121CFD10000810010F10F5
:101CE000021680F218E824CD50EC783280E808E83B
:101CF00024CD50E2780080DE88BD0208887F63E84A
:101D000023C2E012E31075F06484C0F07E2612E86E
:101D1000BC7E2C742C12E8CFD0E080A47F13121864
:101D20009812186BE5BCA2E7923DC2E7F8E8121DD5
:101D30006012F16E10000810010D10021280EE18F2
:101D4000B800EA783280E608B833E2780180DEE84D
:091D5000A23D92E7F5BC79A1F770
:101D5900021E117F6380027F12547F305C01237E53
:101D69002875F06484E5F075F00A84C0F012E8B5CE
:101D79007E2D742C12E8CFD0E07E2F12E8B50F7EAD
:101D89003590C0D9305C0390C13502817C7F6412E3
:101D9900189812187AA8BDE8121D5C12F16E10008D
:101DA9000810010D10021280EE18B8FFEA780F80B2
:101DB900E608B810E2780080DE88BD02081A7F5272
:101DC900121898121875E5BE7F517E2C128EA0F557
:101DD900BE79A2F70202CD7F37121898121870A89F
:101DE900BC5300037F367E32E812E8BC12F16E1054
:101DF900000810010710020780E718180880E2E5BB
:101E0900BC54FC48F5BCF52B02081A7F49121898F6
:101E190012187FA8BE121E4B12F16E100008100195
:101E29001110021A80EFE8240AF8242450E778DB1D
:101E390080E3E824F6F8247F40DB788180D788BEE8
:101E490080C6E8F424DC75F00A847F487E3B02E80A
:101E5900BC7F5212189812187FA8BF121E9212F155
:101E69006E10000810011110021A80EFE82408F81A
:101E7900245750E778A880E3E824F8F824A040DB49
:101E8900786080D788BF021E11E8F424A923C47F93
:031E9900517E3B3C
:101E9C0002E8BC123948754A00D210C211D214D2D1
:101EAC007575791475340012F2E57F007E0290BCD2
:101EBC007F128149904DE87F087E2612E8FBE52BC6
:101ECC0054030F7E3912E8BC12283412E56312A7B2
:101EDC008B12F16E10000810011A10022480C5201C
:101EEC007504057980BE1579E579B4FF05C2757561
:101EFC00790180B02075EB1579E57970A7D27580E2
:101F0C00A3C210C21402081D121870E5BE7F097E10
:101F1C003A02E8BC121875A8BF1218D6120BF612AA
:101F2C001938A8BF12199212187FE5BC1219EB7F51
:101F3C002DA20A1220647F36A26712206412187A2E
:101F4C00E5BC7F3F7E3212E7DCA8BE1203251218D7
:101F5C0057E5BC7F487E3212E7DC121875E5BE7F70
:101F6C00517E2C02E8BC120BF67F1BA20D122064D2
:101F7C007F24A20E12206412186BE5BC121D607F28
:101F8C0009E5BCA2E7122064A8BF12215212187AEC
:101F9C00E5BD121D5CE52B54037F367E3212E8BC86
:101FAC0012187FA8BF121E92A8BE121E4B121861E7
:101FBC00A8BC022197120BF67F09A20F1220647F96
:101FCC0012A208122064121861E5BDA2E37F481228
:101FDC002064E5BDA2E57F5A1220647F51A20C1249
:101FEC0020647F24A20B1220647F2DA2091220648E
:101FFC0012186BA8BD021A9612185785BE1085BF11
:01200C0011C2
:10200D00121B52121861A8BE120953A8BF120991D2
:10201D00120999121870E5BE7F3F7E3A12E8BC1284
:10202D00185CA8BF120919121857A8BD121BB112BE
:10203D001875A8BC121C7B121870121C161218757C
:10204D00A8BD121CFD121861E5BDA2E07F6C8007D2
:10205D00120BF67F48A25E744E400274597E3A020E
:10206D00E8CF120BF67F097E347401205A027403F7
:10207D0012E8BC7F36802E1287FA7F7312845112BC
:10208D0088497F6C1284607F2D801A121861E5BD1E
:10209D00A2E77F63122064121870E5BE7F097E3AB5
:1020AD0012E8BC7F481220C37E1E90BA1A3053032B
:1020BD0090BA15028149121861E5BDA2E192532231
:1020CD001218981F1220B212F16E1000081001059F
:1020DD0010020D80EFE5BDB2E1F5BD1255F780E4BC
:1020ED0022128018EBF516F5147F6C128460127FA6
:1020FD00FC7F647E23E51612E839C3E5169514F5C9
:10210D00167F731284517F2D809B7F2E121898128B
:10211D00186BA8BFE824FA5002780312215212F16D
:10212D006E10000810010D10021280E818B800E4BE
:10213D00780580E008B806DC780180D8799DE8F74D
:10214D00F5BF02081A7F2D7E2C7420B80502742E5F
:10215D0012E8CF7E32E802E8BC7F5B1218981218A5
:01216D006110
:10216E00A8BCE812219712F16E10000810010D1094
:10217E00021280EE18B800EA780380E608B804E28E
:10218E00780180DE88BC02081A7F5A7E2CE802E8AD
:10219E00BCD26875480A12B23BD21412384B12895F
:1021AE0025123FDDC26B12020280F3D214751501A7
:1021BE001287B475B901E5BC20E71C1288E475A638
:1021CE00FF12893112283F12F16E12825110000F48
:1021DE00500512837980E70515E515242050D102AC
:1021EE00057012220202023D1222020205AD1222D7
:1021FE000202088B12220E1218708548BE0255F785
:10220E0012383D12385712646F12F2E590BAB6D2F8
:10221E004912A002129FBB1227EF12F16E1000148A
:10222E0010010510021B80F50548E548640A70028E
:10223E00F54880CF1548E54864FF7003754809805E
:10224E00C2854849123857E5582212B23B12383D22
:10225E00854849C250E558B40F02D25012646F80BF
:10226E003AD22775480A12384B12646F12F2E512F1
:10227E009F2590BF8420290390BF8F1228CBC26A5E
:10228E00123FDD106A0280E1C22712878C85494811
:10229E00122664123857D22912646F12F2E590B9E1
:1022AE00CC12A00020500E1228B512F16E100010A4
:1022BE001001AE80F812283F12F16E10000280FB62
:1022CE000205AD12383DE55830E7137F1B90BF6E07
:1022DE007E0512814912F16E12F1260205AD1238F9
:0722EE005712646F85594986
:1022F50012F2E512282990BF8F12A000129FC51275
:10230500F16E10000810010A10020C80F512236905
:1023150080DB12237680D612F2E512282990BAC600
:1023250012A000129FC5129FC912F16E100008106D
:10233500010A10020C80F512238280DB12239080A3
:10234500D612262A12385712646F12F2E590BED8BB
:1023550012A00012286E12F16E100005100288807E
:10236500F80205AD0559C3E558955950037559004F
:10237500221559E55964FF7003855859220549D33B
:10238500E5491495584003754900221549E5496406
:10239500FF700585584905492212383DE55830E753
:1023A500057F240222DB12385712646F12F2E59082
:1023B500BAD112A0001228C012F16E10000A100145
:1023C5000280F81226D380DE0205AD12383DE558AD
:1023D50030E7057F2D0222DBC26B7559FF12646F52
:1023E50012F2E5122819E55930E70312283490BA9C
:1023F500E312A000129FD512F16EE55820E70610F2
:10240500000810011110021B80F00559C3955950A1
:10241500CF7559FF80CA1559E55964FE70C28558B4
:102425005980BDE55920E711D26B75A70075830763
:10243500C4F582E0B2E7F080A7306B031226810273
:1024450005AD12383DE55830E7057F360222DB122F
:10245500385712646F12F2E590BAEE12A0001228F6
:092465009C40091226C81226FD54
:10246E001224740205AD121875E5BD75F00584F5DC
:10247E00BCF5BDF5BEF5BF1207C71255F705C6DF91
:10248E00F92212383DE55820E7087F5190BAF8023C
:10249E0022DE12F2E590BF9A12A00012283F12F12E
:1024AE006E125457D2AC10001FE55830E7F8306D5D
:1024BE00F51225CA7E207F00501390BFEB12817C4F
:1024CE0012F16E12F12680CAC2AC0205AD1B8B133F
:1024DE0090B9E912817C12F16EC26B7B007514B853
:1024EE001226BD1288B31288655025A814E8243828
:1024FE004004A60105140BC3E5139B50E678B812F1
:10250E0026FF306B0312860612385712646F8082D4
:10251E001287FAE51660E6D26B128910C003128795
:10252E00CBD003A91580C412383DE55830E7057F9E
:10253E005A0222DB12385712646F12F2E590BB0377
:10254E0012A00012286312F16E10003510010280E5
:10255E00F875460512259250157F007E3574079545
:10256E004612E83912F16E12F126D546E7D390BF26
:10257E00A5500390BFEB12A00012F16E12F126804F
:10258E00B30205AD12545712EFC7745212EFD8743E
:10259E005412EF88E5580475590012EFB6128200F6
:1025AE00401612878C1288E4128251400B0559C3D3
:1025BE00E558955950ECC322C2ACD322125457D2CF
:0D25CE00AC12F000204CF1B440F712F00503
:1025DB00B4400312F005B452E2F53812F005B454CE
:1025EB00DA12F005FA60D424EF40D012F005E5388A
:1025FB0070C912F00512F0051281E57B007E031203
:10260B0082DC50102050B412F005204C03B440F77C
:10261B00DEED80A71288C30B1281E5DAE0C322122C
:10262B00270AE55924C8F88602E54924C8F99860B9
:10263B0013146010500F18E608F618E86970F7A726
:10264B00021226FD22E559640F60F91908E618F607
:10265B0008E86970F7A70280E812270A78C8C25009
:10266B00E6B4FF02800708B8D8F6D25022B8D702DA
:10267B00D250A615807C78B812270CE4F9F5A77513
:10268B008307E9C4F582E030E70AE924B8F8243877
:10269B00400276FF09C3E5589950E71226C878B86F
:1026AB0079C8E6B4FF028002F70908E8243850F233
:1026BB00804079B877FF09E9243850F82279C87738
:1026CB00FF09E9242850F82212270AC23D78D7B611
:1026DB00FF04A900D23D18B8C7F5203D0279D819DF
:0826EB0078C8B6FF0122C3E824
:1026F300995007C6C7C6081980F478C81227177FF0
:102703000412811CDFFB2278C81227177F0412886A
:10271300FEDFFB2275C703E54875F004A42480F5AA
:10272300C62212F2E5C23C12813BE53760531460C6
:102733004D14604514603D14603514602D146025FC
:1027430014600E146010146012146035146011804C
:102753003012205D802B12206F80261220EE802104
:10276300122004801C1220988017122084801212D9
:102773001FC1800D121F728008121F208003121FB9
:102783001412F16E12F12A12281912AE5AA81F0858
:10279300E814C23BB51D02D23B75F007203C03751C
:1027A300F009A4FF7E00303C0C7420303B02743EE1
:1027B30012E89D800A740B303B02740A12E8B5D804
:1027C300CF12F16EE51D10000810011010021880E1
:1027D300B9651F7003751DFF051D80AE7005851F4C
:1027E3001D80A7151D80A375F003A4227F7B7E00A7
:1027F30090BEF012817CE54824F640087E0A90BF23
:102803005112817C2212847D7E05745B12E8997ECD
:102813001D745C02E8991228087E3490BF0102817E
:102823007C12847D80031228087E3190BF050281CB
:042833007C122808E3
:102837007E3190BFF602817C12847D7E00800C126F
:10284700847D7E18800512847D7E2D90BFF60281DF
:102857007C1228637E3190BA2402817C12283F7E45
:102867001A90BA2902817C12283F80B912283F7E2C
:102877001890B9D602817C12283F7E1A90BFFB02BE
:10288700817C12847D7E0090B9D612817C7E319046
:10289700BFFB02817C12283F7E1A90C00012817C08
:1028A70012F16ED3100006C310010280F62212281F
:1028B7003F7E1A90BAC002817C12283F7E1890BAD8
:1028C700DC02817C7F007E2012817C02F16E128403
:1028D7007D90C00502817A12847D90C01602817AAC
:1028E70012847D90BE2002817A12847D90BE3102CF
:1028F700817A1228467E2C90BE59301A057E0090A8
:10290700BE5302817C12847D90BEB302817A125F2E
:10291700A10FBF00010E8E04EF799AF7FB7F017EAE
:1029270028A25C924EC25C12E6CFA24E925C78B8A7
:10293700E654F070091F7E2890BE1B128149E4FF00
:10294700FE78ADE612E7D07E0A742C12E8CF7E0C33
:1029570018E612E7D07E16742C12E8CF7E1818E618
:1029670012E7D0303D0A90BE157F147E0112817C9C
:10297700227F097E0178AEE612E7657E0D743A1272
:10298700E8CF7E1278BDE612E7657F097E2378BE21
:01299700E659
:1029980012E76B7E30743A12E8CF7E3508E612E70C
:1029A800650886040886037F127E0012E69612E701
:1029B8001A78C4E612E3107E2912E7827E3B748BF4
:1029C800305D010402E8CF780C7F1C7E02E812E833
:1029D8001D7E09742E12E89D7E0CE51012E81DEF8D
:1029E8002405FF7E1E12F2000EBE3FF9EF2403FFFE
:1029F800D8D922C3740C951375F008A4241CFF7E43
:102A080017742012E89DC3740C951175F008A4245E
:102A18001CFF7E17743F02E89D751600AD6FAC6E03
:102A2800AB6D7403129991E4F5F7A4E5F7F9540F27
:102A38006046E4F5F7A4E5F76510703CE4F5F7A403
:102A4800E5F775F008A47F80CF9FFFE4F5F7A4E5CC
:102A5800F7D2B2241DFE12F200E954F0601A1F12D8
:102A6800F200EE6516700DEF651770081F12F20080
:102A78001F12F2008E168F17D2B21299AFED30E7FF
:102A8800A122AD6FAC6EAB6D7403129991E4F5F7AA
:102A9800A4E5F7540F601DE4F5F7A4E5F765107099
:092AA80013E4F5F7A4E5F765114C
:102AB1007009D2B28D6F8C6E8B6D22D2B21299AF2A
:102AC100ED30E7CBD32278B97998E6F70809E6F734
:102AD10022D215C210C21112F2E5129AC6303C136D
:102AE10090B8B97F1C7E0512817C12F16E12F12320
:102AF10002023DC221C24D1299F0E56F20E7E112B9
:102B01009B0479B8E7540F60EEE764FF60D279B9AE
:102B11008710098711302109799887100987118059
:102B21000A12F2E5122978C23D800512F2E5D23D82
:102B31001229151228191229CF12F16E122A218594
:102B410011131229FB85111312F16E7998A710093F
:102B5100A711E59030E20FC221304D24C24D12F190
:102B61002A12F164801AE53524AA500302023AE5DB
:102B71003524C3500B90BE087F7312813712F16E5A
:102B81002021C810000810011C10023780BDE5117A
:102B910014F51170AD75110C1510E510B407005046
:102BA1008A051080A679B9E76510700609E76511F5
:102BB1006099E51104F511640D7087751101051017
:102BC100022B2C122A8A501DC3740C951175F00822
:102BD100A4241BFF7E0290BDFE12814912F16E12E8
:102BE100F12A022B2C129B04122AC7E59020E21035
:082BF100E53524DC500AD22175
:102BF900D24D129AC6022AF812F2E51228E71229D2
:102C09001579B8E75403600312297812DB4B79B8B8
:102C1900E764C3701712DB4B12321912DB5B1232F5
:102C2900FE756A101298ABD2331234BE12F16E10CF
:102C3900001710013279B8E764C370A4100202804A
:102C4900EEE53524FA4099807C1299F0129B04E54F
:102C59006F20E70A79B8E7540F60EEB7FF8212993F
:102C6900D2129B04022BE91299D2129B0479B8E77C
:102C7900540F60F3B7FFED80D012289C40517FC0FC
:102C8900129B221299A2129B4C60F8B4FFBB78C622
:102C9900866C08866B756A0012B1741298AB1218AB
:102CA9008EE56C65BD701BE56B65BC7015E57064E0
:102CB900FC700F78BEE66577700808E665787002E3
:102CC9008049022BE97995A76F09A76E09A76D7944
:102CD90095876F09876E09876D129B0412DB4B126A
:102CE900DB5B1232FE756A101298ABC2331233B530
:102CF90090B8CFD23C12813B12278A902D087302DB
:102D09002BE9023F26022D90022C827F6C12812E24
:102D190012F126D2201299F0E56F30E70F1280B533
:102D29001255F71256D51256B7022AD2129B04121F
:102D390099D212188EACBFADBE85BDBF85BCBE7819
:102D4900C686BD0886BC1255F712B174E56C6C7065
:012D59000D6C
:102D5A00E56B6D700812B16A12B0FD801F12B12FB7
:102D6A00E56B54036403700612B16A12B0FD129740
:102D7A00FAE56B5403700312B17480CF7F00129B83
:102D8A0022C220022BE912F2E57F6490C1CE1281A1
:102D9A00377F7990C1DB12813712F16E75160010F8
:102DAA00000A10010910020280F505160516C25321
:102DBA0012DB5B75370090B8E9122725902DCA738C
:102DCA00022CD8022DB8022FBD022FC2022DB80242
:102DDA002DF1022DF6022DB8022E34022E38022EC3
:102DEA003C022E43022E4712547380031254687811
:102DFA000A122F16740B12EF86122F5E12EFAF1201
:102E0A002F971298AB1299081297E0129C3D123034
:102E1A00A6D5150C75150A122FA71231CB12EFAFD2
:102E2A00100204E57F70DB022CD8780A8006780449
:102E3A00800278011254738009780A80027801129C
:102E4A005468122F16740B12EF7B122F5EE548128C
:102E5A00EF67E5165403443012EF88742A12EF889C
:102E6A0012EF8812EFAF122F971298AB129908122D
:102E7A0097E0129C3D1230A6D51548854815122FA9
:102E8A00A7E51C12EF67E51B12EF67E51B2548F55E
:102E9A001BE4351CF51CE4A27792E7A27492E0A227
:102EAA007392E112EF67AD75AC74AB73E57DC41232
:102EBA002ED7AD78AC77AB76E57D122ED71231E9F5
:0A2ECA0012EFAF100204E57F709FC5
:102ED400022CD8540F2375F00584F8C3EB33FBECB4
:102EE40033FCED33FDC3EB33FBEC33FCED33FD205E
:102EF400E713EB28FBE43CFCE43D12EF67EC12EF34
:102F040067EB02EF67C3EB98FBEC9400FCED9400D5
:102F140080E8884812284D90BDF812817A12F16E2B
:102F2400E4F54AF549756A207515011298AB1297B4
:102F3400E0D5150E854815E5492401F549E4354ADF
:102F4400F54AE57F70E5744012EFD8747812EF8883
:102F5400746312EF88742302EF7B1231A6799AE727
:102F640012EF6712DB5BE53A12EF7BE53B12EF7B76
:102F7400E53C12EF7BE53D12EF7BE53E12EF7BE58E
:102F84003F12EF7B740112EF67E54A12EF67E549E0
:102F940002EF6712DB56E4F51CF51BF514F5137507
:102FA400150122753800E51412EF67E51312EF6777
:102FB4000513E5137002051422125473800312548E
:102FC4005D12284D12310012F12E756A207515011B
:102FD40075A6FF754A0112984F1297E0129C3D1294
:102FE40030A6D5150975151E1230CA12F1381231E2
:102FF400CBE57912EF67E412EF67E57112308B12BB
:09300400EF67E57012EF67E57B50
:10300D0024ACFFE55F340912EF6DEF12EF67E515A4
:10301D0020E036857D56E412EF67E52EC412EF6D84
:10302D0012EFBE12F13810020630559B12303F02DE
:10303D002CD8744012EF88744512EF88744F12EF3C
:10304D0088744612EF8802EFBEE556123065C4FA59
:10305D00E57D1230652A80BFFBC41230722323CB6D
:10306D001230722B22540FFC24F650027C0090304B
:10307D0081EC932200000101010202030303FA24F3
:10308D0040400A24804003EA3322D2E72274FF2213
:10309D0020E703C3132224C022E53F701F7F7B7EF0
:1030AD000078AEE612E823EE2404FE743A12E89D91
:1030BD00EE2404FEE53E12E81D12F16E22C015C08D
:1030CD0016D212128FCFC212D016D01578AEE612CC
:1030DD00EF7BE53E12EF7BE53F12EF7BE54512EF0F
:1030ED0067E55212EF67740A12EF6774C012EF674B
:1030FD0002EFBE744012EF88745412EFD8744E1262
:10310D00EF88743012EF88E5165403443012EF88BF
:10311D001231A6742312EF7BE53D12EF7B799AE70E
:10312D0012EF6712DB5B78ABE60812EF7BE6081255
:0D313D00EF7BE60812EF7BE612EF7BE53E2C
:10314A0012EF7B1236ACE51212EF7BE51112EF7B20
:10315A00740112EF6790C02712320B756A10129829
:10316A00AB740212EF67E412EF67787B12EF6078B4
:10317A007D12EF60787712EF60E4FEFF780712EFB6
:10318A006012EF60E57412EF67E57512EF67E412FB
:10319A00EF67E412EF6712EF6002EFBE75C70375BF
:1031AA00C6FF75B901C217751D0085BC1C85BD1BFC
:1031BA0085BE1A85BF19125D1CEE12EF67EF02EF8A
:1031CA0067E57512EF67E57412EF67E57312EF674B
:1031DA00E57812EF67E57712EF67E57612EF67E5B4
:1031EA001664016011E55E12EF67E57A12EF67E592
:1031FA0016640260012278BCE612EF6708E602EF65
:10320A006775A700E493700122A312EF8880F51274
:10321A00DB5B857946787A796412DB7774641261AC
:10322A00178E471232FE756A20D23D1298AB129958
:10323A0008123335303D09307406C23D8E1E8F1F89
:10324A00E57F602BE54C24FFF54CE54D34FFF54D49
:10325A00454C600512980180D2751D3C1298AB123C
:10326A0099081297E0123335E57F6003D51DED12F8
:10327A0033969033AE12E8FB203D0DAE1EAF1F12FF
:10328A0033969033A712E8FBE546FD700B90C15DBB
:10329A00305D1190C159800C04700E90C159305D97
:0632AA000390C1557F38BE
:1032B000024DBAE4FFFC7E05305D047E027FB3124E
:1032C0005EA2AC06AB07125D6C7F38C23DE51C60A8
:1032D00007D23D7E2C12E88AE51B203D026007D212
:1032E0003D7E3012E88AE51A203D026007D23D7E1D
:1032F0003412E88AE5197E3812E88A024DBFE540AB
:1033000075F03CA42541FFF54CE435F0FEF54D7C0D
:10331000007D10125EAF0F8F4BAF4CAE4D7C007D29
:103320003C125D827C00AD4B125EAFEE4F70010F20
:103330008F4C8E4D2278647973C2D112334CFF7852
:10334000677976D2D112334CFE02F200C3E796FBC6
:103350000809E796FC0809E796FDA2E792175003D3
:1033600012603775135A30D10E751320B217AA4761
:10337000125DB6AB04AC05E546600B04600BAA46D3
:10338000125DCDEB03FBEB03FBEB543FFBE5132B93
:103390002017029B9B22EE141430E701E4FEEF1489
:1033A0001430E701E4FF2205057088A88870050540
:1033B0002020F8202012F2E57E1E7F1C12F200DF92
:1033C000FB12F2007E1E7F1C12F200DEFB7E1D7FD0
:0633D0001D12F200DEFBFD
:1033D6007F007E2178ADE612E81D7E29742E12E864
:1033E6009D7E2D18E612E81D7E35742E12E89D7E10
:1033F6003918E612E81D7F077E21745412E89D7E77
:1034060025744F12E89D7E2D78AEE612E81D7E35B6
:10341600743A12E89D7E39E53E12E81D78AE123602
:10342600AC7F0E7E21744C12E89D7E25744112E815
:103436009D7E2DE51212E81D7E35743A12E89D7EBA
:1034460039E51112E81D7F157E25744412E89D7E2C
:103456002DE54012E8237E35743A12E89D7E39E563
:103466004112E81D7F217E0190C12812817C7E0ECB
:10347600AC77AB7612E6CF7E2B85795F85787B12AB
:10348600EC7A7F287E0190C12C12817C751D2B75EC
:103496001E10E5741236607E25742F12E89D751D88
:1034A6002D751E2BE5751236607F367E0290C1188B
:1034B60012817CE57212364A12358E20330312369B
:1034C6003B12DB56AE4DAF4C7C007D40125EAFBF6B
:1034D60000010F0FAC07AD07E4FED23D1298AB1208
:1034E600990812352EE57F602CE54C24FFF54CE556
:1034F6004D34FFF54D454C600512980180DE751D73
:103506003C0E1298AB129908123533E57F6006120D
:1035160097E0D51DED7F783033027F3612DD681FC8
:083526001F7E00743002E89DD5
:10352E00DD03AD040E7F783033027F36E55E20E793
:10353E002EE57A8549F0A4A9F0E57A854AF0A4290A
:10354E00F9E435F0FAE55E8549F0A429E435F02A70
:10355E00FAE55E854AF0A42A30330113CF9FFF129D
:10356E00F200103D18C3EF9B50131BEF6B600E8FD4
:10357E00018B0712F2001FEF6970F8AF01AB072243
:10358E0090C0DD305C0390C0F6754A40754900AFBF
:10359E0076E577FE20E76B7005EF24105064EF247C
:1035AE00A8EE34FD401190C0E2305C0390C0FA7575
:1035BE004A1975499A8075EF2450EE34FB401190EC
:1035CE00C0E7305C0390C0FF754A0C7549CD805C36
:1035DE00EF24A0EE34F6401190C0EA305C0390C1A7
:1035EE0004754A067549668043EF24F0EE34F140C7
:1035FE001390C0ED305C0390C109754A04754944BF
:10360E00802A8028EF2490EE34E8401190C0F030EC
:10361E005C0390C10E754A0275498F800F90C0F3FE
:10362E00305C0390C113754A0175499A227F40128E
:10363E00817A7F4612DD687F5F02DD687E2112E3AC
:10364E001012E8397E2F90C130305D0390C13502E3
:0D365E00817CAE1E75F064305C0375F032A7
:10366B0084C0F0F87004EE2404FEE51D12E89DEE14
:10367B002404FEE8600712E88AEE2404FED0E0750D
:10368B00F00A305C0375F00584A8F012E88AEE248A
:10369B0004FE742C12E89D0E0EE8305C012302E848
:1036AB008AE53E2541F51124C45003F511D3E635C7
:1036BB0040F51224E85002F5122212AE54C2101239
:1036CB00F2E57F057E0990B6E81281497F127E06EE
:1036DB009036F512E8FB7F2B7E0190375D12E8FBED
:1036EB007F267E2A9037CF02E8FB113007FE1FE0C2
:1036FB0001E101F80F00061B00F80C00180E007C0E
:10370B0010007006003C2000E006003E4001E00483
:10371B00001E8003C004001F0003C000000F000741
:10372B008000000F800780000017800F000000272B
:10373B00C00F00000043C00F00000083E00F00200B
:10374B000301F00700C00F01F80383007F87FE0120
:10375B00FC000E3E180000030000000018000003E0
:10376B0000000000380000000000000030000000E6
:10377B0000000000FC761F0E1C6030ECFCBC3F17F9
:10378B002DF0F978613866264F619A706070C60E1D
:10379B001EE330E06060C60C1CC360C0E0618C0CA3
:1037AB0018C7C0C0C0E18C1C39C611C0C4C19C99DC
:1037BB0031963180C8C1FF1E31E7E180F0C0EE1CAD
:1037CB0031C38180061238E18034D340659640794D
:1037DB00E640C3448082230012F2E57F3E7E1790C1
:1037EB00BF3B12814912F16ED2A47F8CDFFEC2A4C3
:1037FB00C2AFD2C075C0107581D874FE12381612C4
:10380B00F12AE4F5F9F5FBC2B480F7D2A6C2A512F2
:10381B00AE3912F12A02AE5A75C703E54875F004AA
:10382B00A42480F5C6C23C75B901E5BC047002D274
:10383B003C22121870E5BEF54824F650037548007B
:10384B00753400753704C228D229D22A75C703E50F
:10385B004824E75003754800E54875F004A424801C
:10386B00F5C6751607751700C23C123898123898B2
:10387B001238981238988517581558755900E5481D
:10388B00B40A09E5586005F46002055922203C1D75
:03389B0075B901FB
:10389E0005C6AABCABBDACBEADBFEA1238B9EB12C1
:1038AE0038B9EC1238B9ED1238B922203C07F515AB
:1038BE00B4FF03D23C22C0C7C0C61287B475A7049A
:1038CE00851683E517C4F8F58275B90105C6E5BC02
:1038DE00F0C582F82406F92403C582E5BDF0E5BEE5
:1038EE00F0E5BFF075B90105C6E5BCF0E5BDF0E544
:1038FE00BFF08516838982E4F075B90105C685BCD3
:10390E001385BD14E4F0F08882E5BEF0E5BFF075D6
:10391E00B901E5BCF0E5BDF0E5BEF0E5BFF075839D
:10392E0006E51723541E24B0F582E513F0E514F0D6
:10393E0075A700D0C6D0C705172212B06478BEA6F0
:10394E004808E4F6F55908761808F6D23608760ACD
:10395E0008F6060876BEC237C22BC21AC21FC25460
:10396E00C255129B6F12384BC229C22AC207C227F8
:10397E00C268121861E5BDA2E59243C24AE4F52E73
:10398E00F534F536F52F78B6F678B5F678A9F678DB
:10399E009EF678B8A65E08A67A12E638C26BC233D7
:0239AE00C2381D
:1039B000C240C223C2221239D075460278C5A6463B
:1039C000C23AD221C219C226E4F542F541F540229D
:1039D000E45407205E09B4040040027403801B1203
:1039E0001866C313A9BC600C14A9BD600714A9BE56
:1039F0006002A9BFE94001C45407F5372212383DDF
:103A000012646F1207BE12F2E512286EE5580470B8
:103A10000A7F327E0590BF6E12814990C1C512A007
:103A2000021207187F7290C1BA12813712F16E101C
:103A3000000510020480F8D322C3220200EF1218FE
:103A400061E5BD20E7051239FD40F0123948129DAD
:103A5000E012B23B789F7680754A001297B1D2107F
:103A6000C211C213C212123EC712544775A61E12CB
:103A7000ED8612D7F320250CE59054057009E53545
:103A800024E25003023B74E5322418400D75F00C1B
:103A900084E5F070E0123FE080DB7532F012B23B5B
:103AA000E53124F39205201203123E20123B302010
:103AB000371A12A6D1200A0312B6CA123FE0128F9B
:103AC0009E123FE0129DE3123FE0803779247B1184
:103AD000123B1712F2E512EB0412E31E12E68E12ED
:103AE000E4D71215841215111228F979607B1D1282
:103AF0003B17799B7B1D123B1779D67B0E123B1728
:0F3B0000123FE030120E301A0B8009E532241606
:103B0F0050F212179D023A69D3E9953250FAE556F1
:103B1F00D23D12160FE552F556C23D12160F02F1A5
:103B2F006E301238E54024EE40267A0AC3E53F9501
:103B3F004B601D402824E24017305405C254757F56
:103B4F0001E54B0475F03C8485F04B1297C0DADC2D
:103B5F0079BCE7D2E7F57F09877EC27722F4042488
:103B6F00E250ED80D412F2E57F2A7E0E90C02B1228
:103B7F00814975A6FFC2101012137F367E0890BAC6
:103B8F000712814912F16E12F1230200EFD22112B6
:103B9F00B23B1297C07F1E7E0B90BF491281491214
:103BAF00F16E123BC77F3E7E0790BB961281491282
:103BBF00F16E12F11D0237F3D2201214E3C237D285
:103BCF0015D214120BF675B90575B902129939D2BF
:103BDF005512982D7D0012B122129943E56A6005A6
:103BEF001297E080F712188E85BEBC85BFBD856B1E
:103BFF00BE856CBF75B90575B90285BD6C85BC6B8B
:103C0F00756A20129939123C9A857A621299437516
:103C1F006A001298AB7570FC854077854178851FD7
:103C2F00797818797A12DB7712B1741297D812F16A
:103C3F003879B877C309A77109A77209A77309A7BC
:103C4F007409A77509A77709A778129943756A10A0
:103C5F001298AB7F087810797212DB7985627C85B8
:023C6F005E7D78
:103C710079C0A71509A71409A77409A77509A7721F
:103C810009A77309A76C09A76B129AC6125FA18EC7
:103C91007E8F7F129AED0297D878107F0EE4F60896
:103CA100DFFCF564F565F567F5687515FC751AC0F7
:103CB100751DC0756640756940754A0112984F308F
:103CC1005503023D501297E0E571B510004002F531
:103CD10010E4F511E512207502E513C3957950063C
:103CE100207545857913D3E57A9514E5156480FF30
:103CF100E55E64809F400C857A14855E15857B1690
:103D0100855F173074B3C2D178647973123D2E7810
:103D1100677976123D2ED2D178187973123D2E78BB
:103D21001B7976123D2E809185791280B9D3E79661
:103D31000809E7960809E66480FFE764809F20D1BF
:103D410001B3400AE7F61819E7F61819E7F622E574
:103D51001AB4C00E7873791812DB7778737964120C
:103D6100DB7778187964C2D1123DC17418126117DA
:103D71008E47AE1EAF1F781B7967D2D1123DC1C3EA
:103D8100E51F9FE51E9E50048E1E8F1F7EFF7FFF45
:043D9100AC1EAD1F98
:103D9500125EAF7A04EF8AF0A4E5F0CE8AF0A42E85
:103DA500FEE435F0BEFF011E60051460057EFF8E42
:103DB5001F22EE7E0020E7F77EFE80F3C3E697FB29
:103DC5000809E697FC0809E697FD1818191930E760
:103DD50003126037C3EB33FBEC33FCED33FDEB3300
:103DE500EC33FBED33FC30D105AA47125DCD0BBB9F
:103DF50000010C751E03751FFFEC24FC40048C1E8E
:103E05008B1FE627FB0809E637FC0809E637A2E71A
:103E150013F618EC13F618EB13F62210131978B5F0
:103E2500E624FA401AE57124F64008E57924F640BF
:103E35000280330606802F12F134E59030E2DFD29E
:103E450020753612D22EE4F534F55A129BA1123E96
:103E5500D5C2191239D012AA0012AA2DD212853F45
:103E65004B205E02D2281239C8307335E53F20E079
:103E750030E55D455C602A75A7009006FAE0255C93
:043E8500F0FBA3E0CB
:103E8900355DF0FCA3E03400F0FDA3E02401F0F877
:103E9900A3E03400F0F9125F488C4E8B4D2275A7D0
:103EA900009006FDE0F9A3E04960F2121884C3E529
:103EB9004D9560F5BCE54E9561F5BD0255F775A7C1
:103EC900009006FA7F05E4F0A3DFFC22D214123F2A
:103ED9001BE6F008DFFB857A62123F117570FE78E8
:103EE9003A797112DB771297DD123F1185627A8573
:103EF9005E7B7570C01297DD123F1BE0F608DFFB91
:103F090075A700D254C2142274FF7870F608B880DD
:103F1900FB2275A7049004F078707F102212F2E555
:103F290012F16EC258C259123948753901754A01E0
:103F390012DB5612984F1261158E47C210D211D258
:103F490014D212129BA112AA0012AA2D12ED867583
:103F5900A6FF753609753200E59020E206E535249D
:103F690005400CE59054057019E53524E25013C25B
:103F790011C21212F2E512F16E12F12612F1640267
:103F89002CD8C221E54AB40202D22112984F128FCD
:103F99009E30260F1264D1129DE3753606E5367000
:103FA900FCC226129DE0123FE0E54A20E021B4025E
:0F3FB90009753900E53670F98092E53960FAFD37
:103FC80024E24002053912984F2026C9DDF880E91D
:103FD80075390080E475370410003A100116100294
:103FE80016E52F5407600312AE4E20784C20790A4C
:103FF800207A1F220241F2024139E5376009146034
:10400800091460090242AD02421302427EC27902DB
:1040180042D402416C20110C3037091214E3753474
:1040280000C27822E53724FC500FE53764076003A7
:1040380002434A02430E0241032011FAE59020E2AE
:10404800028056753400201203D2132278A9E67034
:1040580017C226767DE5377005106B02D26BD277D2
:10406800753614D22E029B96E5376043146040B42F
:104078000227200B24E6249B401F2414501C12AA5C
:104088000090BF1C7F207E0812814912F16E7536A0
:1040980008D22E78A9E624ECF622241940FB241431
:1040A80050F712AA0012AA2D90BF257F2980D72089
:1040B80028E7E54824F640E1E5580460DC7F5D7EAA
:1040C80010E6249B40D324145015C2330559C3E588
:1040D8005895595005855859D22690BF0A80A92469
:1040E8001940B6241450B2E5596002155910260635
:1040F800E5596002155990BF13808D10780122751B
:0F4108003900E53424384007754A017534002228
:10411700700AE54A30E0F2754A0280F014600875CB
:104127004A0612AA2D8006754A0412AA007539019B
:1041370080DA302909C229D22A7559008005302A28
:104147001BD229129FB1129F7FE53524AF4004751A
:10415700340022753700C229C22A80F320684E3006
:104167002703D26A2220110A3037071214B6C27AFF
:104177008015D2221244E612F16E107A0122E5343C
:10418700243840071239D075340022700FAA37122D
:1041970039D06A70F274011239D180EB041239D127
:1041A70024FC50E3E537B40706D22880DA8036C20C
:1041B70028E53724FC2324BEF879C4E7F9A7480982
:1041C700A75979C4E8F78648088607E537B405058F
:1041D700754818D2361238578F59E537640670027A
:1041E700D20702418E1244C202446CE537601D14A7
:1041F700600F14601114600BE53724F9400B02437C
:10420700C480740242AD0242FD02439120110A208C
:104217001207C279123EA78012D223124CA6107938
:104227000122E534243840077546017534002278A9
:10423700D87020304A0BC24AE624F85004B24380B3
:104247000AD24A7614E54624FE40DDE54660D915D4
:064257004680D8B600D538
:10425D00B40500500C04F54624FA50C97546058086
:10426D00C424F950051285A480BB100FB8D20F805D
:10427D00B4D223E53464C86003124CA61079012230
:10428D00E534243750097011105B3CD25B80381037
:10429D000802D208124CA6802E100C2BD20C8027AF
:1042AD00D223124CA610790122D24BE5342437408B
:1042BD0002801424FC402824047010C258C25920D6
:1042CD001105D22E75360775340022D258C25914F5
:1042DD00700280F3C258D2591460ECD25880E812A3
:1042ED00186BE5BCB2E7F5BC79A1F71255F780D78D
:1042FD0078B8A65E08A67A2011CD753605D22E8027
:10430D00C630122B129FEB055BE55B75F00B84E558
:10431D00F0F55BE55A24F64009E55A955B500375B7
:10432D005B00129FEF12F16EE5346003D534D27548
:10433D00340022D229D22A75480A024432C24010D2
:10434D0007F1302903024432129FAD129FC1102A8A
:10435D001BC2330559C3E558955920E7025008751E
:10436D005900E548B41816E558B4FF037559001205
:10437D009FD512F16EE5346003D534C122D22A12D5
:10438D009FB180EE301223129FEB155BE55B30E79A
:10439D000C755B0AE55A24F64003855A5B129FEFB4
:0343AD0012F16E9C
:1043B000E5346003D534DA75340022D229D22A7567
:1043C0004817804CC2401007F2202944129FAD12BA
:1043D0009FC1102A22C2331559E55930E71C855870
:1043E00059E558B4FF03755900E548B41802800A2E
:1043F000D22A129FB1800E855859E558B4FF037533
:104400005900129FD512F16EE5346003D534B52200
:1044100020106220115F7F180548E5486418700875
:10442000F54830270375480A123823303C2DDFE861
:10443000802620105A2011577F181548E54830E78C
:1044400005754817800A64097006302703754817F8
:10445000123823303C05DFE275480A1238571264DF
:104460006FE532244C5005129F7F8003129F257503
:10447000340002F16E1244A97F15E5486B70048A7E
:104480004880020548123823303CD0DFED80CC1242
:1044900044A97F15E5486A70048B488002154812CC
:1044A0003823303CB6DFED80B27A007B09E537B4C3
:1044B0000401227A0A7B17B40601227418FAFBF56C
:1044C000482275A704758307E559C4F582E0E0F535
:1044D00073E0F574E0F575E0F576E0F577E0F578F2
:1044E00075A70002646FE59020E23EE53424375062
:1044F0003812452A124507205E4F7F2C90B7A6122E
:07450000457190B7AF806A1E
:10450700E534243775F009A42435FF205E0624BE60
:1045170050027F3EEF249B50027F627E32748912E5
:10452700E8CF2275A7049000317E087F3AE4F0DFD8
:10453700FDE5822446F582E43583F583DEED75A734
:1045470000227F2C121866E5BD12455AE5BE1245BA
:104557005AE5BFF8C4124560E8540775F009A490FE
:10456700B7942582F58250020583EF2409FF028163
:01457700370C
:109DDD00029E9A12F2E5E53724FC40F4B4FE1420FD
:109DED00110EE590F45407600122E532247450EF12
:109DFD0002A6DD12F2E512EA7212EB0412E31E1254
:109E0D00E68E12E4D77E197F3612E45812F04D1209
:109E1D00E46EC206E53760051460338053C23A1212
:109E2D009F3E124D61124EF61251DC126F3B126FB6
:109E3D0063124A14E54864186009E54824F6500396
:109E4D001252C712A67312E1A1124DFC8014D23A20
:109E5D00129F64124580124DCB12DCCE12A67312E6
:109E6D00E1621267B012EB4B1262811265808012B3
:109E7D00129F4A12DC0B12EC1D12DC9D12A67312FE
:109E8D00E17930101412E3E112E3B0800C12F2E527
:109E9D00E53724F9401E129F273022091244E6E5CA
:109EAD00347002C222302309124CA6E5347002C26E
:109EBD002302F16E12281975170012EE317F12125E
:109ECD00DD5630124A75100075A7047583061265AC
:109EDD002AE51075F009A42415FFF5177E00E5128B
:109EED00602F75F06484E5F00F12E81D1F7E0EE5FE
:109EFD001112E3667516231266E60510C3E55A9531
:109F0D00104006E51024F550BF301203129FEF806C
:109F1D0088745D12E8CF80D5C2493029051227EF2C
:109F2D00800312281990B9CC12A002202A76029F24
:109F3D00D5301223305E2030501D02A2E9301217A9
:039F4D00305E067D
:109F5000200B1102A94A12DD4F7F1712F26075170C
:109F60002002EE3112E9E912E98A3012112051057E
:109F700012EA49800612E09F12DE7F125BDE22E4C5
:109F8000FEFFE54824F6400D90BF5112817C7E16FD
:109F9000E54802E88AB40E0690BF5702817C90BF64
:109FA0005E12817C7E12E54824F702E8237D208042
:109FB0000C7D3F302A077D633029027D3C7F008085
:109FC000247D2080127D3E800E7D3CE54975F007A2
:109FD000A42406800A7D3FE55975F007A42409FFF3
:109FE00064027001FF7E1CED02E89D7D2080027DF1
:109FF0003FE55B75F009A42416FF7E09ED02E89D9C
:10A00000C24912A066B4FF012275100012A07D792A
:10A0100020E030E702792F304917121BABFAB40465
:10A0200008E510700C79658008EA146510700279F3
:10A0300023E97E1812E89D7E20E51230E70890BAE9
:10A040000712817C8016E51112A0F31267462010DA
:10A0500005201102800630120312A0A50510C3E5E9
:10A0600058951050A7227E207F0012817C129F7F7E
:10A070007E007F0690A12512E8FBE5582275A70413
:10A0800075830712652AE51075F007A42409FFF50A
:0DA09000177E00E51212E89D7805EE24040D
:10A09D00FEE012E89DD8F62212A1B012A1C6FD7CF9
:10A0AD0000AE1CAF1B125EA2BE003A8F00C3E57A54
:10A0BD009513FFE55E9514FE402B7C007D28125E06
:10A0CD00AFC3EF98401F75F0058404FB24F95002CF
:10A0DD007B067E2CAF170F12F2000F12F2000F123B
:10A0ED00F2000EDBEF2264B4602464B475F03284A8
:10A0FD00C0F012E88ACE2404CED0E075F00584C0FD
:10A10D00F012E88ACE2404CED0E02302E88A90A192
:10A11D002102817C2D2D2D000140FFFFFFE0FFFF6F
:10A12D00FFFFC25030124220283FE558F4603A201C
:10A13D004803200934D250E559F5103033096558DC
:10A14D006005204802051012A17A12A1D675A70448
:10A15D009006DCE512F0E511F0E517F0E510F0756D
:10A16D00A7049006E0ECF0EBF075A7002275A704AC
:10A17D0075830712652A7813E0F608B819FA900668
:10A18D00D07811E6F008B819FAE51CF516F0E51BC4
:10A19D00F515F012A1B09006DAE514F0E513F0759F
:10A1AD00A7002275A704758306E51023541E24B05D
:10A1BD00F582E0F513E0F5142212186BE5BD248746
:02A1CD00E5BDEE
:10A1CF00923B500224912212A1C675F005A485F08E
:10A1DF0012F511E4F519FEF51CF51D129939C23D62
:10A1EF00C2567F3C12DE04303D05751900807DDFBD
:10A1FF00F3E5596558700A301007EE24D35002D298
:10A20F00568C1B8D1AE519FD24E250DEAE1CAF1DD6
:10A21F007C00125EA2EFF51924F650CEAC1BAD1ADE
:10A22F0012DD3E20D1108E048F05E51975F0A7A41D
:10A23F00AEF0FF125EA2AC12AB117AA0125DCDEBA5
:10A24F0033FBEC33FC20D11AEF9BEE9C5014C3E58B
:10A25F001213FCE51113FBC3EF9BEE9C4004AC06FD
:10A26F00AB07204807203B048C128B119006E2E5C8
:10A27F0019F012A2BEAC16AB157AC8125DA4A912C2
:10A28F00A811125F48ED7005EC249E50057C807B71
:10A29F000822C3E57A305602E55C9513FFE55E3080
:10A2AF005602E55D9514FEC3EF9BFBEE9CFC22AEC0
:10A2BF0016AF157C00E519FD24F6501A125EA27C2C
:10A2CF00007D06125D827C007D05125EA28F10EE6E
:09A2DF00F51724E950037517FF7F
:10A2E8002212DD4F12A30612A34912E63D12A36FF4
:10A2F80020480912A45D12A48D02A4F080747F176F
:10A308007E2020480E748A204D101262EE500E7482
:10A318002F8007746A305F02746712E8CF75A7044C
:10A328009006D07811E0F608B819FA7F177E007801
:10A3380012751905E60812E8CFEE2406FED519F4C1
:10A348002275A7049006D8E0F516E0F515E0F51497
:10A35800E0F513E0F512E0F511E0F517E0F510E08F
:10A36800FCE0FB75A700227F187E26AC14AB130215
:10A37800E6CF9006E4E0F51CA3E0F51B7F2A304EFB
:10A3880013121861E5BF90BFBBB4010390C1B412AA
:10A39800813780420F7E00745312E89D9005CBE010
:10A3A800F830E705E53F30E0091F7E00E8540F125A
:10A3B800E8B59004EEE0FEF51EA3E0FFF51F12A439
:10A3C80005E51E24E9500C7E06742B12E8CF7E0C9E
:10A3D80012E8CF12A435C20375172A75162712661C
:10A3E800B5202415205F15D2037F2A7E1E90A42352
:10A3F800304E0390A42C02E8FB205FEB227C007D0A
:10A408003C125EAFA805EF7F2A7E0812E7D67E12BF
:10A41800743B12E8CB7E14E802E7D00707384C9E5D
:0FA42800BAF264380707387CE6C2E67C38AC1C11
:10A43700AB1B7A48305D027A27125DA4A91EA81FBC
:10A44700125F48ED4C60027BFF7F207E28EB12E70E
:10A45700DC7E3902A9DD7F2B90BF6412817AE51774
:10A46700F46022AE17AF107C007D3C125EAFA805EA
:10A47700EF7F2A7E0C12E7D67E16743B12E8CB7E5E
:10A4870018E812E7D022AE12AF117C007D0A125EE7
:10A49700AFA805EF7F207E3012E7D67E3A742C12E4
:10A4A700E8CF7E3CE812E8B50F7E29744502E89DA7
:10A4B70074858007748720560274867E2912E8CF38
:10A4C700301707742D7E3A12E8CF227C007D0A12DE
:10A4D7005EAFA805EF7F2A7E3012E7D67E3A742C4E
:10A4E70012E8CF7E3CE802E8B512A621E54824F63B
:10A4F700500512A4D280B9E559046558600D12A41D
:10A50700D212A4B7E559655860AA22A217923D8EC8
:10A517001E8F188515179006D0E0F5118558101570
:10A52700101251BCC3E51195105002F404F924A68A
:10A537005005C374B399F9E975F00584F924EE5011
:10A5470002791190A661E993F5F01207D2E5CC7074
:10A5570004E930E702747F23A4A9F0E51B2517FD62
:10A56700E51C3516FEC3ED99F515EE9400F5167545
:10A57700A700758306E55823541E24B0F582E0A38F
:10A58700F513E0F51412A621203D2C2017291218E7
:10A597006BE5BD2487E5BD5002249175F007A4FB48
:10A5A7009518E5F0951E400FEB9FE5F09E4008EFEC
:10A5B7009518EE951E500EA23D9217AE1EAF1812BB
:10A5C700A4D202A4B7306B1012A5BEE53F20E00766
:10A5D70074867E2212E8CF2275A7009006E0E51662
:10A5E700F0A3E515F012A4D212A4BB74857E231242
:10A5F700E8CF85581012A17A12A30612A3498C1628
:10A607008B1512A36F12A28412A16C12E63D90065D
:10A61700E2E0F51912A2BE02A45DC3E57A30560244
:10A62700E55C9513FFE55E305602E55D9514FE92F5
:10A6370017500312601FAC16AB157AC8125DA4A998
:10A6470006A807125F487E037FE7ED700CEB24181E
:10A65700EC34FC4004AE04AF032200172E43576CC2
:10A667008092A4B6C5D3DFE6EDF3F8FD305E4F3038
:10A67700504C75A7009006E0E0A3FCE0FBECA2E7D6
:10A687009217402024FE50047F3B8022AE04AF0384
:10A697007C007D14125EAF74542F2017029F9FFF1A
:10A6A7007462800C12602FEC24FE50E07F6D743DC5
:10A6B7007E0012E89D7E017D197C0312A6C6227FCB
:10A6C7003D12F200EF2DFFDCF822E537B40206E574
:10A6D70034243750292212F2E512EA7212E31E12CD
:10A6E700A85D12DB9912E18912A8B51265807F2057
:10A6F7007E2B12E45812EB0412F04D1244E612E5D9
:10A707006312A78B125B7802F16E20041EE579FDB8
:10A7170024A050027D5FED24CD401E744520750CAA
:10A727002DFFF51212A7601FBF44F922C39DFFF545
:10A737001212A7600FBF46F92220750EED2413FFF2
:10A74700F51212A7600FBF78F922C374779DFFF542
:10A757001212A7601FBF12F922EF24BA4008243350
:10A76700FCC374329C1404FC24D750047C23800956
:10A77700EC2375F005842413FC7E0512F2000EEC21
:10A78700B506F822E59020E206E5342437400312A7
:10A79700A7117F457E047D1212F2000EDDFA7F437A
:10A7A7007E00746412E89D7F4F7D1212A8467F3B9E
:10A7B7007D1212A8467F597D1612A8467F317D1655
:0EA7C70012A8467F637D1A12A8467F277D1ACE
:10A7D50012A8467F6D7D1E12A8467F1D7D1E12A8FC
:10A7E500467E057F1912F2000FBF72F97804E579EC
:10A7F50024CD50027809E8305C0123F87F1B12A8AC
:10A80500357F6B12A83518305C01187F2512A835E5
:10A815007F6112A83518305C01187F2F12A8357F8B
:10A825005712A83518305C01187F3912A8357F4DAD
:10A835007E00E875F00A847004E802E88AE802E818
:10A8450023EF6512600C7E04EE20E00712F2000E85
:10A85500DDF62212F23080F790C07A7F287E2C1226
:10A86500817C7E3B12E6E6AC5EAB7A7F307E19C218
:10A875003D12E72590BF687F5D7E2D12817C78B9FA
:10A88500C3E57A9618FBE55E96FC7F507E19D23DAE
:10A8950002E725E51164B4700122E51112F0BD78D7
:10A8A50031790F7D0B12F1C31F1E90A94502E8FBFC
:10A8B500E5716012E57012F0BD7831790F7D0412F3
:10A8C500F1BF0DBD0AF97F0112A91D7F1D12A91D3A
:10A8D5007E2312A9277E3F12A9277E247F1712A95E
:10A8E500317E397F0212A9317E247F0712A93B7E72
:10A8F500397F1C12A93B7E317F0212F2007F1C12A8
:10A90500F2007F0F7E2412F2007E3E12F2007F0CD1
:10A915007E2E90EBF202E8FB7E2A12F2000EBE3983
:10A92500F9227F0812F2000FBF17F9227D0612F2F5
:10A93500000E0FDDF9227D0612F2000E1FDDF92251
:10A945000303E0A0E012DD4F7F1890B7E412817A8F
:10A955007F217E01744112E89D7F2A7E0174531286
:10A96500E89D9005BEE0F51AA3E0F519A3E0F51EF4
:10A97500A3E0F51D851A1C85191B75172012A9FA68
:10A98500E519251DF51BF51DE51A351EF51CF51EEA
:10A9950075172912A9FA9005BA12A9EAAC1AAB19CA
:10A9A50075172012A9B89005BC12A9EAAC1EAB1DFB
:10A9B500751729EC7006EB24CD4001227A48305DED
:10A9C500027A27125DA4125F48ED4C600122AF1791
:10A9D5007E07EB12E7827E1A0F90C13D305D039032
:10A9E500C14002817CE0FEA3E0FD129D19C3EB9DF1
:10A9F500F8EC9EF9227516270266E6129D1975A7D1
:10AA0500049005B478737F06E6F008DFFBECF0EB05
:10AA1500F0E0E0E0FCE0FDE0FEE0FFEF2DFFEE3CC6
:0EAA25009005C0F0EFF0801275A7049005BAFE
:10AA3300E0FBE0CBF0EBF0E0E0E4F0F075A7002200
:10AA430075A7049005B478647F06E0F608DFFB750C
:10AA5300A7001268F59005BEE51CF0A3E51BF022E4
:10457800D23C799E77008002C23C129939E4F5104A
:10458800F511F512F513F514F515F516F517C23DE5
:104598001248C5203D1F1248C5203D19E51F30E5CA
:1045A8001130E40E1245EF303C08799EE724F550AF
:1045B8000122D510DBAE14AF157C00AD12125E7C63
:1045C8008F55AE16AF177C00AD13125EA21260A90C
:1045D8007E00E55530E7011E2DFFE43E30E7027FFF
:1045E80000740A2FF55622C235E51CAF1DBFFF0522
:1045F8000FD235F404FABF003F532CF8E518AF1971
:10460800BFFF050FD262F404BF002D20E72A205B0C
:104618000123FF24AA4021E51AAE1BBEFF050ED2D6
:1046280061F404BE00128547F0A4E5F020E70920F4
:104638005B0123FE24AA5001227C807B80305166D6
:10464800302163C006C0078AF0E545A4AEF0FFE557
:1046580056205B011375F009A4ACF0FD125EA2743C
:10466800FFBE0001EFFA24C050027A3FD007D006FF
:10467800E55212F0BD303504B2D5B2D1EA8CF0A4BF
:1046880030E70205F0748025F020D10495F095F00C
:0A469800FCEA8BF0A430E70205F005
:1046A200748025F030D50495F095F0FBC3EC2F20F3
:1046B2006203C39F9FFFEB2E306103C39E9EFE20C9
:1046C2003C64200C0512475C406412473E405F1276
:1046D200F200E51EFD24FB50550E12F200ED24F609
:1046E200504C1E1F12F200ED24F150421E0F12F226
:1046F20000ED24EC50380F12F200ED24E7502F1F8A
:104702001F0E0E12F200ED24E250231E0F0F12F2C2
:1047120000ED24DD50180E12F200ED24D8500F1EC9
:104722001E1F1F02F20012473E4003799E0722E934
:10473200242AFFE82461FE12475C401DEF246040FA
:1047420018243F5013EE2460400F243F500AEF24F8
:10475200D6FFEE249FFEC322D322532CF8432C040F
:10476200EE10E706D2E7F404D261FE24D340EAEF6A
:1047720010E706D2E7F404C262FF24D340DBEFB5B0
:1047820006005003CED26070057480FE8062FF2462
:0D479200FD5060904848938EF0A4AAF033CB
:10479F00CA33CA33CA33CA33CA33FA904872938FB3
:1047AF00F0A433C5F033CA90489393FB1248109589
:1047BF0070500224B412F0BDEA8BF0A430E702056A
:1047CF00F0C3748095F020D50425F025F0FEEA8C17
:1047DF00F0A430E70205F0C3748095F030D10425C2
:1047EF00F025F0FFC3227A01EE6F70097B16BF022E
:1047FF00BB7A0380B7BF01047B0080B07B0D0A80BA
:10480F00ABE52C540723C390481A73800E800E809B
:10481F0024801E8010800A80108012EB22742D9B42
:10482F0022742D2B22745A9B22745A2B2274879B2D
:10483F002274872B2274B39B22FFFFCCAA92807124
:10484F00665D554E4944403C383533302E2C2A286E
:10485F00272524232221201F1E1D1C1B1A1A19185D
:10486F001817178181818282838384858687898A3D
:10487F008B8D8F90929496989B9D9FA2A4A7A9AC85
:10488F00AFB1B4B400010203040405060708090A16
:10489F000A0B0C0D0D0E0F0F101111121313141410
:1048AF00151516161612983312B191E4F5F7E4E5C3
:1048BF00F7D2B264C022203D071248B47003D23D34
:1048CF0022056D056D12B1917D008DF7E485F71FFF
:1048DF008DF7C3E5F79573F5188DF7E4E5F7957444
:1048EF00F5198DF7E4E5F78DF7C3E5F79576F51A2A
:0C48FF008DF7E4E5F79577F51B8DF7E4E5
:10490B00E5F78DF7E4E5F7F51E8DF7C3E5F7957A37
:10491B00F51C8DF7E4E5F78DF7E4E5F7D2B2543FDC
:10492B0030E50244C0955EF51D156D156DE510243F
:10493B00784001227E00AF55EF30E7011E0512E5EE
:10494B001FA2E592D5400EE515951EF515E51494BD
:10495B0000F514800BE515251EF515E43514F5143B
:10496B007800E51E600620D50318F404C39FF5F00C
:10497B00E89E30E701220513E5F0A42517F517E5AE
:10498B00F03516F51622303D03D23D221248B460A5
:10499B00F81248B460F3E546600A1248B460EA12B4
:1049AB0048B460E5056D056D056D12B1917D008D07
:1049BB00F7C3E5F79573F5188DF7E4E5F79574F5FF
:1049CB00198DF7E4E5F78DF7C3E5F79576F51A8DB5
:1049DB00F7E4E5F79577F51BD2B2156D156D156DEF
:1049EB0022307424129939C23D75101E1249912040
:1049FB003D167902124A58400CA806A907124731F6
:104A0B00400312F200D510E422200F4030123D205B
:104A1B0006CF304806200C03204FC6E546790260CE
:094A2B0014790614600F791614C9
:104A3400600A79361460057976147017129939C2B0
:104A44003D7896124991203D0A124A58400312F2C9
:104A540000D8F022532CF8AB18E519FC33926212FB
:104A64004AAABC002BEB89F053F00784FF24DF40F3
:104A74001FAB1AE51BFC339261124AAAAA47125DC6
:104A8400CDBC000CEB89F053F00784FE24DF500208
:104A9400D32274562F2062029F9FFF741F2E306111
:104AA400029E9EFEC322500312602FE920E40122DD
:104AB400C3EC13FCEB13FBE920E50122C3EC13FC6C
:104AC400EB13FBE920E60122C3EC13FCEB13FB22FE
:104AD40074542F2062029F9FFF741D2E3061029E2A
:104AE4009EFE2279B4203249201D46EFB50600927D
:104AF40060AC06AB074004AC07AB06904B36EC2326
:104B040004938BF0A4A9F0EC23938BF0A429F990DF
:104B14004B9693C9904C96E52C54079313E9500196
:074B2400F4904C9EF9E52C12
:104B2B005407932975F0B484A9F022FFFFFFFF7F90
:104B3B00FF55553FFF33332AAA24921FFF1C7119CF
:104B4B00991745155513B1124911110FFF0F0F0E80
:104B5B00380D790CCC0C300BA20B210AAA0A3D099B
:104B6B00D8097B092408D30888084207FF07C10727
:104B7B00870750071C06EB06BC06900666063E062A
:104B8B001805F405D105B005900572000000000072
:104B9B0001010101010101010102020202020202F3
:104BAB0002020303030303030303030404040404C7
:104BBB00040404040505050505050505050606069B
:104BCB000606060606060607070707070707070771
:104BDB000808080808080808080809090909090944
:104BEB00090909090A0A0A0A0A0A0A0A0A0A0B0B1C
:104BFB000B0B0B0B0B0B0B0B0C0C0C0C0C0C0C0CF2
:104C0B000C0C0C0D0D0D0D0D0D0D0D0D0D0D0E0ECA
:104C1B000E0E0E0E0E0E0E0E0E0F0F0F0F0F0F0FA2
:104C2B000F0F0F0F0F10101010101010101010107E
:104C3B00101011111111111111111111111111125A
:104C4B001212121212121212121212121313131335
:104C5B001313131313131313131313141414141414
:104C6B0014141414141414141414151515151515F3
:104C7B0015151515151515151515161616161616D3
:104C8B00161616161616161616161600FFFF00FF2A
:104C9B000000FF002EB5875B2D5A88E537606C143A
:104CAB006036B402507F347E12E53424375046F818
:104CBB00904DE812E8FBE824FC501179A1E77E0542
:104CCB0090BC8A20E70390BC940F803A24040F7E9B
:104CDB002312E8BCD26480627F357E02E534243730
:104CEB00401410641090BB8D30081B1281497E1A42
:104CFB0090BF3A801122700590BB9F800990B8112C
:104D0B00200C0390B81D12814980C97F35E53424EE
:104D1B0033402A2404501B7D0F600C7D1E1460074A
:104D2B007D3C1460027D78ED305D02C3137E2B1247
:104D3B00E7827E0090BBA012814902F16E7E0524B2
:104D4B00FE500590B9F4800990B7F4200F0390B88A
:104D5B000012814980E4E546604A14603C14602EE1
:104D6B0014602014601290C171205D41904DE17F61
:104D7B00367E3412E8FB803C90C171305D0390C1EC
:104D8B006D802A90C16D305D0390C169801F90C109
:104D9B0069305D0390C165801490C165305D0390EF
:104DAB00C161800990C15D305D0390C1597F367E32
:104DBB003312817C7E3C7422305D02748302E8CF17
:104DCB00305D0890C149305BE4800690C151205B97
:104DDB00DC90C14D80D70508B28D8DB5BA09100690
:104DEB00000A10F248922492249224F2480A1006E8
:0E4DFB0000305E5220434F20284CE55864FFE4
:104E09006046E54824F640407F3FE55804F9C23D35
:104E1900124E52121BAB601AB404047401D23D75D0
:104E2900F003A4243CB5070A7E3A303D027E3612CF
:104E39004E540F0F0FD9D7E55975F003A4243EFF3F
:104E4900124E520F0F124E52227E3D12F2000EBE2A
:104E590040F922C248C249305E56202853E55864B9
:104E6900FF604DE54824F64047121BAB6042D2492A
:104E7900B40402803B1465597036D248304E31E58E
:104E8900596558602B307428124EBF121861E5BF5E
:104E9900B4011DE5BD20E618202416205F129006F6
:104EA900E4E0700CA3E024CE400624255002055905
:104EB90022305FFC80E820113375A7009006E4E0FA
:104EC9007028A3E0302402F404305F02F4042404BF
:104ED900F924F74015E924FC4003D26C2270012221
:104EE900306C097536A7D22ED22FC26C22305E08DB
:104EF900307405E558B4FF0122C244C24D780075EB
:104F0900A70475830712523E88188A1E8E168F17BA
:104F1900C23EC23BE54824F65003024FCFD23EE5DC
:104F29005860F7E8655970F22048EF12508430D183
:074F39003BAE16AF17A818EC
:104F4000E54670551207D2E5CC49604DD244E5CC18
:104F50007033E924CD402EE975F038A4ACF0FB1293
:104F60005FBE125FBEEBFDF511124FE5304D2CC256
:104F700006C23B8043E546705C1207D2E5CC700563
:104F8000E924CD50501259AF75A704758307A818AE
:104F900012523E8A1E8E168F178037121861E5BD99
:104FA000A2E0B3923B50113074281247314026A939
:104FB00007A806D20612DDEB125001124FF812506C
:104FC00041890788061E1F90523912E8FB8006307F
:104FD000D103125019A81808C3E558984003024F8E
:104FE0000875A7002274562F2062029F9FF9741F34
:104FF0002E3061029E9EF822E51865586001227DE0
:10500000057A00EA12F0BD12F1C30A0AED24F2405B
:10501000020A0AEA244C50EB22AE16AF17124AD409
:105020001E303E021E1EE51E12E89DEE2404FEE523
:105030001212E89D303E09EE2404FEE51312E89DAD
:1050400022E5186558603CC001C000C012C013853D
:1050500018101251BCD013D012D000D001E510307E
:075060003B07C395705002ED
:1050670024B412F0BD203B07AE16AF17124FE5E58B
:10507700112402FD7A0612F1C31DDAFA22121BABC4
:10508700B40457E8705412187FE5BD604D78C6A682
:105097001308A61208A62C12DB8675A704758307CA
:1050A7007510011264FB12DB8015101264FB12618C
:1050B700158E628F6312619D8B1C8A1B12DB8C20FD
:1050C700320E12516C203B08D24D1271461250E23B
:1050D70078C6861308861208862C2212187FAABD66
:1050E7007C027BB3125DCD8C128B13AA1DA91F12F4
:1050F7005E0FA91CA81B125F488C1D8B1FAC12AB3F
:1051070013AA19A91A125E0FA91CA81B125F488CB3
:10511700198B1AE56E251AF9E56D3519F8C3E56E91
:10512700951AFBE56D9519FAC3E554951FFDE56FD3
:10513700951DFCE554251FFFE56F351DFEE52C2366
:10514700652C30E206ECCEFCEDCFFD75A70490058B
:10515700C2E8F0E9F0ECF0EDF0EAF0EBF0EEF0EF9A
:10516700F075A70022D23BC3E5649573C5659574B6
:0E517700F564E5669575600404600822E56441
:1051850024E0500822E5642420400122C3E5679508
:1051950076F567E5689577F566E5699578600904BC
:1051A500600122E566F48002E5668562F0A474E09C
:1051B50025F04002C23B2212DB8675A704758307E2
:1051C5001264FB12DB8005101264FBC02C126514FF
:1051D500D02C891002DB8C30125120064E780075D8
:1051E500A70475830612523E30D139124AD4E546DA
:1051F50024FE500A0E0F90523412E8FB8026EA7006
:1052050007745D12E899801C75F06484ADF0700F29
:10521500ED75F00A847008E5F00E12E88A80051E27
:10522500ED12E81D08C3E55A9850B475A70022038E
:105235000340A040030340E040D2D1E8C4F582E03A
:10524500FA797312529730D146AF06532CF8EDBF59
:10525500FF07F40460390FD262BF00331253CB400D
:105265002E797612529730D126E5822403F582E015
:10527500F512E0F513EEA2E713FEED13BEFF07F4FA
:1052850004600C0ED261BE00061253E8400122C232
:10529500D122C3E09709FDE09709FEE09760090474
:0352A500700AEE9E
:1052A80030E7068007EE30E703C2D122E546600EFC
:1052B80014600BF9EDCEA2E713CE13D9F8FD227CCA
:1052C800007B44E54660207C007BCC1460197C019F
:1052D8007B981460127C037B3014600B7C067B6027
:1052E8001460047C0C7BC08C148B157AE9125DA4C5
:1052F800A847125F468C168B1775C70075C60475CC
:1053080010DF75B901E5BC20E76FF51385BD1205FF
:10531800C605C675B901532CF8C3E5BE9573FBE500
:10532800BF9574FC05C675B901E5BC9575FD5005BA
:10533800D262126037C3E5159BE5149CE49D4033A7
:105348008C198B18C3E5BD9576FBE5BE9577FCE512
:10535800BF9578FD5005D261126037C3E5179BE50C
:10536800169CE49D400D8C1B8B1A125392E5322437
:1053780028401305C6E5C68006E5C62404F5C670B0
:105388000205C7D510012202530AAE19AD181252F0
:10539800B4ED1253CBAE1BAD1A1252B4EE13ED138B
:1053A8001253E8124AD4E54624FB50080E0F9052D7
:0B53B8003902E8FB1EE51312E89DEE31
:1053C3002404FEE51202E89D75F0067FFDA946B9A7
:1053D300000575F0027FFF84C5F02F500205F0C56C
:1053E300F0FF24DE228547F0A430E70205F0E5F064
:1053F300A946B9000280050475F00384FE24E02267
:10540300E537B4020122E5377002D2396402700233
:10541300C239E53724FC799EE76005640B600C22F2
:10542300D27E20081E401C107F1022D27F2008133A
:105433004011107E01227537012275370020390390
:105443007537022275FB0075F9FF802775FBFF7521
:10545300F9FF801F1220C32053F2125488759E85D2
:10546300759D2D8014125488759E84759D2D800919
:10547300125488759E83759D09C2AC759852C26D8E
:10548300C26EC26F22C25375FBFF75F90022C23D83
:105493001254F6203D012275BC4175BD3075BE30F6
:1054A30075BF301228297F5A90B7021281377F6463
:1054B30090B70E1281377F6E1254FB7E20A8BC1268
:1054C3008F6188BC7E26A8BD128EAA88BD7E2CA8BB
:1054D300BE128EAA88BE7E32A8BF128EAA88BF12C1
:1054E300288912F16E1000051002B880F81255F7E2
:1054F30012F2E51218897F4B7E0890C13912814957
:105503007E20E5BC12E8CF12552E7E26E5BD12E8BB
:08551300CF1255377E2CE5BED6
:10551B0012E8CF1255377E32E5BF12E8CF1255375E
:10552B0002F16E24BF500E24E6400A2224D050050F
:10553B0024F6400122D23D2275C70375C6FE1280A8
:10554B00B51255F775C6FC75BC2675BD6475BEA93D
:10555B0075BF701255F775C6FB1280B575BC64121A
:10556B0055F775C6FA75BC1475BD1475BE0075BFBD
:10557B000C1255F775C6F975BC4E75BDBF75BE00DF
:10558B0075BF191255F775C6F875BC0A75BD7E75D2
:10559B00BE0075BF011255F775C6F775BC0175BD19
:1055AB002375BE4575BF671255F775C6F675BC02F8
:1055BB0075BDAB75BE0175BF011255F775C6F512FA
:1055CB0080B575BE0275BF0A1255F775C6F4128009
:1055DB00B575BCE11255F775C6F31280B11255F7CC
:1055EB0015C61255F715C61255F715C675B90575BB
:1055FB00B902227515001287B475B901E5BC648137
:10560B0060031280980515E515242050E975C70332
:10561B0075C68075B90505C6E5C6241C50F512562E
:10562B002F028606E4F5C7F5C674261280B675BD43
:10563B004E125649125646E41256461280B6125571
:10564B00F705C6227F3E7E00E54B12E8397E10E55A
:10565B004C12E8397E20E54D12E8397E30E54E12CA
:10566B00E839227F467E00E56C12E8397E10E56B47
:10567B0012E8397E20E56A12E8397E30E57F12E8C0
:0E568B0039227F2E12189812289C40167F2D6F
:1056990012812E1256B012185CE4F5BCF5BD75BE28
:1056A900021255F70205227F0E756F0280057F02EF
:1056B900756F00E4F56EF56D740612998674D8124B
:1056C90099BED2B2129B37056FDFED22E4F56CF576
:1056D9006B756A00E56B700C7F797E32E56C12E7B9
:1056E900DC12F16E12B16AE56B2404F56BE4356CDA
:1056F900F56C30E7DF2212570502027012F2E57FDE
:105709005A7E0590BF4912814912F16E12B23BD2FD
:1057190020C210D214D215C25512188E85BF6C85BD
:10572900BE6BE56B540360051297FA80F5856CBF73
:10573900856BBE75B90575B902129AC6125FA17B50
:1057490017756F7FE4F56EF56D758002C2B275F756
:1057590053856FF7856EF7856DF7A4D2B212B10341
:10576900BB172B756A007539FC75F08412B17F7C03
:1057790007783986F708DCFBD2B2756A1E75F084A2
:1057890012B17F8EF7A48FF7A4D2B2756A0012B155
:105799006A12B0FDE56E2404F56E7C041297FADCFA
:1057A900FBDBA612188E85BEBC85BFBD856BBE8589
:1057B9006CBF75B90575B90279B877C309A73A09F4
:1057C900A73B09A73C09A73D09A73E097700097727
:1057D900180977050977CE09772709773B09775B98
:1057E90009770009A7BD09A7BC129AC6029AEDD28A
:1057F90014D215125806C214C21502023D756F0063
:10580900756E00756D0074031299BE784075A70016
:10581900900700E4F5F7C2B2C2B2E5F7F0A3D8F3F6
:10582900D2B212F2E585354B856F4C856E4D856D8B
:105839004E7F0012565175A70090070078107F0916
:10584900E8540370020F0FE0F54BA3E0F54CA3E019
:10585900F54DA3E0F54EA3C083C082125651D08204
:10586900D083EF2407FFD8D812F16E100009100178
:105879002F10020280F522100214E5352496400209
:10588900800C756D00536EFCE56E24FC800AE56D95
:1058990024C0F56DE56E34FFF56EE56F34FF8026A3
:1058A900100214E53524964002800C756D00536E84
:1058B900FCE56E2404800AE56D2440F56DE56E343F
:1058C90000F56EE4356F540FF56F02580FD214D2FC
:1058D900151258E4C214C21502023D756F00756EA7
:1058E90000756D0012B191784075A700900700E42A
:1058F900F5F7E4E5F7F0A3D8F6D2B212F2E585356B
:105909004B856F4C856E4D856D4E7F0012565175D6
:0F591900A70090070078107F09E8540370020F71
:105928000FE0F54BA3E0F54CA3E0F54DA3E0F54EF1
:10593800A3C083C082125651D082D083EF2407FFC0
:10594800D8D812F16E10000910012F10020280F54C
:1059580022100214E53524964002800C756D005320
:105968006EFCE56E24FC800AE56D24C0F56DE56EDD
:1059780034FFF56EE56F34FF8026100214E53524F8
:10598800964002800C756D00536EFCE56E24048011
:105998000AE56D2440F56DE56E3400F56EE4356F6B
:1059A800547FF56F0258ED20740122D24475A70088
:1059B800758307E559C454F02407F582E0F51A24E5
:1059C8004C40E7A3E0F512A3E0F5131207D289389B
:1059D800121861E5BDA2E0923BE51A4006957050A9
:1059E8000224B4F51A203B05D20612DDEBE51A12A3
:1059F8005B12E5152437F51DE43514F51CE517246D
:105A080037F51FE43516F51E85CC12853813AC1210
:105A1800AB137A04125D9675380124FA401A0538DA
:105A28002402401405382401400E053805382401A5
:105A38004006053805380538C3E51A945A5002243B
:0E5A4800B4F51AC23BC23CC23D751B00A23B26
:105A5600823C406D203B2CE51A75F008A4951BFB93
:105A6600E5F0303D04940180029400FC5008EB24DC
:105A7600A0FBEC3405FC125B19125AC8923B40039A
:105A8600125AEB203C2CE51A75F008A4251BF9E404
:105A9600303D010435F0FAE994A0FBEA9405FC5088
:105AA60004AB01AC02125B19125AC8923C400312B5
:105AB6005AEBE51B2538F51B5094203D04D23D805A
:105AC6008D22E51F2517FEE51E35167016EE24916C
:105AD6004011E51D2515FFE51C35147006EF2491D0
:105AE600400122D3228E027C8A7B3B125DA4ED24E8
:105AF60002FE8F027C8A7B3B125DA4ED2439FF02F5
:105B0600F20012610880311260FB804675F008A42D
:105B1600ACF0FB751900C3EB9468F9EC9401FA40FC
:105B2600080519AC02AB0180ED8C108B11531903DB
:105B3600E51920E0CD1260FB125B6DAF05E5192477
:105B4600FE500312601F8E168F17E51920E0B8125B
:105B56006108125B6DAF05E5191460061460031247
:105B6600601F8E148F1522AC06AB07AA12A913026A
:055B76005E0F125C5AF5
:105B7B00203D4974857F227E0812E8CF7E083017BE
:105B8B003CAC1EAB1FEB2418EC34FC402F125D75A4
:105B9B00E51B60077F207E0812E8EA7F207E10E578
:105BAB001A12E8EA7F237E17742E12E8CB7F207E31
:105BBB001BE51B7011E519C2E012E8EA227F207E7B
:105BCB000E740A02E8EAE51975F0058475F005A470
:105BDB0002E8EA125C5A203D5E74857F227E3A12FF
:105BEB00E8CF301753AC1EAB1FEB2418EC34FC4042
:105BFB0046EC7033EB249C402E7E2D125C4C125FD6
:105C0B00BEC0E07F2A7E2EEB12E8EA7E39D0E0C2DE
:105C1B00E012E8EA7F347E3712F2001E12F2001F08
:105C2B0012F2000E02F2007E30125C4C125FBEEBE1
:105C3B007F2A7E3112E1DD227F2A7E39740A02E847
:105C4B00EA7F2912F2300FBF34F90EBE40F322D295
:105C5B003D30126612186BE5BDF51C75F00AA4F801
:105C6B0024E15002781EE4FCFBFEFFC23D12993981
:105C7B00125CC6203D44D8F8751DCEE51C14600996
:105C8B00751D9C146003751D6AC217EC30E705D2B5
:105C9B001712602F8C018B00E9487003D23D22EE66
:055CAB007008EF251D4B
:105CB0004003D23D22AC06AB077A1C125DA4125FF2
:105CC000488C1E8B1F22203D071248B47003D23D22
:105CD00022056D12B191E4F5F7C2B2C2B2ADF7F58B
:105CE000F7C2B2C2B2E5F7FAD2B230E4E3ED2FFF69
:105CF000E43EFEE56D2408F56D12B191E4F5F7C2BE
:105D0000B2C2B2ADF7D2B2EA30E508EB2DFBEC340B
:0C5D100000FC22C3EB9DFBEC9400FC2285
:08F308000000000000000000FD
:00000001FF
